:100000000C94712D0C94A22D0C94A22D0C94A22D65
:100010000C94A22D0C94DF670C94A22D0C94A22DAD
:100020000C9460670C94A22D0C94A22D0C940FC913
:100030000C94A22D0D9434BB0C94A22D0C94A22DE3
:100040000C94A22D0D94F51C0C94A22D0C94A22DB1
:100050000C94A22D0C94A22D0D945D330D945BB3E2
:100060000C94A22D0C944B3F0C94A22D0C94A22D19
:100070000C94A22D0C94A22D0C94A22D0C94A22DC4
:100080000C94A22D0C94A22D0C94A22D0C94A22DB4
:100090000C94A22D0C94A22D0C94A22D0C94A22DA4
:1000A0000C94A22D0C94A22D0C94A22D0C94A22D94
:1000B0000C94A22D0C94A22D0C94A22D0C94A22D84
:1000C0000C94A22D0C94A22D0C94A22D0C948B3F79
:1000D0000C94A22D0C94A22D0C94A22D0C94A22D64
:1000E0000C94A22D4E3E523E573E5F3E743E8D3ED6
:1000F000B23EDC3E0F025101E3016101B301EF01A9
:100100007101AB01F70167014701E901DB01AF01B3
:10011000FF01C701F101ED01E1018B016B01CD018F
:10012000BF015901D3014B01F901BB0153015D012D
:100130009D01D101CF01FB01CB017B01B901F5018B
:100140000702070207023F013F013F015F015B0118
:100150003F013D01A101B5011302C9017701DF0192
:10016000010273018D018F0183014D01110295017F
:10017000DF0115026F0135019B010B02910137016F
:1001800087010902890105023B013901E501A50149
:10019000C50149010902FD01B1019901084AD73B96
:1001A0003BCE016E84BCBFFDC12F3D6C74319ABD46
:1001B00056833DDA3D00C77F11BED9E4BB4C3E916A
:1001C0006BAAAABE000000803F05A84CCDB2D44E59
:1001D000B93836A9020C50B9918688083CA6AAAA5B
:1001E0002ABE000000803F07634236B79BD8A71A9B
:1001F00039685618AEBAAB558C1D3CB7CC5763BDA9
:100200006DEDFD753EF6177231BF000000803F08AE
:10021000000000BE922449123EABAAAA2ABECDCC51
:10022000CC4C3E00000080BEABAAAAAA3E00000053
:1002300000BF000000803F0000000000084178D3AC
:10024000BB4387D1133D190E3CC3BD4282AD2B3E4B
:1002500068EC8276BED98FE1A93E4C80EFFFBE01EB
:10026000C4FF7F3F0000000000000D9429B50D94ED
:100270004BB50D946AB50D9466B50D9473830D94CA
:1002800087830D94BE970D9465670D9408720D9445
:1002900068340D947CB50D9476810D94F2B40D9470
:1002A000D06E0D94F0330D94B6810D9418680D94B2
:1002B000065A0D948A6B0D9497830D94CA810D9400
:1002C00069830D941A340D94E7650D9488A80D94F4
:1002D00066340D94A3770D94516B0D945DA30D942A
:1002E0001FB50D945C340D94CCB40D94C25B0D9489
:1002F000BAB40D9472560D9428830D9433A00D94C6
:100300004C640D94B0510D94E8B40D94B4470D9421
:1003100051B50D945CB50D944C6B0D94D4B40D9403
:10032000DEB40D9447B50D94A1440D940BB50D9416
:10033000B0440D948AB50D9455B50D94E7810D9494
:100340005C670D949CB40D946D6A0D9474B50D9416
:10035000B6440D941B4B0D9460340D94FB560D94D4
:100360009E340D9486B50D9434340D94A1B40D943F
:10037000CF8F0D9451830D94A2810D94A6960D9468
:10038000756B0D9444690D9479420D9478B50D9474
:10039000E06A0D94B0B40D94FF820D945B6B0D94E4
:1003A000D1820D94AF820D945E810D9475510D94A0
:1003B00026B60D94FB400D9490340D9418440D9482
:1003C00033B50D94276B0D940C340D946EB50D94CC
:1003D00053670D9476340D946E670D940D6B0D94E8
:1003E00042340D94F56A0D94D71F0D9459830D94E2
:1003F00062340D948D810D94E2820D9482B50D943A
:10040000BE340D94C4B40D946E9B0D9460B50D94E0
:1004100061830D948FB50D9458B50D943B460D94A2
:10042000E2330D9401B50D94A6B40D9415B5486151
:100430007264636F6465642044656661756C7420E2
:1004400053657474696E6773204C6F6164656400F2
:1004500053746F7265642073657474696E6773207A
:1004600072657472696576656400202020452F44AA
:10047000203D20002020204D393030204B004C6999
:100480006E65617220616476616E63652073657468
:1004900074696E67733A0046696C616D656E7420AD
:1004A00073657474696E67733A2044697361626C32
:1004B0006564002020204D32303020440046696CB5
:1004C000616D656E742073657474696E67733A004C
:1004D0002020204D3230392053004175746F2D5249
:1004E0006574726163743A20533D3020746F2064E8
:1004F000697361626C652C203120746F20696E74A1
:1005000065727072657420657874727564652D6F9C
:100510006E6C79206D6F76657320617320726574DF
:100520007261637473206F72207265636F76657297
:10053000696573002046002020204D32303820535A
:10054000005265636F7665723A20533D4578747248
:1005500061206C656E67746820286D6D2920463AAD
:10056000537065656420286D6D2F6D2900205A0039
:100570002046002020204D32303720530052657431
:10058000726163743A20533D4C656E67746820282D
:100590006D6D2920463A537065656420286D6D2F76
:1005A0006D29205A3A205A4C69667420286D6D29AD
:1005B000002044002049002020204D3330342050BA
:1005C00000504944206865617462656420736574F5
:1005D00074696E67733A002044002049002020208F
:1005E0004D33303120500050494420736574746994
:1005F0006E67733A00205A0020590020204D323097
:1006000036205800486F6D65206F666673657420EC
:10061000286D6D293A00204500205A0020590020FD
:10062000580020420020540020204D323035205305
:1006300000416476616E636564207661726961620F
:100640006C65733A20533D4D696E20666565647232
:1006500061746520286D6D2F73292C20543D4D69E0
:100660006E2074726176656C206665656472617473
:100670006520286D6D2F73292C20423D6D696E69B0
:100680006D756D207365676D656E742074696D6539
:1006900020286D73292C20583D6D6178696D756D2A
:1006A000205859206A65726B20286D6D2F73292C94
:1006B00020205A3D6D6178696D756D205A206A65FC
:1006C000726B20286D6D2F73292C2020453D6D61A4
:1006D00078696D756D2045206A65726B20286D6D97
:1006E0002F73290020540020204D32303420530035
:1006F000416363656C65726174696F6E3A20533D46
:10070000616363656C65726174696F6E2C20543D22
:100710007265747261637420616363656C65726194
:1007200074696F6E00204500205A00205900202077
:100730004D3230312058004D6178696D756D204122
:100740006363656C65726174696F6E20286D6D2FCF
:100750007332293A00204500205A002059002020F9
:100760004D3230332058004D6178696D756D2066CB
:10077000656564726174657320286D6D2F73293A05
:1007800000204500205A0020590020204D393220F9
:10079000580053746570732070657220756E6974AB
:1007A0003A0053657474696E67732053746F726591
:1007B0006400454550524F4D204572726F72004D96
:1007C0006561737375726520617667203D202564CD
:1007D0000A004432313330202D20544D433231331E
:1007E000300A0074656D705F70696E64613D2564E8
:1007F000206F66667365745F7A3D25642E253033FD
:10080000640A0074656D705F70696E64613D256493
:10081000432074656D705F73686966743D25647507
:100820006D0A0063616C5F7374617475733D256458
:100830000A004438202D20526561642F5772697474
:10084000652050494E44410A000020006D657368E0
:1008500020626564206C6576656C696E673A20007D
:1008600029002C20002C2000706879736963616C6A
:1008700020636F6F7264696E617465733A2028003B
:1008800029002C20002C2000776F726C6420636F8D
:100890006F7264696E617465733A202800204600A7
:1008A0002045004731205A004D3234004D32362069
:1008B00053256C75004D31303620530047312046AA
:1008C0002564004731204531204634383000473117
:1008D000205A002046323030300020590047312065
:1008E00058004D383300506F736974696F6E207211
:1008F0006561642066726F6D20656570726F6D3A18
:10090000004D3233202573002E67636F0046656506
:1009100064726174653A007265636F7665725F6DCB
:10092000616368696E655F73746174655F61667445
:1009300065725F706F7765725F70616E69632C209E
:10094000696E697469616C20007265636F766572A7
:100950005F6D616368696E655F73746174655F6123
:10096000667465725F706F7765725F70616E6963E0
:100970002C20696E697469616C20007265636F7602
:1009800065725F6D616368696E655F7374617465DC
:100990005F61667465725F706F7765725F70616EBC
:1009A00069632C20696E697469616C2000637572DB
:1009B00072656E745F706F736974696F6E5B5A5F96
:1009C000415849535D3A0043757272656E742070E8
:1009D0006F736974696F6E20595F415849533A00CB
:1009E00043757272656E7420706F736974696F6E8F
:1009F00020585F415849533A004166746572207728
:100A0000616974696E6720666F722074656D703AF3
:100A100000473120452D3120463438300047312001
:100A200045352046313230004D3833004D313930B4
:100A300020532564004D313039205325640047325E
:100A40003820582059004731205A32352046383056
:100A500030004D31343020532564004D3130342086
:100A600053256400494E54340055564C4F202D20D8
:100A7000656E6400737470730055564C4F002042CD
:100A80003A0020453A00543A005A206C69766520B5
:100A900061646A757374206F7574206F662072616B
:100AA0006E67652E2053657474696E6720746F20BD
:100AB000302E20436C69636B20746F20636F6E74FB
:100AC000696E75652E005A206C6976652061646ACE
:100AD000757374206F7574206F662072616E676520
:100AE0002E2053657474696E6720746F2030002067
:100AF000573A0020453A00543A004B494C4C3A20B2
:100B0000004175746F0020452F443D0041647661BB
:100B10006E6365204B3D0022283229005400496E47
:100B200076616C6964205420636F64652E00496EA1
:100B300076616C6964204D20636F64652E004D32D0
:100B400032302053256900203A2000004C414E47A6
:100B50002053454C20464F5243454400222831291A
:100B60000020453A00205A3A0020593A0020453AE0
:100B700000205A3A0020593A00583A004D3131339A
:100B800020530020002E0020423A0020453A005415
:100B90003A0020413A0020503A002042403A0020DA
:100BA000403A00202F003A00205400202F0020421D
:100BB0003A00202F006F6B20543A002569206D69A0
:100BC0006E2C2025692073656300496E76616C691F
:100BD00064204D20636F6465004D65736820626515
:100BE00064206C6576656C696E67206E6F74206139
:100BF00063746976652E000A002020000A4D656145
:100C0000737572656420706F696E74733A000A5A66
:100C100020736561726368206865696768743A204B
:100C2000002C004E756D20582C593A2000476F203B
:100C3000686F6D652066696E6973686564004D65EF
:100C4000736820626564206C6576656C696E6720E8
:100C500061637469766174656400557073616D7069
:100C60006C652066696E697368656400426564201E
:100C70006C6576656C696E6720636F72726563740C
:100C8000696F6E2066696E697368656400206D69BE
:100C900063726F6E73004578636573736976652060
:100CA000626564206C6576656C696E6720636F723F
:100CB00072656374696F6E3A200062616279737461
:100CC0006570206170706C69656400636C65616E4D
:100CD0002075702066696E69736865642000002065
:100CE0006F66667365743A20006D6573682062658F
:100CF00064206C6576656C696E673A20004732380F
:100D0000205730003A200054656D7065726174752B
:100D100072652063616C6962726174696F6E2064D0
:100D20006F6E652E20436F6E74696E7565207769EE
:100D30007468207072657373696E672074686520CB
:100D40006B6E6F622E0000205A20736869667420F3
:100D5000286D6D293A0050494E44412074656D70EC
:100D6000657261747572653A2000002F3600537405
:100D700065703A200000205A207368696674202844
:100D80006D6D293A0050494E44412074656D70657F
:100D90007261747572653A20002F362028736B6972
:100DA000707065642900537465703A2000005A45DC
:100DB000524F3A20000073746172742074656D7034
:100DC000657261747572653A200050494E44412045
:100DD00070726F62652063616C6962726174696FC1
:100DE0006E20737461727400473238205730000AE5
:100DF00000205A3A200020593A200020583A20007A
:100E00004732382C2066696E616C20004732382CDE
:100E10002066696E616C20004732382C2066696E4E
:100E2000616C20004732382C20696E697469616CEE
:100E300020004732382C20696E697469616C20008B
:100E400043524153485F4445544543544544004D43
:100E5000323900627573793A207061757365642068
:100E6000666F7220696E70757400627573793A20CE
:100E700070617573656420666F72207573657200AA
:100E8000627573793A2070726F63657373696E6708
:100E9000002055706C6F616420696E2070726F67FE
:100EA0007265737300696E697469616C207A73741A
:100EB0006570732061667465722072657365743A3B
:100EC0002000696E697469616C207A73746570734F
:100ED000206F6E20706F7765722075703A20004623
:100EE0006163746F7279205245534554004E6F769A
:100EF000203237203230313700436F6D70696C65B6
:100F0000643A2000286E6F6E652C206465666175FA
:100F10006C7420636F6E66696729004E6F762032AD
:100F20003720323031372031363A33363A343600D2
:100F30007374617274001B5B324A1B5B313B314836
:100F40004F726967696E616C2050727573612069B8
:100F5000331B5B323B3348507275736120526573AB
:100F60006561726368002500202020202020002079
:100F700020202020200045524153494E4720616CDB
:100F80006C206461746100466163746F72792052F1
:100F9000455345540043524153485F5245434F56D1
:100FA000455200473238205900473238205800FF58
:100FB000FFFF0000A0400000A04000000040000033
:100FC0007F43000056439AD95143000000000000BF
:100FD00080C09A99193E00007F43000052430000F0
:100FE000524300000000000080C09A99193E6563DA
:100FF000686F3A004572726F723A00000021104229
:101000002063308440A550C660E770088129914A6A
:10101000A16BB18CC1ADD1CEE1EFF13112100273F1
:10102000325222B5529442F772D662399318837BBA
:10103000B35AA3BDD39CC3FFF3DEE3622443342041
:10104000040114E664C774A44485546AA54BB5280A
:10105000850995EEE5CFF5ACC58DD55336722611D1
:10106000163006D776F6669556B4465BB77AA7195A
:10107000973887DFF7FEE79DD7BCC7C448E5588699
:1010800068A7784008611802282338CCC9EDD98EAA
:10109000E9AFF9488969990AA92BB9F55AD44AB731
:1010A0007A966A711A500A333A122AFDDBDCCBBFFA
:1010B000FB9EEB799B588B3BBB1AABA66C877CE401
:1010C0004CC55C222C033C600C411CAEED8FFDEC4A
:1010D000CDCDDD2AAD0BBD688D499D977EB66ED511
:1010E0005EF44E133E322E511E700E9FFFBEEFDD9A
:1010F000DFFCCF1BBF3AAF599F788F8891A981CA77
:10110000B1EBA10CD12DC14EF16FE18010A100C255
:1011100030E3200450254046706760B9839893FB04
:10112000A3DAB33DC31CD37FE35EF3B1029012F3A5
:1011300022D2323542145277625672EAB5CBA5A854
:101140009589856EF54FE52CD50DC5E234C324A0F5
:101150001481046674476424540544DBA7FAB799E4
:1011600087B8975FE77EF71DC73CD7D326F2369145
:1011700006B01657667676154634564CD96DC90EAC
:10118000F92FE9C899E9898AB9ABA9445865480695
:10119000782768C018E1088238A3287DCB5CDB3F44
:1011A000EB1EFBF98BD89BBBAB9ABB754A545A37E5
:1011B0006A167AF10AD01AB32A923A2EFD0FED6C14
:1011C000DD4DCDAABD8BADE89DC98D267C076C6435
:1011D0005C454CA23C832CE01CC10C1FEF3EFF5D24
:1011E000CF7CDF9BAFBABFD98FF89F176E367E5585
:1011F0004E745E932EB23ED10EF01E7C3C3E5E2BB2
:101200003D3F2F5B5D3B2C2A225C004D383420583B
:101210002059205A2045004D3234004D32332025CC
:1012200073006175746F25692E67000A002F000A2C
:10123000002E0044656C6574696F6E206661696C90
:1012400065642C2046696C653A200046696C65200F
:1012500064656C657465643A002E002E002E002EC5
:10126000004E6F772066726573682066696C653A18
:1012700020004E6F7720646F696E672066696C6529
:101280003A20002220706F73002220706172656E18
:10129000743A2200535542524F5554494E4520430B
:1012A000414C4C207461726765743A220074727903
:1012B000696E6720746F2063616C6C207375622D9A
:1012C00067636F64652066696C657320776974680D
:1012D00020746F6F206D616E79206C6576656C731C
:1012E0002E204D4158206C6576656C2069733A005C
:1012F000256920686F757273202569206D696E7588
:101300007465730054494D454F55543A004D313181
:10131000300046756C6C20525820427566666572C6
:101320000022206661696C65643A204275666665D4
:10133000722066756C6C2100456E717565696E670B
:1013400020746F207468652066726F6E743A202274
:10135000002200456E717565696E6720746F207498
:1013600068652066726F6E743A20220022206661E2
:10137000696C65643A204275666665722066756CB4
:101380006C210022004D36303000507275736120A0
:101390006933204D4B33206F6B00507275736120A1
:1013A0006933204D4B332072656164792E007A5F7A
:1013B0006D696E3A20007A5F6D61783A20005A209C
:1013C0004F666673657400795F6D696E3A200079C7
:1013D0005F6D61783A20005920767A64616C656EA1
:1013E0006F7374206F64206D696E3A0059206469D0
:1013F0007374616E63652066726F6D206D696E3AFD
:1014000000416E6F0059657300785F6D696E3A2018
:1014100000785F6D61783A200044657461696C7989
:101420002058595A206B616C2E0058595A2063611C
:101430006C2E2064657461696C73004E796E69204E
:1014400070726F76656475207A206B616C69627268
:101450006163692E00492077696C6C2072756E207B
:101460007A2063616C6962726174696F6E206E6F5D
:10147000772E004E796E692070726F7665647520E4
:1014800078797A206B616C6962726163692E205A87
:10149000616265726520746F20707269626C697A2E
:1014A0006E65203132206D696E2E00492077696C9F
:1014B0006C2072756E2078797A2063616C69627233
:1014C0006174696F6E206E6F772E20497420776982
:1014D0006C6C2074616B6520617070726F782E2067
:1014E0003132206D696E732E004E796E69207072F4
:1014F0006564656872656A6920747279736B7520BA
:1015000070726F20504C412E004E6F77204920772B
:10151000696C6C2070726568656174206E6F7A7A90
:101520006C6520666F7220504C412E00446F6272D1
:10153000792064656E2C206A73656D207661736511
:10154000207469736B61726E61204F726967696E96
:10155000616C2050727573612069332E204368637B
:1015600065746520616279636820566173207072CA
:101570006F7665646C61206B616C69627261636E29
:10158000696D2070726F636573656D3F0048692CEB
:10159000204920616D20796F7572204F72696769EB
:1015A0006E616C20507275736120693320707269AE
:1015B0006E7465722E20576F756C6420796F75207C
:1015C0006C696B65206D6520746F20677569646553
:1015D00020796F75207468726F756768207468650C
:1015E0002073657475702070726F636573733F004C
:1015F0005A61636E75207469736B6E6F7574206CBD
:10160000696E6B752061205679206275646574651A
:1016100020706F737475706E6520736E697A6F7663
:10162000617420747279736B75206F746163656E79
:10163000696D20746C616369746B6120646F6B7594
:1016400064206E65646F7361686E657465206F7089
:1016500074696D616C6E69207679736B792E205098
:10166000726F686C65646E657465207369206F6263
:1016700072617A6B792076206E617369207072696D
:1016800072756363652076206B617069746F6C6539
:10169000204B616C69627261636500492077696CF7
:1016A0006C20737461727420746F207072696E7430
:1016B000206C696E6520616E6420796F7520776992
:1016C0006C6C206772616475616C6C79206C6F77EB
:1016D000657220746865206E6F7A7A6C6520627915
:1016E00020726F746174696E6720746865206B6E18
:1016F0006F622C20756E74696C20796F752072652D
:10170000616368206F7074696D616C2068656967DA
:1017100068742E20436865636B2074686520706967
:1017200063747572657320696E206F7572206861CD
:101730006E64626F6F6B20696E20636861707465A0
:10174000722043616C6962726174696F6E2E004E23
:10175000796E69207A6B616C696272756A6920764C
:101760007A64616C656E6F7374206D657A69206B45
:101770006F6E63656D20747279736B792061207070
:101780006F76726368656D20686561746265647503
:101790002E004E6F7720492077696C6C2063616C56
:1017A0006962726174652064697374616E63652037
:1017B0006265747765656E20746970206F66207449
:1017C0006865206E6F7A7A6C6520616E642068654A
:1017D000617462656420737572666163652E004E84
:1017E000656A6472697620706F6D6F6369207365D6
:1017F0006C667465737475207A6B6F6E746F6C753C
:101800006A69206E656A63617374656A73692063CF
:101810006879627920767A6E696B616A696369209A
:1018200070726920736573746176656E692074697E
:10183000736B61726E792E0046697273742C204945
:101840002077696C6C2072756E20746865207365F2
:101850006C667465737420746F20636865636B20B5
:101860006D6F737420636F6D6D6F6E206173736540
:101870006D626C792070726F626C656D732E0053AF
:1018800070757374656E692057697A61726461203E
:1018900076796D617A6520756C6F7A656E652076F4
:1018A00079736C65646B79207673656368206B610E
:1018B0006C69627261636920612073707573746909
:1018C000206B616C69627261636E692070726F6314
:1018D0006573206F64207A616361746B752E20508C
:1018E0006F6B7261636F7661743F0052756E6E69E3
:1018F0006E672057697A6172642077696C6C206426
:10190000656C6574652063757272656E74206361C1
:101910006C6962726174696F6E20726573756C7444
:101920007320616E642073746172742066726F6DCF
:101930002074686520626567696E6E696E672E2027
:10194000436F6E74696E75653F00436863657465C7
:10195000206F70616B6F76617420706F736C65645B
:101960006E69206B726F6B206120706F7A6D656E8F
:10197000697420767A64616C656E6F7374206D652E
:101980007A6920747279736B6F7520612068656164
:10199000746265643F00446F20796F752077616ED3
:1019A0007420746F20726570656174206C6173744B
:1019B000207374657020746F20726561646A75733A
:1019C000742064697374616E636520626574776501
:1019D000656E206E6F7A7A6C6520616E6420686532
:1019E00061746265643F0057697A61726461206D59
:1019F000757A657465206B64796B6F6C6976207A93
:101A00006E6F76752073707573746974207A206DAB
:101A1000656E752043616C6962726174696F6E20D6
:101A20002D3E2057697A61726400596F7520636199
:101A30006E20616C7761797320726573756D6520B6
:101A40007468652057697A6172642066726F6D20D0
:101A500043616C6962726174696F6E202D3E20571C
:101A6000697A6172642E004A6520746F20504C417F
:101A70002066696C616D656E743F004973206974FE
:101A800020504C412066696C616D656E743F00505A
:101A9000726F73696D20766C6F7A746520504C415B
:101AA0002066696C616D656E7420646F2065787462
:101AB0007275646572752C20706F20746520737464
:101AC00069736B6E65746520746C616369746B6FA8
:101AD0002070726F207A61766564656E6920666930
:101AE0006C616D656E74752E00506C656173652058
:101AF000696E7365727420504C412066696C616D2B
:101B0000656E7420746F20746865206578747275D2
:101B10006465722C207468656E2070726573732022
:101B20006B6E6F6220746F206C6F61642069742E1D
:101B30000050726F73696D207A61766564746520F8
:101B4000504C412066696C616D656E742061207037
:101B50006F207465206F626E6F7674652057697AA6
:101B60006172646120737469736B6E7574696D2042
:101B7000726573657420746C616369746B612E00A7
:101B8000506C65617365206C6F616420504C41201E
:101B900066696C616D656E7420616E642074686541
:101BA0006E20726573756D652057697A6172642065
:101BB0006279207265626F6F74696E672074686500
:101BC000207072696E7465722E005072656465686B
:101BD000726976616D20747279736B752E20507204
:101BE0006F73696D2063656B656A74652E00507252
:101BF0006568656174696E67206E6F7A7A6C652EB0
:101C000020506C6561736520776169742E004A65A8
:101C10002066696C616D656E74207A6176656465B5
:101C20006E3F0049732066696C616D656E74206C4F
:101C30006F616465643F00567365206A6520686F54
:101C4000746F766F2E00416C6C20697320646F6E28
:101C5000652E204861707079207072696E74696EAB
:101C600067210050726F73696D206F6369737465CB
:101C700074652068656174626564206120737469AD
:101C8000736B6E65746520746C616369746B6F2E21
:101C900000506C6561736520636C65616E206865DA
:101CA000617462656420616E64207468656E207082
:101CB0007265737320746865206B6E6F622E0050BE
:101CC000726F73696D206E61686C65646E657465B2
:101CD00020646F206D616E75616C752061206F707E
:101CE00072617674652070726F626C656D2E205023
:101CF0006F207465206F626E6F7674652057697A05
:101D000061726461207265626F6F746F76616E6973
:101D10006D207469736B61726E792E00506C656111
:101D2000736520636865636B206F75722068616EF0
:101D300064626F6F6B20616E6420666978207468DE
:101D4000652070726F626C656D2E205468656E2020
:101D5000726573756D65207468652057697A617264
:101D600064206279207265626F6F74696E67207497
:101D70006865207072696E7465722E0057697A61A9
:101D8000726400205761746368646F6720526573E2
:101D9000657400496E666F726D61636500496E66B9
:101DA0006F2073637265656E004B616C2E207072DC
:101DB000766E6920767273747679004669727374F0
:101DC000206C617965722063616C2E0057616974C3
:101DD00020666F7220757365722E2E2E00506F75FF
:101DE0007A69746520626568656D207469736B75C6
:101DF000005573656420647572696E67207072693E
:101E00006E740056796A6D6F75742066696C616DC9
:101E1000656E7400556E6C6F61642066696C616DEF
:101E2000656E74005679736F7576616D2066696CA6
:101E3000616D656E7400556E6C6F6164696E6720CC
:101E400066696C616D656E7400556E6B6E6F776E52
:101E500020636F6D6D616E643A2022004C6164698D
:101E6000740054756E650053442063617264205B96
:101E7000466C73684169725D00534420636172640B
:101E8000205B6E6F726D616C5D005465706C2E200E
:101E90006B616C2E205B4F4E5D0054656D702E2083
:101EA00063616C2E205B4F4E5D005465706C2E207C
:101EB0006B616C2E205B4F46465D0054656D702E45
:101EC0002063616C2E205B4F46465D005465706C4C
:101ED0006F746E69206B616C696272616365206406
:101EE0006F6B6F6E63656E612E20506F6B726163F6
:101EF000756A746520737469736B656D20746C61A9
:101F00006369746B612E0054656D706572617475E0
:101F100072652063616C6962726174696F6E2069B9
:101F2000732066696E69736865642E20436C69630B
:101F30006B20746F20636F6E74696E75652E00542C
:101F400065706C2E206B616C2E20202020202020BC
:101F50002020200054656D702E2063616C2E20209F
:101F60002020202020202020005465706C6F746198
:101F70000054656D706572617475726500506F64B0
:101F8000706F726100537570706F7274005A617374
:101F90007461766974207469736B0053746F702078
:101FA0007072696E740053544F505045442E200097
:101FB000537465707261746520746F6F206869670F
:101FC000683A2000497320737465656C20736865F6
:101FD0006574206F6E20686561746265643F0043BC
:101FE000656C6B6F767920636173203A00546F746F
:101FF000616C207072696E742074696D65203A009E
:1020000046696C616D656E742063656C6B656D20EF
:102010003A00546F74616C2066696C616D656E7412
:10202000203A00436173207469736B75203A202055
:10203000005072696E742074696D653A2020004604
:10204000696C616D656E74203A20200046696C6190
:102050006D656E7420757365643A20200053746159
:1020600074697374696B61202000537461746973BF
:10207000746963732020004572726F72202D207383
:102080007461746963206D656D6F72792068617326
:10209000206265656E206F7665727772697474650B
:1020A0006E00527963686C6F737400537065656479
:1020B0000020536F66747761726520526573657492
:1020C000004C65686B65207A6B6F73656E693A00CA
:1020D000536C6967687420736B65773A004D6F6461
:1020E000202020202020205B74696368795D004DEA
:1020F0006F646520202020205B73696C656E745DC1
:10210000004D6F6420205B7679732E2076796B6F9B
:102110006E5D004D6F6465205B6869676820706F55
:102120007765725D0053746176206B6F6E632E204D
:102130007370696E2E0053686F7720656E6420732C
:10214000746F70730054657A6B65207A6B6F73657A
:102150006E693A0053657665726520736B65773AF0
:10216000004E61737461767465207465706C6F7471
:10217000753A005365742074656D7065726174758D
:1021800072653A004E6173746176656E69005365DD
:102190007474696E6773004368796261207A617054
:1021A0006F6A656E6900576972696E672065727241
:1021B0006F720053656C662074657374207374616C
:1021C00072742020005A6B6F6E74726F6C756A7433
:1021D00065203A00506C6561736520636865636BC8
:1021E000203A0053656C662074657374204F4B0071
:1021F0004E657A61706F6A656E6F20202020004EF8
:102200006F7420636F6E6E6563746564004D6F74E8
:102210006F72004865617465722F546865726D69EC
:1022200073746F7200546573742076656E74696C94
:1022300061746F72750046616E207465737400532B
:10224000656C66746573742073656C68616C2020BE
:102250000053656C6674657374206661696C6564AF
:102260002020004C6576792076656E74206E6120A2
:102270007472797363653F004C65667420686F748F
:10228000656E642066616E3F0053656C66746573AD
:1022900074206572726F72202100456E6473746FD2
:1022A00070206E6F742068697400456E6473746F7B
:1022B000707300456E6473746F7000507265646E65
:1022C00069207469736B6F76792076656E743F0050
:1022D00046726F6E74207072696E742066616E3F14
:1022E000004B6F6E74726F6C61205A206178697355
:1022F000202000436865636B696E67205A2061780F
:1023000069732020004B6F6E74726F6C61205920CE
:1023100061786973202000436865636B696E67208C
:102320005920617869732020004B6F6E74726F6C56
:102330006120582061786973202000436865636BD1
:10234000696E67205820617869732020004B6F6E9A
:1023500074726F6C6120686F74656E642020004336
:102360006865636B696E6720686F74656E642020B2
:10237000004B6F6E74726F6C6120656E6473746F66
:10238000707300436865636B696E6720656E647384
:10239000746F7073004B6F6E74726F6C6120626546
:1023A00064202020202000436865636B696E6720ED
:1023B000626564202020202000567365204F4B204A
:1023C0002020202020202020202000416C6C206331
:1023D0006F727265637420202020202000426564A3
:1023E000202F204865617465720041786973206C04
:1023F000656E67746800417869730053656C667434
:10240000657374202020202020202020005772692E
:1024100074696E6720746F2066696C653A20007677
:102420006F6C756D652E696E6974206661696C6587
:1024300064002053697A653A20004B617274612010
:1024400076796A6D75746100436172642072656D9E
:102450006F766564005344207072696E74696E67AC
:10246000206279746520006F70656E206661696C0A
:1024700065642C2046696C653A20006F70656E5269
:102480006F6F74206661696C6564004B6172746182
:1024900020766C6F7A656E61004361726420696EAC
:1024A00073657274656400534420696E69742066B4
:1024B00061696C0046696C652073656C6563746561
:1024C000640046696C65206F70656E65643A200033
:1024D0006572726F722077726974696E6720746FAB
:1024E0002066696C650053442063617264206F6BE1
:1024F0000043616E6E6F7420656E74657220737533
:10250000626469723A200050726176793A005269C9
:102510006768743A004F626E6F766F76616E6920FD
:102520007469736B7500526573756D696E672070A1
:1025300072696E74004F626E6F76656E69207469A1
:10254000736B7500526573756D696E672070726983
:102550006E7400506F6B7261636F766174005265C8
:1025600073756D65207072696E7400526573656E67
:10257000643A2000506C656173652072656D6F76FA
:102580006520737465656C20736865657420667278
:102590006F6D20686561746265642E00426C6163D2
:1025A0006B6F7574206F636375727265642E205251
:1025B00065636F766572207072696E743F00526554
:1025C000636F766572696E67207072696E74202021
:1025D000202000686F77746F2E707275736133649A
:1025E0002E637A00686F77746F2E70727573613323
:1025F000642E636F6D00666F72756D2E70727573E9
:102600006133642E637A00666F72756D2E70727519
:10261000736133642E636F6D007072757361336420
:102620002E637A00707275736133642E636F6D0070
:102630005469736B20706F7A6173746176656E0094
:102640005072696E742070617573656400546973AB
:102650006B20707265727573656E005072696E746E
:102660002061626F72746564005072696E74657285
:1026700020646973636F6E6E6563746564006120C6
:10268000737469736B6E65746520746C61636974CF
:102690006B6F00616E64207072657373207468657F
:1026A000206B6E6F620050726564656872656A7453
:1026B0006520747279736B7521005072656865616D
:1026C0007420746865206E6F7A7A6C652100507290
:1026D000656465687265760050726568656174004E
:1026E000506F77657255700050726F73696D20631B
:1026F000656B656A746500506C6561736520776110
:102700006974004E656A6472697665207A617665DF
:1027100064746520504C412066696C616D656E740F
:102720002070726F73696D2E00506C656173652047
:102730006C6F616420504C412066696C616D656E00
:10274000742066697273742E004A6520504C4120D3
:1027500066696C616D656E74207A61766564656E1C
:102760003F00497320504C412066696C616D656E75
:1027700074206C6F616465643F002020506C616E52
:102780006E657242756666657242797465733A2049
:1027900000506C6561736520706C616365207374B3
:1027A00065656C207368656574206F6E206865616F
:1027B000746265642E004E6168726976616E69208C
:1027C00050494E44410050494E444120486561748F
:1027D000696E67005469736B61726E61206E656229
:1027E000796C61207465706C6F746E65207A6B61B2
:1027F0006C6962726F76616E610054656D706572AE
:1028000061747572652063616C6962726174696F6D
:102810006E20686173206E6F74206265656E207231
:10282000756E2079657400504944206B616C2E20D0
:1028300020202020202020202020005049442063F8
:10284000616C2E20202020202020202020200050DD
:102850004944206B616C2E20756B6F6E63656E61F1
:10286000005049442063616C2E2066696E6973686C
:10287000656400504944206B616C696272616365F4
:10288000005049442063616C6962726174696F6EC3
:1028900000506F7A61737461766974207469736B28
:1028A000005061757365207072696E7400556D69B2
:1028B0007374657465206C697374207061706972DB
:1028C00075206E6120706F646C6F7A6B752061206B
:1028D0007564727A756A7465206A656A20706F64BF
:1028E00020747279736B6F7520626568656D206DF9
:1028F0006572656E69207072766E69636820342037
:10290000626F64752E20506F6B75642074727973DA
:102910006B61207A61636879746920706170697293
:102920002C207679706E657465207469736B6172A2
:102930006E752E00506C616365206120736865655B
:1029400074206F6620706170657220756E646572A8
:1029500020746865206E6F7A7A6C65206475726980
:102960006E67207468652063616C69627261746966
:102970006F6E206F66206669727374203420706FEA
:10298000696E74732E20496620746865206E6F7AB4
:102990007A6C652063617463686573207468652070
:1029A00070617065722C20706F776572206F66663B
:1029B00020746865207072696E74657220696D6D2F
:1029C0006564696174656C792E006F6B004F666693
:1029D000004E6F206D6F76652E005A61646E612027
:1029E0005344206B61727461004E6F205344206326
:1029F00061726400547279736B61004E6F7A7A6C05
:102A0000650046696C616D656E74206E657A6176ED
:102A10006564656E0046696C616D656E74206E6FED
:102A200074206C6F61646564004261727661206E2F
:102A3000656E6920636973746100436F6C6F722007
:102A40006E6F7420636C656172004E65004E6F009E
:102A500050726F73696D20616B7475616C697A7502
:102A60006A74652E00506C656173652075706772BD
:102A70006164652E005679736C61206E6F766120FB
:102A80007665727A65206669726D776172653A0063
:102A90004E6577206669726D776172652076657222
:102AA00073696F6E20617661696C61626C653A0072
:102AB000506F73756E6F7574205A004D6F76652078
:102AC0005A00506F73756E6F75742059004D6F7694
:102AD00065205900506F73756E6F75742058004DE6
:102AE0006F76652058004578747275646572005081
:102AF0006F73756E6F7574206F7375004D6F7665AB
:102B00002061786973004D65736820426564204CCC
:102B10006576656C696E67004B616C6962726163B2
:102B2000650043616C6962726174696F6E00207A3E
:102B3000203900206F662039004D6572696D207262
:102B400065666572656E636E69207679736B752054
:102B50006B616C69627261636E69686F20626F6439
:102B600075004D6561737572696E67207265666583
:102B700072656E636520686569676874206F66209A
:102B800063616C6962726174696F6E20706F696EE7
:102B900074004D6572656E65207A6B6F73656E6942
:102BA0003A004D6561737572656420736B65773AA1
:102BB00000486C61766E69206E616269646B6100C9
:102BC0004D61696E004D32323120496E76616C691B
:102BD0006420657874727564657220004D323138F6
:102BE00020496E76616C69642065787472756465DD
:102BF0007220004D32303020496E76616C6964205D
:102C0000657874727564657220005265706F7274B5
:102C1000696E6720656E6473746F7020737461747D
:102C20007573004D313137204B616C2E20707276F8
:102C30006E6920767273747679004D313137204693
:102C400069727374206C617965722063616C2E0007
:102C50004649524D574152455F4E414D453A4D61AF
:102C6000726C696E2056312E302E323B20537072BA
:102C7000696E7465722F6772626C206D617368751E
:102C80007020666F722067656E36204649524D5738
:102C90004152455F55524C3A68747470733A2F2F05
:102CA0006769746875622E636F6D2F7072757361DA
:102CB00033642F50727573612D69332D506C7573A9
:102CC0002F2050524F544F434F4C5F56455253495B
:102CD0004F4E3A312E30204D414348494E455F54C6
:102CE0005950453A5072757361206933204D4B330A
:102CF0002045585452554445525F434F554E543A1F
:102D00003120555549443A30303030303030302D54
:102D1000303030302D303030302D303030302D30BC
:102D200030303030303030303030300A004D3130DB
:102D30003920496E76616C696420657874727564B7
:102D4000657220004D31303520496E76616C6964C2
:102D500020657874727564657220004D31303420BE
:102D6000496E76616C696420657874727564657209
:102D7000200055766F6C6E656E612072656D656EB4
:102D800069636B61004C6F6F73652070756C6C6567
:102D900079005A61766573742066696C616D656E41
:102DA00074004C6F61642066696C616D656E7400BF
:102DB0005A61766164656E692066696C616D656EE5
:102DC0007475004C6F6164696E672066696C616D33
:102DD000656E740043697374656E69206261727612
:102DE00079004C6F6164696E6720636F6C6F72006D
:102DF0004C6576793A004C6566743A00567962659E
:102E000072206A617A796B610053656C6563742026
:102E10006C616E67756167650043657374696E61A7
:102E200000456E676C697368004B494C4C45442EF5
:102E30002000496E76616C696420657874727564EF
:102E4000657200566C6F7A74652066696C616D6599
:102E50006E7400496E736572742066696C616D658D
:102E60006E74005072696E742046414E3A20004ED6
:102E70006F7A7A6C652046414E3A004578747275D7
:102E800064657220696E666F00207A203400206FBE
:102E9000662034005A6C657073756A6920707265BB
:102EA000736E6F7374206B616C69627261636E69BB
:102EB000686F20626F647500496D70726F76696E1D
:102EC00067206265642063616C6962726174696F16
:102ED0006E20706F696E74004B616C696272756A06
:102EE00069205A0043616C6962726174696E67207F
:102EF0005A004B616C696272616365204F4B0043FD
:102F0000616C6962726174696F6E20646F6E6500D6
:102F10004B616C6962726F766174205A0043616C18
:102F2000696272617465205A005A616872697661DB
:102F30006E69204F4B2E0048656174696E6720648E
:102F40006F6E652E005A6168726976616E6900481D
:102F5000656174696E670046696C2E2073656E73D7
:102F60006F7220205B6F6E5D0046696C2E2073656A
:102F70006E736F72205B6F66665D002046726565DA
:102F8000204D656D6F72793A20005469736B6172E0
:102F90006E61206E6562796C61206A65737465206C
:102FA0007A6B616C6962726F76616E612E20506F10
:102FB00073747570756A74652070726F73696D20B3
:102FC000706F646C65206D616E75616C752C206B23
:102FD000617069746F6C61205A6163696E616D65BF
:102FE0002C206F6473746176656320506F73747501
:102FF00070206B616C6962726163652E005072694A
:103000006E74657220686173206E6F7420626565EE
:103010006E2063616C6962726174656420796574A5
:103020002E20506C6561736520666F6C6C6F772025
:10303000746865206D616E75616C2C2063686170C9
:103040007465722046697273742073746570732C92
:103050002073656374696F6E2043616C696272618D
:1030600074696F6E20666C6F772E00507275746F86
:103070006B00466C6F7700446F6B6F6E636F7661A9
:103080006E6920706F687962750046696E69736851
:10309000696E67206D6F76656D656E747300207A5A
:1030A000203400206F66203400486C6564616D2018
:1030B0006B616C69627261636E6920626F6420701B
:1030C0006F646C6F7A6B7900536561726368696EC7
:1030D00067206265642063616C6962726174696F04
:1030E0006E20706F696E740049746572616365204B
:1030F00000497465726174696F6E2000446F6E657B
:1031000020736176696E672066696C652E00446F76
:103110006E65207072696E74696E672066696C6591
:10312000004A652062617276612063697374613F51
:1031300000497320636F6C6F7220636C6561723F2E
:103140000056796D656E69742066696C616D656E97
:1031500074004368616E67652066696C616D656EB9
:103160007400527963686C6F73742076656E742E88
:103170000046616E20737065656400656E717565EB
:10318000696E67202200457874727564657200204C
:1031900045787465726E616C205265736574005079
:1031A00072696E7465722073746F707065642064E8
:1031B000756520746F206572726F72732E20466978
:1031C0007820746865206572726F7220616E642069
:1031D000757365204D39393920746F2072657374A9
:1031E0006172742E202854656D70657261747572F9
:1031F000652069732072657365742E205365742091
:10320000697420616674657220726573746172748A
:10321000696E6729004E6F204C696E65204E756D92
:10322000626572207769746820636865636B737583
:103230006D2C204C617374204C696E653A20004EF1
:103240006F20436865636B73756D207769746820C0
:103250006C696E65206E756D6265722C204C6173B1
:1032600074204C696E653A200020746F6F206C6F7B
:103270006E6720657874727573696F6E2070726501
:1032800076656E746564004C696E65204E756D627E
:103290006572206973206E6F74204C617374204CCA
:1032A000696E65204E756D6265722B312C204C6104
:1032B0007374204C696E653A20005072696E7465B3
:1032C000722068616C7465642E206B696C6C2829AF
:1032D0002063616C6C6564210020636F6C64206501
:1032E0007874727573696F6E2070726576656E742E
:1032F000656400636865636B73756D206D69736DDC
:10330000617463682C204C617374204C696E653A5B
:10331000200043485942413A004552524F523A0028
:10332000456E642066696C65206C697374006F700B
:10333000656E0054524947474552454400656E64E6
:1033400073746F7073206869743A2000536C6565FC
:10335000702E2E2E005679706E6F7574206D6F74FE
:103360006F72790044697361626C65207374657073
:103370007065727300446174756D3A0044617465E0
:103380003A00506F757A6520616B7475616C6E6977
:103390000043757272656E740043726173682064D5
:1033A00065742E2020205B6F6E5D00437261736830
:1033B000206465742E20205B6F66665D0020436F7D
:1033C000756E7420583A200056796D656E61206FD5
:1033D0006B3F004368616E67656420636F7272655E
:1033E00063746C793F005A63686C6164697400436C
:1033F0006F6F6C646F776E0050726F2075737065BD
:10340000736E6F75206B616C696272616369206FA6
:10341000636973746574652070726F73696D20746D
:1034200069736B6F766F7520747279736B752E206C
:10343000506F74767264746520746C616369746B28
:10344000656D2E00506C6561736520636C65616EFF
:1034500020746865206E6F7A7A6C6520666F7220C2
:1034600063616C6962726174696F6E2E20436C696E
:10347000636B207768656E20646F6E652E00204C4C
:1034800061737420557064617465643A20005679E4
:1034900062657274652065787472756465723A004D
:1034A00043686F6F73652065787472756465723AEE
:1034B000005A6D656E612075737065736E612100D1
:1034C0004368616E6765207375636365737321007C
:1034D0005469736B207A205344005072696E7420D3
:1034E00066726F6D205344005465706C6F742E20AB
:1034F0006B616C6962726163650054656D702E204A
:1035000063616C6962726174696F6E0043616C69BA
:1035100062726174696E67205A005A6B616C6962ED
:10352000726F7661740043616C69627261746500E8
:1035300052657365742058595A206B616C696272C8
:103540002E0052657365742058595A2063616C6966
:1035500062722E004B616C6962726163652058591A
:103560005A0043616C6962726174652058595A004F
:103570002042726F776E206F757420526573657488
:1035800000426567696E2066696C65206C697374BA
:10359000004B616C6962726163652058595A206EF4
:1035A00065707265736E612E204C6576792070723D
:1035B00065646E6920626F64206D6F63207670723F
:1035C0006564752E0058595A2063616C6962726196
:1035D00074696F6E20636F6D70726F6D697365646F
:1035E0002E204C6566742066726F6E742063616C69
:1035F0006962726174696F6E20706F696E74206E9B
:103600006F7420726561636861626C652E004B6146
:103610006C6962726163652058595A206E657072D8
:1036200065736E612E20507265646E69206B616CEB
:1036300069627261636E6920626F6479206D6F6385
:10364000207670726564752E0058595A2063616C3B
:103650006962726174696F6E20636F6D70726F6DF5
:10366000697365642E2046726F6E742063616C69A5
:1036700062726174696F6E20706F696E7473206E10
:103680006F7420726561636861626C652E004B61C6
:103690006C6962726163652058595A207620706F98
:1036A0007261646B752E20582F59206F7379206DCD
:1036B00069726E65207A6B6F73656E652E20446F3C
:1036C000627261207072616365210058595A2063EB
:1036D000616C6962726174696F6E20616C6C2072DA
:1036E000696768742E20582F5920617865732061AE
:1036F000726520736C696768746C7920736B657789
:1037000065642E20476F6F64206A6F6221004B61F1
:103710006C6962726163652058595A207620706F17
:103720007261646B752E205A6B6F73656E692062CF
:10373000756465206175746F6D617469636B792060
:103740007679726F766E616E6F207072692074691F
:10375000736B752E0058595A2063616C69627261EF
:1037600074696F6E20616C6C2072696768742E20BA
:10377000536B65772077696C6C20626520636F728C
:10378000726563746564206175746F6D61746963DB
:10379000616C6C792E004B616C69627261636520AB
:1037A00058595A2073656C68616C612E204B616CAE
:1037B00069627261636E6920626F6420706F646C0D
:1037C0006F7A6B79206E656E616C657A656E2E001E
:1037D00058595A2063616C6962726174696F6E2016
:1037E0006661696C65642E204265642063616C6962
:1037F00062726174696F6E20706F696E7420776198
:1038000073206E6F7420666F756E642E004B616C52
:103810006962726163652058595A207620706F7210
:1038200061646B752E20582F59206F7379206A734D
:103830006F75206B6F6C6D652E2047726174756CAF
:10384000756A69210058595A2063616C6962726116
:1038500074696F6E206F6B2E20582F592061786528
:1038600073206172652070657270656E646963753E
:103870006C61722E20436F6E67726174756C617437
:10388000696F6E7321004B616C69627261636520C0
:1038900058595A2073656C68616C612E204E6168BE
:1038A0006C65646E65746520646F206D616E756112
:1038B0006C752E0058595A2063616C69627261748C
:1038C000696F6E206661696C65642E20506C65615D
:1038D000736520636F6E73756C7420746865206DFA
:1038E000616E75616C2E004B616C6962726163651B
:1038F0002058595A2073656C68616C612E204C65A4
:10390000767920707265646E6920626F64206D6FD5
:1039100063207670726564752E2053726F766E65C3
:103920006A7465207469736B61726E752E005859E4
:103930005A2063616C6962726174696F6E2066619E
:10394000696C65642E204C6566742066726F6E74B7
:103950002063616C6962726174696F6E20706F6957
:103960006E74206E6F7420726561636861626C654D
:103970002E004B616C6962726163652058595A2050
:1039800073656C68616C612E20507265646E69208D
:103990006B616C69627261636E6920626F64792029
:1039A0006D6F63207670726564752E2053726F762A
:1039B0006E656A7465207469736B61726E752E0032
:1039C00058595A2063616C6962726174696F6E2024
:1039D0006661696C65642E2046726F6E7420636147
:1039E0006C6962726174696F6E20706F696E747356
:1039F000206E6F7420726561636861626C652E0071
:103A00004B616C696272616365205A2073656C68F2
:103A1000616C612E2053656E736F72206A65206F32
:103A200064706F6A656E79206E65626F2070726572
:103A3000727573656E79206B6162656C2E204365CB
:103A40006B616D206E612072657365742E00426536
:103A500064206C6576656C696E67206661696C656B
:103A6000642E2053656E736F7220646973636F6E8A
:103A70006E6563746564206F72206361626C65209B
:103A800062726F6B656E2E2057616974696E672074
:103A9000666F722072657365742E004B616C69628B
:103AA00072616365205A2073656C68616C612E20B9
:103AB00053656E736F72206E657365706E756C2ED4
:103AC000205A6E6563697374656E612074727973D0
:103AD0006B613F2043656B616D206E612072657381
:103AE00065742E00426564206C6576656C696E674E
:103AF000206661696C65642E2053656E736F722059
:103B00006469646E7420747269676765722E2044FC
:103B10006562726973206F6E206E6F7A7A6C653F92
:103B20002057616974696E6720666F7220726573D1
:103B300065742E004B616C696272616365205A2066
:103B400073656C68616C612E2053656E736F7220B3
:103B50007365706E756C207072696C69732076790C
:103B6000736F6B6F2E2043656B616D206E612072E9
:103B7000657365742E00426564206C6576656C69BA
:103B80006E67206661696C65642E2053656E736F85
:103B9000722074726967676572656420746F6F2044
:103BA000686967682E2057616974696E6720666F5F
:103BB000722072657365742E005A6168726976614D
:103BC0006E692062656400426564204865617469BD
:103BD0006E6700426564204F4B2E0042656420648E
:103BE0006F6E650056707261766F205B756D5D005B
:103BF000526967687420736964655B756D5D005216
:103C00006573657400567A61647520205B756D5D1F
:103C100000526561722073696465205B756D5D009B
:103C20004B6F72656B636520706F646C6F7A6B7934
:103C300000426564206C6576656C20636F72726506
:103C4000637400566C65766F20205B756D5D004C6B
:103C50006566742073696465205B756D5D005670E0
:103C600072656475205B756D5D0046726F6E7420C1
:103C7000736964655B756D5D00426564004E656ED9
:103C800069207A6B616C6962726F76616E61207611
:103C90007A64616C656E6F737420747279736B797A
:103CA000206F64207469736B6F766520706F646C2D
:103CB0006F7A6B792E20506F73747570756A7465A6
:103CC0002070726F73696D20706F646C65206D6118
:103CD0006E75616C752C206B617069746F6C6120FE
:103CE0005A6163696E616D652C206F6473746176CF
:103CF0006563204E6173746176656E6920707276BB
:103D00006E69207672737476792E004469737461DB
:103D10006E6365206265747765656E2074697020D6
:103D20006F6620746865206E6F7A7A6C6520616EAC
:103D300064207468652062656420737572666163CF
:103D40006520686173206E6F74206265656E2073F4
:103D50006574207965742E20506C656173652066EA
:103D60006F6C6C6F7720746865206D616E75616C27
:103D70002C206368617074657220466972737420C8
:103D800073746570732C2073656374696F6E20465D
:103D900069727374206C617965722063616C696209
:103DA000726174696F6E2E00446F6C6164656E6938
:103DB000206F7379205A004C6976652061646A75BA
:103DC0007374205A0041646A757374696E67205A6F
:103DD000004175746F20686F6D6500207C2041750F
:103DE00074686F723A200056736500416C6C004134
:103DF00063746976652045787472756465723A20DB
:103E0000009A138A13AE13B613BE13C713CF13EC65
:103E100013D71305140114091411142A1419145575
:103E2000143B14AB1473140915E9148D152C159B50
:103E300016F01592174F173818DF17EB187F1896E2
:103E4000194A192A1AE7197B1A671AE91A8F1A8070
:103E50001B311BEE1BCA1B231C0E1C461C371C915E
:103E60001C631C1C1DBF1C7C1D831D9D1D931DBB45
:103E70001DA91DCC1DF11DDD1D141E031E361E24A3
:103E80001E491E621E5C1E671E791E9A1E8A1EBB7C
:103E90001EAA1E071FCC1E541F3F1F711F691F85BE
:103EA0001F7D1F9B1F8D1FA61FB01FC41FED1FDF8F
:103EB0001F12200020312023204C203F206A205D4B
:103EC000207720AB20A220B120D020C120EF20DD20
:103ED00020132101213621252154214521732161FF
:103EE000218E218421A6219721B321D421C521E34C
:103EF00021FF21F0210D2213223622252251223FBB
:103F0000227822632289229A22AA22B322D022BBBB
:103F100022F322E122172305233B2329235F234D8C
:103F20002383237123A7239523CB23B923DD23EAFE
:103F300023F623FB230D241F24322448243A24553E
:103F40002467247B2499248B24A724B424C224D05E
:103F500024E624F1240E250725262515254425359C
:103F6000255E2553256B2574259C25BE25E425D388
:103F7000250726F62524261926402630265B264DC1
:103F800026692693267E26BA26A626D826CE26E0A1
:103F900026F726E82629270327622749277A27912B
:103FA00027C627B627FA27D4273B28272861284F7A
:103FB0002881287328A12891283429AD28CA29CD21
:103FC00029D129E929DA29FB29F429152A022A3AD3
:103FD0002A292A4D2A4A2A652A502A902A752ABB5C
:103FE0002AB02ACD2AC22ADF2AD42AE62AFC2AEFBE
:103FF0002A062B222B182B332B2E2B622B392BA28C
:104000002B922BC02BB12BC52BDC2BF32B0A2C3A7C
:104010002C232C502C2D2D442D5B2D852D722DA263
:104020002D922DC32DB02DE22DD42DF62DF02D097E
:104030002EFC2D212E192E292E322E532E432E6387
:104040002E6F2E7B2E8E2E892EB82E942EE42ED8F7
:104050002EFF2EF22E1D2F102F372F292F4F2F45D9
:104060002F572F692F7B2FFD2F8A2F72306B308AAD
:10407000307730A3309E30C830A930F130E830FCC2
:10408000300E313131213152314131713162317B68
:104090003186318F319F3115323F3269328732BAE2
:1040A00032D932F3321933123320332E3333333DC6
:1040B000334C33643355337C3375339133823399C6
:1040C00033AB33BD33D333C833EF33E6334434F843
:1040D000337E34A0348E34C034B134DA34D034FA80
:1040E00034E8340C3526351A3542353035623554CE
:1040F0003570358135C535913549360E36CB368E1E
:104100003655370E37D037963745380D38B43886A0
:10411000382E39E738C03972394E3A003AE43A9BC2
:104120003A763B343BC73BB93BDB3BD33BF03BE40C
:104130003BFF3B113C053C313C203C4F3C433C6A3F
:104140003C5E3C793C0B3D7D3CB73DA83DC53DD137
:104150003DDB3DEB3DE73DEF3D457872656D65200C
:104160007370616E206F6620746865205A207661D6
:104170006C756573210043616C63756C6174696F64
:104180006E206F6620746865206D616368696E6576
:1041900020736B657720616E64206F66667365744B
:1041A000206661696C65642E00203C2000574152F6
:1041B0004E494E473A2046726F6E7420706F696E9A
:1041C00074206E6F7420726561636861626C652E25
:1041D000205920636F6F7264696E6174653A0000E4
:1041E000497465726174696F6E3A2000496E766138
:1041F0006C69642062656420636F727265637469C0
:104200006F6E206D61747269782E205265736574CB
:1042100074696E6720746F206964656E746974795F
:104220002E00496E76616C69642062656420636F5C
:104230007272656374696F6E206D61747269782E35
:1042400020582F592061786573206172652066615E
:10425000722066726F6D206265696E67207065728C
:1042600070656E646963756C61722E00496E76616B
:104270006C69642062656420636F7272656374693F
:104280006F6E206D61747269782E20536869667450
:10429000206F7574206F662072616E67652E005AFC
:1042A00065726F20706F696E7420636F72726563E0
:1042B00074696F6E3A00496E76616C69642062655C
:1042C0006420636F7272656374696F6E206D6174D0
:1042D0007269782E204C656E677468206F66207452
:1042E0006865205920766563746F72206F7574203D
:1042F0006F662072616E67652E0059207665637463
:104300006F72206C656E6774683A00496E76616CF6
:1043100069642062656420636F7272656374696F9B
:104320006E206D61747269782E204C656E677468BA
:10433000206F6620746865205820766563746F72FC
:10434000206F7574206F662072616E67652E00584D
:1043500020766563746F72206C656E6774683A00CE
:10436000556E646566696E65642062656420636F7E
:104370007272656374696F6E206D61747269782EF4
:104380000000004041FFFFBF4000005C43FFFFBF53
:104390004000005C430000464300004041000046EE
:1043A0004300004041FFFFBF400000E442FFFFBF69
:1043B0004000005743FFFFBF40000057430000CCC0
:1043C000420000E4420000CC42000040410000CC2A
:1043D0004200004041000046430000E44200004625
:1043E0004300005743000046435A00205A3A005900
:1043F0000020593A00580020583A0024F4D4305094
:10440000C38E20C2A24017828B7011127A910D8147
:104410006CD90AA861E108C7586607615143061EB6
:104420004B5D05C145A7041A411104093D9803716C
:104430003931034036DB0265339102D430540280B7
:104440002E1D02632CEE01752AC501B028A00110B3
:104450002781018F2564012B244B01E0223401AC1C
:10446000211F018D200D01801FFC00841EED00978F
:104470001DDF00B81CD200E61BC600201BBC006478
:104480001AB200B219A8000A19A0006A189900D13E
:1044900017910040178B00B516840031167E00B3CB
:1044A0001579003A157300C7146F0058146A00EEAE
:1044B0001366008813630025135E00C7125B006C4F
:1044C00012570015125400C111510070114F0021F4
:1044D000114B00D61049008D1047004610440002D1
:1044E000104200C00F4000800F3E00420F3C00060B
:1044F0000F3B00CB0E3800930E37005C0E350027C3
:104500000E3400F30D3200C10D3100900D3000600B
:104510000D2E00320D2D00050D2C00D90C2B00AEF8
:104520000C2900850C29005C0C2700350C27000E97
:104530000C2600E80B2400C40B2400A00B23007DF4
:104540000B23005A0B2100390B2100180B2000F817
:104550000A1F00D90A1E00BB0A1E009D0A1D00800A
:104560000A1D00630A1C00470A1B002C0A1B0011CD
:104570000A1A00F7091A00DD091900C4091900AB6D
:10458000091900920917007B091800630917004CEC
:1045900009160036091600200916000A091500F54B
:1045A000081500E0081400CC081400B8081400A492
:1045B000081400900813007D0812006B08130058BF
:1045C00008120046081200340811002308110012D6
:1045D00008110001081100F0071000E0071000D0DA
:1045E000071000C0071000B0070F00A107100091CE
:1045F000070E0083070F0074070F0065070E0057B2
:10460000070E0049070E003B070D002E070E002085
:10461000070D0013070D0006070D00F9060C00ED4D
:10462000060D00E0060C00D4060C00C8060C00BC09
:10463000060C00B0060C00A4060B0099060C008DB9
:10464000060B0082060B0077060B006C060B006160
:10465000060A0057060B004C060A0042060A0038FC
:10466000060A002E060A0024060A001A060A00108E
:1046700006090007060A00FD050900F4050900EB1C
:10468000050900E2050900D9050900D0050900C7A0
:10469000050900BE050900B5050800AD050800A51F
:1046A0000509009C050800940508008C0508008495
:1046B0000508007C050800740508006C0507006506
:1046C0000508005D050700560508004E0507004770
:1046D0000507004005080038050700310507002AD6
:1046E000050700230507001C050600160507000F37
:1046F0000507000805060002050700FB040600F593
:10470000040700EE040600E8040600E2040700DBEC
:10471000040600D5040600CF040600C9040600C341
:10472000040600BD040600B7040600B1040500AC91
:10473000040600A6040600A00405009B04060095DC
:10474000040500900406008A040500850405008025
:104750000406007A04050075040500700405006B6A
:1047600004050066040500610405005C04050057AB
:10477000040500520405004D0405004804050043EB
:104780000405003E0404003A040500350405003029
:104790000404002C04050027040400230405001E63
:1047A0000404001A04040016040500110404000D9A
:1047B000040400090405000404040000040400FCCF
:1047C000030400F8030400F4030400F0030400EC05
:1047D000030400E8030400E4030400E0030400DC35
:1047E000030400D8030400D4030400D0030400CC65
:1047F000030400C8030300C503030024F404D92004
:104800001BC40C5C0E9804C4095F0265077101F4B7
:1048100005F900FB04B30048048700C10369005890
:1048200003550003034500BE023A008402310053E1
:10483000022A002902250004022000E4011C00C80D
:10484000011900AF011700980114008401130071D1
:104850000110006101100051010E0043010D0036EE
:10486000010B002B010B0020010B00150109000CAE
:1048700001090003010800FB000800F3000800EB39
:10488000000700E4000600DE000600D8000600D2A3
:10489000000600CC000500C7000500C2000500BDF1
:1048A000000400B9000400B5000400B1000400AD2C
:1048B000000400A9000400A5000300A20003009F5B
:1048C0000004009B00030098000300950002009381
:1048D000000300900003008D0002008B000300889D
:1048E0000002008600020084000300810002007FB5
:1048F0000002007D0002007B0002007900020077C8
:1049000000010076000200740002007200010071D4
:104910000002006F0002006D0001006C0002006ADE
:1049200000010069000200670001006600010065E7
:1049300000010064000200620001006100010060EB
:104940000001005F0002005D0001005C0001005BEF
:104950000001005A000100590001005800010057F1
:1049600000010056000100550001005400010053F1
:1049700000000053000100520001005100010050EE
:104980000001004F0001004E0000004E0001004DEC
:104990000001004C0001004B0000004B0001004AE8
:1049A00000010049000100480000004800010047E4
:1049B00000010046000000460001004500000045DF
:1049C00000010044000100430000004300010042D8
:1049D00000000042000100410000004100010040D1
:1049E0000001003F0000003F0001003E0000003ECB
:1049F0000001003D0000003D0001003C0000003CC3
:104A00000000003C0001003B0000003B0001003AB8
:104A10000000003A000100390000003900010038B0
:104A200000000038000000380001003700000037A7
:104A3000000100360000003600000036000100359D
:104A40000000003500000035000100340000003493
:104A50000000003400010033000000330000003388
:104A6000000100320000003200000032000100317D
:104A70000000003100000031000100300000003073
:104A8000000000300001002F0000002F0000002F68
:104A90000000002F0001002E0000002E0000002E5C
:104AA0000001002D0000002D0000002D0000002D51
:104AB0000001002C0000002C0000002C0000002C45
:104AC0000001002B0000002B0000002B0000002B39
:104AD0000001002A0000002A0000002A0000002A2D
:104AE0000001002900000029000000290000002921
:104AF0000000002900010028000000280000002814
:104B00000000002800000028000100270000002706
:104B100000000027000000270000002700010026F9
:104B200000000026000000260000002600000026ED
:104B300000010025000000250000002500000025E0
:104B400000000025000000250001002400000024D2
:104B500000000024000000240000002400010023C5
:104B600000000023000000230000002300000023B9
:104B700000000023000000230001002200000022AA
:104B8000000000220000002200000022000000229D
:104B90000001002100000021000000210000002190
:104BA0000000002100000021000000210001002081
:104BB0000000002000000020000000200000002075
:104BC0000000002000000020000000200001001F65
:104BD0000000001F0000001F0000001F0000001F59
:104BE0000000001F0000001F0001001E0000001E4A
:104BF0000000001E0000001E0000004572723A20F6
:104C00004D494E54454D50204245440054656D7009
:104C1000657261747572652068656174656420628F
:104C20006564207377697463686564206F66662EB7
:104C3000204D494E54454D50207472696767657226
:104C400065642021004572723A204D415854454D0B
:104C500050204245440054656D70657261747572F0
:104C60006520686561746564206265642073776996
:104C70007463686564206F66662E204D4158544504
:104C80004D50207472696767657265642021004524
:104C900072723A204D494E54454D50003A204578A5
:104CA00074727564657220737769746368656420D3
:104CB0006F66662E204D494E54454D5020747269E2
:104CC0006767657265642021004572723A204D4124
:104CD0005854454D50003A20457874727564657299
:104CE000207377697463686564206F66662E204D53
:104CF000415854454D502074726967676572656408
:104D000020210020484F54454E4420544845524DE0
:104D1000414C2052554E415741590020484541547D
:104D200042454420544845524D414C2052554E4135
:104D300057415900544845524D414C2052554E411F
:104D40005741590042454420544845524D414C205A
:104D500052554E415741590020544845524D414CFF
:104D60002052554E41574159202820505245484520
:104D7000415420484F54454E442900205448455240
:104D80004D414C2052554E415741592028205052F8
:104D90004548454154204845415442454429005026
:104DA000524548454154204552524F5200424544D5
:104DB0002050524548454154204552524F520045DB
:104DC00072723A205052494E542046414E2045526C
:104DD000524F52004552524F523A205072696E74EF
:104DE0002066616E207370656564206973206C6F46
:104DF000776572207468656E206578706563746588
:104E000064004572723A20455854522E2046414E55
:104E1000204552524F52004552524F523A20457847
:104E20007472756465722066616E20737065656466
:104E3000206973206C6F776572207468656E2065D9
:104E40007870656374656400202D20496E76616C0E
:104E50006964206578747275646572206E756D6220
:104E60006572202100504944204175746F74756E3D
:104E7000652066696E6973686564212050757420C9
:104E8000746865206C617374204B702C204B692012
:104E9000616E64204B6420636F6E7374616E747313
:104EA0002066726F6D2061626F766520696E746F27
:104EB00020436F6E66696775726174696F6E2E68E4
:104EC00000504944204175746F74756E65206661A9
:104ED000696C6564212074696D656F75740020408C
:104EE0003A006F6B20543A006F6B20423A005049F1
:104EF00044204175746F74756E65206661696C65D8
:104F000064212054656D70657261747572652074DA
:104F10006F6F206869676800204B643A2000204B5F
:104F2000693A2000204B703A200020436C61737373
:104F300069632050494420002054753A2000204BDA
:104F4000753A2000206D61783A2000206D696E3A34
:104F5000200020643A200020626961733A2000102A
:104F6000137D002015780060177300C0196E004093
:104F70001C6900E01E640080215F0040245A00F09C
:104F800026550090295000202C4B00802E4600C052
:104F9000304100D0323C00B034370050363200C0CF
:104FA000372D0000392800103A2300F03A1E00B0D7
:104FB0003B1900503C1400D03C0F00303D0A0080EB
:104FC0003D0500C03D0000F03DFBFF103EF6FF3008
:104FD0003EF1FF403EECFF503EE7FF603EE2FF70D7
:104FE0003EDDFF703ED8FF1000C90210012C0140C9
:104FF00001220170011801B0010E01F001040150FD
:1050000002FA00B002F0003003E600D003DC0090AA
:1050100004D2007005C800A006BE000008B400B0AD
:1050200009AA00D00BA000600E960060118C000051
:1050300015820020197800C01D6E00A0226400B007
:10504000275A00902C500000314600E0343C0010FC
:10505000383200903A2800603C1E00A03D140080C9
:105060003E0A00203F000070012C0190012701B092
:10507000012201C0011D01F00118011002130130CD
:10508000020E016002090190020401C002FF00004B
:1050900003FA004003F5008003F000D003EB00208A
:1050A00004E6007004E100E004DC004005D700C025
:1050B00005D2004006CD00D006C8008007C30030EE
:1050C00008BE00F008B900C009B400B00AAF00B0D3
:1050D0000BAA00D00CA500000EA000500F9B00C032
:1050E0001096005012910000148C00C0158700B07B
:1050F000178200B0197D00D01B7800001E7300409D
:10510000206E0090226900F024640040275F009028
:10511000295A00E02B5500102E500020304B001073
:10512000324600E033410090353C001037370070C4
:10513000383200A0392D00B03A2800A03B2300608F
:105140003C1E00103D1900903D1400103E0F0070F1
:105150003E0A00C03E0500003F0000544D4320447D
:105160005249564552204F56455254454D50200005
:10517000436F6E74696E7565207769746820616E1F
:105180006F7468657220626F7764656E3F00537458
:105190006174653A2000473736004D3435205A0097
:1051A0004D3435004738300020003E003E002000DE
:1051B0003E003E003E003E0020003E003E0020003B
:1051C00000002D2D2D2D2D2D2D2D2D2D2D2D2D2D69
:1051D0002D2D2D2D2D2D004E2F41004E2F41006DD8
:1051E0006D00004D373031004D37303200496E765A
:1051F000616C6964205049442063616C2E207265A3
:1052000073756C74732E204E6F742073746F726597
:105210006420746F20454550524F4D2E004D35305F
:1052200030004731205A3135204631353030004783
:105230003931004731205835302059313930204537
:105240003020463730303000473930004D3730326B
:10525000004D3730322043004D3730322055004D5D
:10526000373032004731205A313520463135303021
:105270000047393100473120583530205931393015
:10528000204530204637303030004D383300473924
:1052900030004D3834004D313034205330004D381B
:1052A00034004731205831302059313830204634CD
:1052B000303030004731205A3130204631333030E1
:1052C0002E303030004D313430205330004D3130ED
:1052D00034205330004D31303700473120452D30D8
:1052E0002E30373530302046323130302E303030AD
:1052F000303000473120583530205935352045337E
:105300002E3632373733004731205832303020596B
:1053100035352045302E3439333836004731205862
:10532000323030205937352045332E363237373337
:1053300000473120583530205937352045302E343C
:105340003933383600473120583530205939352027
:1053500045332E363237373300473120583230301C
:10536000205939352045302E34393338360047310D
:10537000205832303020593131352045332E3632E5
:1053800037373300473120583530205931313520F7
:1053900045302E34393338360047312058353020E7
:1053A000593133352045332E3632373733004731C4
:1053B000205832303020593133352045302E3636A2
:1053C00031373400473120583230302059313535AB
:1053D0002045322E363237373300473120583130AE
:1053E0003020593135352045320047312058373586
:1053F00020593135352045322E3500473120463190
:10540000303830004731205835302059313535009B
:105410004731204634303030004D32303420533163
:10542000303030004731205A302E31353020463769
:105430003230302E30303000473120452D312E357E
:10544000303030302046323130302E303030303055
:10545000004D383300473930004732310047393288
:105460002045302E3000473120583130302E30204A
:105470004531322E352046313030302E3000473124
:10548000205836302E302045392E302046313030ED
:10549000302E30004739322045302E300047323828
:1054A00000473837004D3130392053323130004D0C
:1054B00031393020533535004D31343020533535B6
:1054C000004D3130342053323130004D313037000F
:1054D000473930004731204531004D3832004731DF
:1054E000204531004D3833004D313036205325648E
:1054F000004D32323020532564003A200020202015
:10550000202020202020202020202020202020209B
:1055100000203A20002020202020202020202020B1
:10552000202020202020202020002020202020209B
:1055300020202020202020002573002020002D2D59
:105540003A2D2D002000200020004C0020200020BB
:1055500046002D2D2D003E555342005344002D2D65
:1055600000252020202020002020002020000120D5
:10557000002020202D2D2D200020205A002020004A
:105580000120004D36303000464C4558202D20205B
:105590003233302F35300050502020202D20203243
:1055A00035342F3130300048495053202D202032DF
:1055B00032302F3130300050455420202D20203201
:1055C00034302F393000504C4120202D20203231F2
:1055D000352F35350041425320202D2020323535DE
:1055E0002F313030006661726D20202D2020323541
:1055F000302F3430004D3234004D323320257300CB
:10560000052E2E00580059005A00457874727564B2
:105610006572004739390044697361626C652066C0
:1056200061726D206D6F64653F0044697361626CE7
:1056300065206661726D206D6F6465004661726DF4
:10564000206E756D626572004D3834005072696E5F
:10565000742066616E3A00457874727564657220D4
:1056600066616E3A0041786973206C656E67746894
:1056700020646966666572656E63653A004D6561B2
:1056800073757265642061786973206C656E6774E8
:10569000683A0025632041584953205347313D253E
:1056A000640A004D3834004731205A313500473202
:1056B000382057005A30005A310059300059310013
:1056C000583000583100456E642073746F70732039
:1056D00064696167004D3434004732382057001B3D
:1056E0005B303B314842656C742073746174757330
:1056F0001B5B313B3248582025641B5B323B3248F0
:1057000059202564001B5B313B3148416D6269655E
:105710006E743A2020256425631B5B323B31485070
:10572000494E44413A2020202025642563004175DC
:10573000746F207265636F7665722063726173683F
:1057400000436865636B2066616E73205B44495358
:105750005D00436865636B2066616E73205B454E38
:105760005D0054656D706572617475726573004299
:10577000656C7420737461747573002D2D2D2D2D3F
:105780002D2D2D2D2D2D2D00466C617368416972D4
:1057900020495020416464723A002D2D2D2D2D2D6D
:1057A0002D2D2D2D2D2D004E6F76203237203230AD
:1057B0003137002D2D2D2D2D2D2D2D2D2D2D2D0065
:1057C000453344763666756C6C0045494E595F30FA
:1057D000346100315F37356D6D5F4D4B33002D2DDA
:1057E0002D2D2D2D2D2D2D2D2D2D0020332E312E17
:1057F000312D5243312062313136004669726D7766
:105800006172653A0025642E25642E25642E256478
:10581000004661696C207374617473004661726D37
:10582000206E756D6265720000726300626574615E
:1058300000616C7068610064657600505255534198
:105840003344465700332E312E312D524331000060
:10585000000A0B02090C0D0E0807030401000000EA
:105860000000000000000000000000000000000038
:1058700000000000000000000000001211100000F5
:105880000000000000000000000000000000000018
:105890000000000000000000000000000000000008
:1058A0000000000000010210202008081020401015
:1058B00020408002010201080402010102040810D4
:1058C00020408080402010080402018004020180F2
:1058D000402010080402010804020101020408101B
:1058E0002040800102040810204080100804088035
:1058F0001020400440801020400480050505050765
:105900000508080808020202020A0A08080404043A
:105910000401010101010101010303030303030366
:1059200003040707070C0C0C0C0C0C0C0C020202F5
:105930000206060606060606060B0B0B0B0B0B0BE8
:105940000B07070A0A0A0A0A0A05050504040408DF
:1059500008000020002300260029002C002F003220
:1059600000000100000301060109010000220025DA
:105970000028002B002E0031003400020100000539
:105980000108010B0100002100240027002A002D3E
:10599000003000330001010000040107010A010288
:1059A0004E414E494E495459494E46CDCCCC3D0A04
:1059B000D7233C17B7D13877CC2B329595E6241FE7
:1059C000B14F0A000020410000C84200401C4620A0
:1059D000BCBE4CCA1B0E5AAEC59D7400407A10F373
:1059E0005A00A0724E18090010A5D4E80000E8760D
:1059F00048170000E40B54020000CA9A3B00000064
:105A0000E1F505000080969800000040420F00007C
:105A100000A08601000000102700000000E803003D
:105A20000000006400000000000A00000000000107
:105A300000000000002C76D888DC674F0823DFC107
:105A4000DFAE59E1B1B796E5E3E453C63AE65199C2
:105A50007696E8E6C28426EB898C9B62ED407C6FEB
:105A6000FCEFBC9C9F40F2BAA56FA5F490055A2AA2
:105A7000F75C936B6CF9676DC11BFCE0E40D47FEAE
:105A8000F520E6B500D0ED902E03009435770500A3
:105A900080841E080000204E0A000000C80C33332A
:105AA00033330F986E12831141EF8D2114893BE639
:105AB0005516CFFEE6DB18D1844B381BF77C1D90C2
:105AC0001DA4BBE424203284725E228100C9F1242B
:105AD000ECA1E53D2700BEA163C8EAF9F30163012B
:105AE000EFA111241FBECFEFD1E2DEBFCDBF00E09A
:105AF0000CBF19E0A0E0B2E0E2E3F8E903E00BBF7D
:105B000002C007900D92AC3DB107D9F72CE1ACED86
:105B1000B9E001C01D92AE35B207E1F71AE5C0EE5B
:105B2000DAE500E006C022970109FE010BBF0F94E1
:105B3000BCC1C63DD10780E00807A9F70F9494BB0C
:105B40000D9407CC0C940000CF92DF92EF92FF925D
:105B50000F931F93CF93DF938C01D42EC62FD72F93
:105B6000D60EDC1671F1F801E080F180C990C70112
:105B70000F94FAC8C816F1F06C2DC7010F942AC90A
:105B8000C7010F94FAC88C15A9F0E2EBF7E08491F5
:105B9000882341F09091C00095FFFCCF8093C60010
:105BA0003196F5CF8091C00085FFFCCF8AE08093CD
:105BB000C60007C0F801808191810196918380839E
:105BC000D0CFDF91CF911F910F91FF90EF90DF9099
:105BD000CF900895EF92FF920F931F93CF93DF938F
:105BE0001F92CDB7DEB78C017B01460FF801808193
:105BF000918149830F94FAC8F70181937F01F801DD
:105C00008081918101969183808349814E11EECFED
:105C10000F90DF91CF911F910F91FF90EF9008951A
:105C2000FF920F931F93CF93DF93CDB7DEB72C97DF
:105C30000FB6F894DEBF0FBECDBF8C01F62E80E309
:105C400090E3A0E3B0E08D839E83AF83B8871C8789
:105C50000B8744E0BE016B5F7F4FCE010B9674DF74
:105C600040E162EA79E1CE010B966EDF40E162EB42
:105C700079E1CE010B9668DF40E162E979E1CE017E
:105C80000B9662DF44E06AE879E1CE010B965CDFB7
:105C900044E066E879E1CE010B9656DF44E06EE819
:105CA00079E1CE010B9650DF44E062E779E1CE0165
:105CB0000B964ADF44E062EC79E1CE010B9644DFBB
:105CC00044E066E779E1CE010B963EDF44E06AE707
:105CD00079E1CE010B9638DF44E06EE779E1CE0141
:105CE0000B9632DF44E062E879E1CE010B962CDFBF
:105CF0004CE062E37BE0CE010B9626DF44E06BE2F2
:105D00007BE0CE010B9620DF44E06DEA72E0CE012D
:105D10000B961ADF44E069EA72E0CE010B9614DFBD
:105D200044E065EA72E0CE010B960EDF44E06DE9D7
:105D300072E0CE010B9608DF44E069E972E0CE0123
:105D40000B9602DF44E065E972E0CE010B96FCDEC3
:105D500080E290E09A87898742E0BE01675F7F4FCB
:105D6000CE010B96F1DE41E067E27BE0CE010B96BF
:105D7000EBDE44E064E272E0CE010B96E5DE44E047
:105D80006CE172E0CE010B96DFDE44E062E27BE084
:105D9000CE010B96D9DE44E06EE17BE0CE010B969E
:105DA000D3DE44E068E172E0CE010B96CDDE41E047
:105DB0006EE47BE0CE010B96C7DE44E064E472E063
:105DC000CE010B96C1DE89E08F1560F444E061ECF2
:105DD00073E1CE010B96B8DE44E06DEB73E1CE01CA
:105DE0000B96B2DE46E551E360E070E049835A83EA
:105DF0006B837C831C870B8744E0BE016F5F7F4F02
:105E0000CE010B96A1DEEEEEFFE08491882341F0F7
:105E10009091C00095FFFCCF8093C6003196F5CFDE
:105E2000E2EAF7E08491882341F09091C00095FF69
:105E3000FCCF8093C6003196F5CF8091C00085FFDE
:105E4000FCCF8AE08093C6002C960FB6F894DEBF94
:105E50000FBECDBFDF91CF911F910F91FF9008959D
:105E60001F93CF93DF93182FCEEEDFE0FE018491D6
:105E7000882341F09091C00095FFFCCF8093C6002D
:105E80003196F5CFE2E9F7E08491882341F09091D3
:105E9000C00095FFFCCF8093C6003196F5CF80916E
:105EA000C00085FFFCCF8AE08093C600FE0184918C
:105EB000EEEEFFE0882349F09091C00095FFFCCF03
:105EC0008093C60031968491F5CF4091A2195091EC
:105ED000A3196091A4197091A5198AE897E00E940E
:105EE00043474091A6195091A7196091A819709144
:105EF000A91987E897E00E9443474091AA19509159
:105F0000AB196091AC197091AD1984E897E00E94CB
:105F100043474091AE195091AF196091B0197091FB
:105F2000B11981E897E00E9443478091C00085FF46
:105F3000FCCF8AE08093C600FE018491EEEEFFE084
:105F4000882349F09091C00095FFFCCF8093C60054
:105F500031968491F5CFE7E6F7E08491882341F00C
:105F60009091C00095FFFCCF8093C6003196F5CF8D
:105F70008091C00085FFFCCF8AE08093C600FE01BF
:105F80008491EEEEFFE0882349F09091C00095FFE8
:105F9000FCCF8093C60031968491F5CF4091B21921
:105FA0005091B3196091B4197091B5198EE597E0CD
:105FB0000E9443474091B6195091B7196091B819A2
:105FC0007091B9198BE597E00E9443474091BA1947
:105FD0005091BB196091BC197091BD1988E597E08B
:105FE0000E9443474091BE195091BF196091C0195A
:105FF0007091C11985E597E00E9443478091C000E8
:1060000085FFFCCF8AE08093C600FE018491EEEE0E
:10601000FFE0882349F09091C00095FFFCCF80936A
:10602000C60031968491F5CFE7E3F7E084918823A9
:1060300041F09091C00095FFFCCF8093C60031964F
:10604000F5CF8091C00085FFFCCF8AE08093C60029
:10605000FE018491EEEEFFE0882349F09091C000AC
:1060600095FFFCCF8093C60031968491F5CF409187
:1060700092195091931960919419709195198EE22B
:1060800097E00E945447409196195091971960915A
:106090009819709199198BE297E00E9454474091AA
:1060A0009A1950919B1960919C1970919D1988E2E1
:1060B00097E00E94544740919E1950919F1960911A
:1060C000A0197091A11985E297E00E945447809130
:1060D000C00085FFFCCF8AE08093C600FE0184915A
:1060E000EEEEFFE0882349F09091C00095FFFCCFD1
:1060F0008093C60031968491F5CFE0EFF6E084916D
:10610000882341F09091C00095FFFCCF8093C6009A
:106110003196F5CF8091C00085FFFCCF8AE0809357
:10612000C600FE018491EEEEFFE0882349F09091D5
:10613000C00095FFFCCF8093C60031968491F5CFC7
:1061400040918A1950918B1960918C1970918D1919
:1061500087EE96E00E944347409186195091871937
:10616000609188197091891984EE96E00E944347E6
:106170008091C00085FFFCCF8AE08093C600FE01BD
:106180008491EEEEFFE0882349F09091C00095FFE6
:10619000FCCF8093C60031968491F5CFE1E3F6E021
:1061A0008491882341F09091C00095FFFCCF8093AB
:1061B000C6003196F5CF8091C00085FFFCCF8AE004
:1061C0008093C600FE018491EEEEFFE0882349F043
:1061D0009091C00095FFFCCF8093C60031968491CA
:1061E000F5CF40918E1950918F196091901970914F
:1061F000911988E296E00E944347409172195091AC
:106200007319609174197091751985E296E00E9476
:1062100043474091C2195091C3196091C4197091BC
:10622000C51982E296E00E94544740917619509138
:10623000771960917819709179198FE196E00E9431
:10624000434740917A1950917B1960917C19709164
:106250007D198CE196E00E94434740917E19509150
:106260007F19609180197091811989E196E00E94EF
:10627000434740918219509183196091841970911C
:10628000851986E196E00E9443478091C00085FF12
:10629000FCCF8AE08093C600FE018491EEEEFFE021
:1062A000882349F09091C00095FFFCCF8093C600F1
:1062B00031968491F5CFE4E0F6E08491882341F0B3
:1062C0009091C00095FFFCCF8093C6003196F5CF2A
:1062D0008091C00085FFFCCF8AE08093C600FE015C
:1062E0008491EEEEFFE0882349F09091C00095FF85
:1062F000FCCF8093C60031968491F5CF4091320B4C
:106300005091330B6091340B7091350B8BEF95E00E
:106310000E9443474091360B5091370B6091380BE8
:106320007091390B88EF95E00E94434740913A0BFA
:1063300050913B0B60913C0B70913D0B85EF95E0CC
:106340000E9443478091C00085FFFCCF8AE0809384
:10635000C600FE018491EEEEFFE0882349F09091A3
:10636000C00095FFFCCF8093C60031968491F5CF95
:10637000E7EEF5E08491882341F09091C00095FF0D
:10638000FCCF8093C6003196F5CF8091C00085FF89
:10639000FCCF8AE08093C600FE018491EEEEFFE020
:1063A000882349F09091C00095FFFCCF8093C600F0
:1063B00031968491F5CF4091AD025091AE0260913B
:1063C000AF027091B0028DED95E00E94434760915D
:1063D000A9027091AA028091AB029091AC020F9435
:1063E0009635AB01BC018AED95E00E944347609170
:1063F000A5027091A6028091A7029091A8020F9425
:10640000A235AB01BC0187ED95E00E944347809126
:10641000C00085FFFCCF8AE08093C600FE01849116
:10642000EEEEFFE0882349F09091C00095FFFCCF8D
:106430008093C60031968491F5CFE1ECF5E084912C
:10644000882341F09091C00095FFFCCF8093C60057
:106450003196F5CF8091C00085FFFCCF8AE0809314
:10646000C600FE018491EEEEFFE0882349F0909192
:10647000C00095FFFCCF8093C60031968491F5CF84
:1064800040919D0250919E0260919F027091A002E6
:1064900087EB95E00E9443476091990270919A02C0
:1064A00080919B0290919C020F949635AB01BC01A8
:1064B00084EB95E00E9443476091950270919602AB
:1064C00080919702909198020F94A235AB01BC0184
:1064D00081EB95E00E9443478091C00085FFFCCF8F
:1064E0008AE08093C600FE018491EEEEFFE08823EF
:1064F00049F09091C00095FFFCCF8093C600319683
:106500008491F5CFEDE7F5E08491882341F09091F7
:10651000C00095FFFCCF8093C6003196F5CF8091E7
:10652000C00085FFFCCF8AE08093C600FE01849105
:10653000EEEEFFE0882349F09091C00095FFFCCF7C
:106540008093C60031968491F5CF409124025091FA
:106550002502609126027091270283E795E00E9450
:10656000434720E030E040E752E460911C02709124
:106570001D0280911E0290911F020F9451BFAB012A
:10658000BC0180E795E00E9443474091220B509167
:10659000230B6091240B7091250B8DE695E00E94F2
:1065A00043478091C00085FFFCCF8AE08093C600FE
:1065B000FE018491EEEEFFE0882349F09091C00047
:1065C00095FFFCCF8093C60031968491F5CFE1E42E
:1065D000F5E08491882341F09091C00095FFFCCFB5
:1065E0008093C6003196F5CF8091C00085FFFCCF27
:1065F0008AE08093C600FE018491EEEEFFE08823DE
:1066000049F09091C00095FFFCCF8093C600319671
:106610008491F5CF40911E0B50911F0B6091200B80
:106620007091210B87E395E00E94434720E030E022
:1066300040E752E4609118027091190280911A02A9
:1066400090911B020F9451BFAB01BC0184E395E014
:106650000E9443478091C00085FFFCCF8AE0809371
:10666000C600FE018491EEEEFFE0882349F0909190
:10667000C00095FFFCCF8093C60031968491F5CF82
:10668000EAEDF4E08491882341F09091C00095FFF9
:10669000FCCF8093C6003196F5CF8091C00085FF76
:1066A000FCCF8AE08093C600FE018491EEEEFFE00D
:1066B000882349F09091C00095FFFCCF8093C600DD
:1066C00031968491F5CF4091270B50E060E070E067
:1066D00080ED94E00E9454478091C00085FFFCCF7C
:1066E0008AE08093C600FE018491EEEEFFE08823ED
:1066F00049F09091C00095FFFCCF8093C600319681
:106700008491F5CF80914E0B8823A1F1EDEBF4E05D
:106710008491882341F09091C00095FFFCCF809335
:10672000C6003196F5CF8091C00085FFFCCF8AE08E
:106730008093C600FE018491EEEEFFE0882349F0CD
:106740009091C00095FFFCCF8093C6003196849154
:10675000F5CF4091440250914502609146027091FC
:10676000470283EB94E00E9443478091C00085FF7D
:10677000FCCF11C0E7E9F4E08491882341F09091C7
:10678000C00095FFFCCF8093C6003196F5CF809175
:10679000C00085FFFCCF8AE08093C6001A3008F461
:1067A0003EC0FE01C491EEEEFFE0CC2349F08091A3
:1067B000C00085FFFCCFC093C6003196C491F5CFD1
:1067C000EEE7F4E08491882341F09091C00095FFBA
:1067D000FCCF8093C6003196F5CF8091C00085FF35
:1067E000FCCF8AE08093C6004091C1135091C21340
:1067F0006091C3137091C41384E794E00E944347EF
:106800004091BD135091BE136091BF137091C0139E
:106810008AE694E0DF91CF911F910C944347DF917A
:10682000CF911F910895AF92BF92CF92DF92EF92D6
:10683000FF920F931F93CF93DF93CDB7DEB7E0970F
:106840000FB6F894DEBF0FBECDBF80E1E3EEF2E0FD
:10685000DE01919601900D928A95E1F780E1E3EFD8
:10686000F2E0DE01519601900D928A95E1F780E108
:10687000E3E0F3E0DE01119601900D928A95E1F7D5
:106880006E0181E2C80ED11C82EAE82E89E1F82E61
:106890008E010F5E1F4F62EB79E1AE014F5F5F4FDC
:1068A00092E9A92E99E1B92E20E030E0F60181911C
:1068B0009191A191B1916F01F70181939193A1936E
:1068C000B1937F01F80181919191A191B1918F01D3
:1068D000FB0181939193A193B193BF01FA0181913F
:1068E0009191A191B191AF01F50181939193A19300
:1068F000B1935F012F5F3F4F24303105B9F60F94FC
:10690000F81180E090E4ACE9B4E480938A199093A4
:106910008B19A0938C19B0938D198093861990933D
:106920008719A0938819B093891910928E19109223
:106930008F19109290191092911980E29EE4A0E0B4
:10694000B0E08093C2199093C319A093C419B09377
:10695000C51910927219109273191092741910922D
:10696000751980E090E0A0E7B1E4809376199093E8
:106970007719A0937819B093791980937A19909325
:106980007B19A0937C19B0937D198DEC9CECACEC39
:10699000BEE380937E1990937F19A0938019B093E2
:1069A000811980E090E0A0E2B0E480938219909396
:1069B0008319A0938419B093851910923A0B109201
:1069C0003B0B10923C0B10923D0B1092360B109229
:1069D000370B1092380B1092390B1092320B109229
:1069E000330B1092340B1092350B8DE39AE0A1E833
:1069F000B1E48093AD029093AE02A093AF02B09346
:106A0000B0026DEC7CEC84E99FE30F9490356093C9
:106A1000A9027093AA028093AB029093AC0265E83E
:106A20007BEE80E692E40F949C356093A502709310
:106A3000A6028093A7029093A8020F94672480E097
:106A400090E0A0E8BFE38093A1029093A202A093FC
:106A5000A302B093A4021092270B80E090E0A0E480
:106A6000B0E48093240290932502A0932602B09371
:106A7000270240E050E064E372E440931C0250932C
:106A80001D0260931E0270931F021092220B10923F
:106A9000230B1092240B1092250B10921E0B1092B8
:106AA0001F0B1092200B1092210B40E050E060E091
:106AB00071E4409318025093190260931A02709384
:106AC0001B0210924E0B8093440290934502A093B8
:106AD0004602B09347020E94B85DEEEEFFE084915B
:106AE000882341F09091C00095FFFCCF8093C600B1
:106AF0003196F5CFEEE2F4E08491882341F0909155
:106B0000C00095FFFCCF8093C6003196F5CF8091F1
:106B1000C00085FFFCCF8AE08093C600E0960FB6E8
:106B2000F894DEBF0FBECDBFDF91CF911F910F91C3
:106B3000FF90EF90DF90CF90BF90AF9008951F939C
:106B4000CF93DF93CDB7DEB72C970FB6F894DEBFA7
:106B50000FBECDBF162F9C878B8786E591E3A0E003
:106B6000B0E089839A83AB83BC8344E0BE016B5F52
:106B70007F4FCE010B962ED843E050E0BE016B5FF5
:106B80007F4FCE0101960F945EC5892B09F0FFC09F
:106B900040E162EA79E1CE010B961CD840E162EB5C
:106BA00079E1CE010B9616D840E162E979E1CE0198
:106BB0000B9610D80F94F81144E06AE879E1CE0101
:106BC0000B9608D844E066E879E1CE010B9602D82E
:106BD00044E06EE879E1CE010B960E94EA2D44E094
:106BE00062E779E1CE010B960E94EA2D44E062EC67
:106BF00079E1CE010B960E94EA2D44E066E779E147
:106C0000CE010B960E94EA2D44E06AE779E1CE01BD
:106C10000B960E94EA2D44E06EE779E1CE010B96D7
:106C20000E94EA2D44E062E879E1CE010B960E94D1
:106C3000EA2D4CE062E37BE0CE010B960E94EA2D48
:106C400044E06BE27BE0CE010B960E94EA2D44E02B
:106C50006DEA72E0CE010B960E94EA2D44E069EAEB
:106C600072E0CE010B960E94EA2D44E065EA72E0E4
:106C7000CE010B960E94EA2D44E06DE972E0CE0150
:106C80000B960E94EA2D44E069E972E0CE010B9672
:106C90000E94EA2D44E065E972E0CE010B960E9465
:106CA000EA2D42E0BE01675F7F4FCE010B960E9446
:106CB000EA2D41E067E27BE0CE010B960E94EA2DCF
:106CC00044E064E272E0CE010B960E94EA2D44E0BB
:106CD0006CE172E0CE010B960E94EA2D44E062E284
:106CE0007BE0CE010B960E94EA2D44E06EE17BE052
:106CF000CE010B960E94EA2D44E068E172E0CE01DD
:106D00000B960E94EA2D41E06EE47BE0CE010B96EB
:106D10000E94EA2D44E064E472E0CE010B960E94EA
:106D2000EA2D1A3070F044E061EC73E1CE010B966D
:106D30000E94EA2D44E06DEB73E1CE010B960E94B8
:106D4000EA2D0E94B85D0F946724EEEEFFE0849177
:106D5000882341F09091C00095FFFCCF8093C6003E
:106D60003196F5CFE0E5F4E08491882341F09091ED
:106D7000C00095FFFCCF8093C6003196F5CF80917F
:106D8000C00085FFFCCF8AE08093C60001C04BDDC8
:106D90002C960FB6F894DEBF0FBECDBFDF91CF911A
:106DA0001F910895682F772767FD70958091A51032
:106DB0009091A61086559F4E0F9443C590939C10BA
:106DC00080939B1021E0892B09F420E0822F089505
:106DD00080919B1090919C1060E070E001960D9462
:106DE000ECC1282F6091581C7091591C90E02A30FA
:106DF00018F0895A9F4F01C0C0960D94B1C5CF932A
:106E0000C82F82958F70EDDF8C2F8F70CF91E9CFD7
:106E1000CF93C82F892FF3DF8C2FCF91F0CF6F92B4
:106E20007F928F929F92AF92BF92CF92DF92EF921A
:106E3000FF920F931F93CF93DF936B017C01EA01C5
:106E4000122F209709F455C0123011F48E2DC9DF8E
:106E5000C601DEDF6091581C7091591C80E290E001
:106E60000F94B1C5702E7C1A8C2F870D09F438C091
:106E70001130D1F088F0123029F5460157018FEF1B
:106E8000881A980AA80AB80AEE24D7FCE094FE2CC7
:106E9000EBBEF601679013C0F60160808FEFC81A51
:106EA000D80AE80AF80A0FC0460157018FEF881A7E
:106EB000980AA80AB80AC6010F94FAC8682E750184
:106EC000640101C0612C6091581C7091591C80E2D2
:106ED00090E00F94B1C5862D92DF219709F0C4CFC1
:106EE0006091581C7091591C8AE090E00F94B1C5D4
:106EF000A8CFDF91CF911F910F91FF90EF90DF907E
:106F0000CF90BF90AF909F908F907F906F9008959B
:106F1000CF93DF93FB0120E030E0DC01ED018D91A8
:106F20008823A1F14115510519F02417350774F58F
:106F30008032A1F38A3051F190ED980F9A3020F40D
:106F4000682F6295607F08C09FE9980F9630A8F47B
:106F5000682F6295607F6057CE0102967981A0ED1F
:106F6000A70FAA3018F4762F7A2B0CC0AFE9A70F21
:106F7000A63018F47755762B05C088279927821BF1
:106F8000930B05C071932F5F3F4FC7CFC901DF91AE
:106F9000CF9108958BE693E00F9444C6F894FFCF09
:106FA000E0919B10F0919C108181882399F082E4FC
:106FB000F9DE882369F0F89428E088E190E00FB6C4
:106FC000F894A895809360000FBE20936000FFCFD7
:106FD0000C9400000895F894C0E0D0E06FEFCE016B
:106FE0000F942AC92196C11580E2D807B9F728E085
:106FF00088E190E00FB6F894A895809360000FBEEA
:1070000020936000FFCF0F931F93CF93DF93CDB7F3
:10701000DEB762970FB6F894DEBF0FBECDBF81E436
:10702000C1DE8823A9F080919B1090919C10FC01F7
:107030002181283741F440E150E060E070E00296A1
:107040000F9454C303C0C4DE0F94EBBC8B0102C089
:1070500000E010E083E4A6DE882331F0B9DE0F946F
:10706000EBBC262F872F02C020E080E21F71422F49
:10707000582F4130F0E25F0710F040E050E2CA01C3
:10708000800F911F8130904220F040E050E2401B81
:10709000510B88E5498B5A8B85DE49895A898823AB
:1070A000D1F080919B1090919C1040E150E0BE0186
:1070B0006F5F7F4F01962CDFAC01009761F0FE01FE
:1070C0003196CF01840F951FD801E817F90719F001
:1070D00021912D93FACFB80180E090E000E120E00B
:1070E0009EDE62960FB6F894DEBF0FBECDBFDF9175
:1070F000CF911F910F910895AF92BF92CF92DF92DF
:10710000EF92FF920F931F93CF93DF93CDB7DEB72C
:1071100060970FB6F894DEBF0FBECDBF81E442DEAC
:107120008823A9F080919B1090919C10FC012181F3
:10713000283741F440E150E060E070E002960F949F
:1071400054C303C045DE0F94EBBC8B0102C000E0CA
:1071500010E083E427DE882331F03ADE0F94EBBCA5
:10716000262F872F02C020E080E21F71E22EF82E2A
:10717000F1E0EF16F0E2FF0618F0E12C90E2F92EB4
:10718000C701800F911F8130904228F0E12C80E2EE
:10719000F82EE01AF10A88E505DE882361F1809176
:1071A0009B1090919C1040E150E0BE016F5F7F4FBB
:1071B0000196AEDE7C010097F1F0CE0101965C01F4
:1071C000C12CD12CCE14DF0461F0F50161915F0177
:1071D000C601800F911F0F942AC9FFEFCF1ADF0A53
:1071E000F1CFC80115DE6091581C7091591C8AE0DE
:1071F00090E00F94B1C5B80180E090E000E121E09B
:10720000A7010DDE60960FB6F894DEBF0FBECDBFAE
:10721000DF91CF911F910F91FF90EF90DF90CF9072
:10722000BF90AF900895CF92DF92EF92FF9280E5EA
:10723000B9DD882309F44CC0CBDD0F94EBBC6B01A6
:107240007C018FEFC816D10411F008F041C086E42C
:10725000A9DD882379F0BCDD0F94EBBC61157105C5
:1072600011F460E004C06130710521F461E08C2DFF
:107270000F9490B586E596DD882399F0A9DD0F94EB
:10728000EBBC6115710511F460E004C0613071055B
:10729000F9F461E08C2DFF90EF90DF90CF900D948A
:1072A000C9B58C2D0F94FEB521E0892B09F420E09F
:1072B0001F922F93DF92CF928EE793E09F938F934D
:1072C0000F9410C60F900F900F900F900F900F908B
:1072D000FF90EF90DF90CF900895089508954F921A
:1072E0005F926F927F929F92AF92BF92CF92DF9206
:1072F000EF92FF920F931F93CF93DF9382E398E077
:107300009F938F930F9421C686EA9FE00F94FAC84B
:10731000C82FC090CB1AD090CC1AE090CD1AF09024
:10732000CE1AC701B6010E946E632B013C01E091A9
:107330009B10F0919C1092810F900F909F3311F051
:1073400091114CC091E0C11101C090E01F929F9338
:1073500083E298E09F938F930F9421C60F900F9034
:107360000F900F9000EB1FE0C3E2D0E0912C80E083
:1073700090E023E0A22E28E0B22EBC0180E090E055
:107380000F941CBD2091AA193091AB194091AC19F2
:107390005091AD190F9483BC20E030E04AE754E4EB
:1073A0000F9451BF0F94F0BC7F936F93DF93CF93F3
:1073B000BF92AF920F9421C693940F900F900F90AD
:1073C0000F900F900F9086E0981609F441C0C80105
:1073D0000F9407C925960E5F1F4FCFCF913221F52D
:1073E00061E086EA9FE00F942AC968E070E080EBD4
:1073F0009FE00F9438C968E170E082EB9FE00F9442
:1074000038C960E370E084EB9FE00F9438C960E511
:1074100070E086EB9FE00F9438C968E770E088EB76
:107420009FE00F9438C914C080E5BCDC882319F0B4
:10743000CFDC6B017C01C701B6010E946E632B019A
:107440003C018AE5AFDC882319F0C2DC2B013C014A
:1074500020E030E04AE754E4C301B2010F9451BF89
:107460000F94EBBCCB0168EE73E00F9440C19F9387
:107470008F93C301B2010F94EBBC7F936F93C7014D
:10748000B6010F94EBBC7F936F9383EE97E09F93CD
:107490008F930F9421C68DB79EB708960FB6F894B8
:1074A0009EBF0FBE8DBFDF91CF911F910F91FF90B7
:1074B000EF90DF90CF90BF90AF909F907F906F90B4
:1074C0005F904F90089566EE87EF9FE00D940CC992
:1074D00060E086E69FE00F940CC960E085E69FE0DF
:1074E0000F940CC960E084E69FE00D940CC96F9284
:1074F0007F928F929F92AF92BF92CF92DF92EF9244
:10750000FF920F931F93CF93DF9382ED97E09F93AA
:107510008F930F9421C688E545DC0F900F90811161
:1075200007C089E53FDC882309F4AAC0C1E001C097
:10753000C0E06C2E712CC3010E944D4C8C2F0F9417
:10754000613680E1EEE3FBE0A9E0BBE001900D9243
:107550008A95E1F7660C771C660C771CC301875F80
:10756000944F3C0180E090E0A8E4B3E4F301808311
:107570009183A283B38320E030E040E752E460913E
:1075800058027091590280915A0290915B020F94B7
:1075900083BC4B015C01E090110BF090120B009149
:1075A000130B1091140B20910D0B30910E0B409189
:1075B0000F0B5091100B6091090B70910A0B809189
:1075C0000B0B90910C0BCAE2DBE0DF93CF93E5E16C
:1075D000CE2EEBE0DE2E0F946D030F941C1D80E188
:1075E000EEE3FBE0A9E0BBE001900D928A95E1F7A4
:1075F000F301108211821282138220E030E040E712
:1076000052E4609158027091590280915A0290910F
:107610005B020F9483BC4B015C01E090110BF09076
:10762000120B0091130B1091140B20910D0B309144
:107630000E0B40910F0B5091100B6091090B709144
:107640000A0B80910B0B90910C0BDF93CF930F944F
:107650006D030F941C1D0F9470362FEF2093B20210
:107660009F938F938FEB97E09F938F930F9421C6F7
:107670008DB79EB708960FB6F8949EBF0FBE8DBF0C
:10768000DF91CF911F910F91FF90EF90DF90CF90FE
:10769000BF90AF909F908F907F906F900895E091F2
:1076A0009B10F0919C1085818F3311F081112BC0BC
:1076B00080919E131F928F9380919F131F928F939F
:1076C0008091A1138F938091A0138F938091A31326
:1076D0008F938091A2138F938091A4131F928F9305
:1076E0008091A5131F928F9387E893E09F938F93C8
:1076F0000F9410C68DB79EB70E960FB6F8949EBF26
:107700000FBE8DBF0895813229F50E9480FD8091C2
:107710009E131F928F9380919F131F928F9380913E
:10772000A1138F938091A0138F938091A3138F93B4
:107730008091A2138F9389E993E09F938F930F9485
:1077400010C68DB79EB70A960FB6F8949EBF0FBEAF
:107750008DBF089582E526DB81113ADB88E522DBC7
:10776000882339F035DB0F94EBBC7093A31360933F
:10777000A21389E517DB882339F02ADB0F94EBBCD1
:107780007093A1136093A0138CE40CDB882329F081
:107790001FDB0F94EBBC609368020895CF93DF93D7
:1077A000EC0160E08E810F94C9B581E090E00F9408
:1077B0000BB461E08E810F94C9B581E090E00F9425
:1077C0000BB460E08E810F94C9B584E690E0DF9140
:1077D000CF910D940BB4CF92DF92EF92FF920F9363
:1077E0001F93CF93DF937C01C0E0D0E0C62ED12C55
:1077F00087010C0F1D1F61E0F80187810F9490B580
:10780000B6010C2E02C0759567950A94E2F7617077
:10781000F80187810F94C9B52196C430D10541F78D
:10782000C701DF91CF911F910F91FF90EF90DF90F3
:10783000CF90B4CFCF92DF92EF92FF920F931F932E
:10784000CF93DF937C01C0E0D0E0C62ED12C87011E
:107850000C0F1D1F61E0F80187810F9490B5B601F0
:107860000C2E02C0759567950A94E2F76170F801D5
:1078700087810F94C9B52196C830D10541F7C7015A
:10788000DF91CF911F910F91FF90EF90DF90CF90FC
:1078900085CF1F93CF93DF93EC01162F642F8C813C
:1078A0000F94C9B58D818F3F19F060E00F94C9B571
:1078B0008F85612F84FF05C0CE01DF91CF911F918D
:1078C000B9CF70E084E0759567958A95E1F7CE01B0
:1078D00082DF612FCE01DF91CF911F917CCF40E0FD
:1078E000D8CF61E0FCDF80E496E00D940BB462E059
:1078F000F6DF80E496E00D940BB4CF93DF93CDB721
:10790000DEB728970FB6F894DEBF0FBECDBF28E0D4
:10791000E3E1F3E0DE01119601900D922A95E1F783
:10792000FC012389421710F04FEF420FFE01319600
:10793000E40FF11DE40FF11D2081260F2068622F56
:1079400028960FB6F894DEBF0FBECDBFDF91CF9162
:10795000C6CFFC016089262F2460208B6C60BFCFCE
:10796000CF93DF93EC01423018F08F8588608F87CA
:107970004B8B1C8A222329F0413019F48F858460B7
:107980008F8780E593EC0F940BB460E08C810F94AB
:10799000C9B560E08E810F94C9B58D818F3F19F014
:1079A00060E00F94C9B56F8564FD19C063E0CE0136
:1079B00012DF84E991E10F940BB463E0CE010BDF99
:1079C00084E991E10F940BB463E0CE0104DF86E912
:1079D00090E00F940BB462E0CE01FDDE13C0606254
:1079E000CE017DDF84E991E10F940BB46F85606275
:1079F000CE0175DF86E990E00F940BB46F8560626D
:107A0000CE016DDF6F856062CE0169DF8CE390E0AF
:107A10000F940BB484E0888BCE019BDF8CE390E065
:107A20000F940BB4CE015DDF88EB9BE00F940BB499
:107A300082E0898B66E0CE0152DF8CE390E00F9408
:107A40000BB41D8ADF91CF9108956F927F928F9230
:107A5000AF92CF92EF920F931F93CF93DF93CDB757
:107A6000DEB73C01162F842F5E854F8538899989B2
:107A7000F301848325830683E782C086A1868286FC
:107A8000538744873587968761E00F9490B5F3015B
:107A900085818F3F19F061E00F9490B561E0F301AB
:107AA00086810F9490B5112319F0F301178603C056
:107AB00080E1F301878720E041E060E1C301DF91CD
:107AC000CF911F910F91EF90CF90AF908F907F90BB
:107AD0006F9046CF8F92AF92CF92EF920F93DC01CF
:107AE00013961C921E921297E2EBF3E0ED93FC9337
:107AF0001F921F921F921F928C2CAE2CC02EE22E32
:107B0000042F2FEF462F61E0A0DF0F900F900F9012
:107B10000F900F91EF90CF90AF908F900895CF93EB
:107B2000DF93EC01423018F08F8588608F874B8B94
:107B30001C8A222329F0413019F48F8584608F87B5
:107B400080E593EC0F940BB460E08C810F94C9B581
:107B500060E08E810F94C9B58D818F3F19F060E090
:107B60000F94C9B56F8564FD19C063E0CE0133DEA3
:107B700084E991E10F940BB463E0CE012CDE84E93B
:107B800091E10F940BB463E0CE0125DE86E990E02D
:107B90000F940BB462E0CE011EDE13C06062CE0112
:107BA0009EDE84E991E10F940BB46F856062CE0193
:107BB00096DE86E990E00F940BB46F856062CE018B
:107BC0008EDE6F856062CE018ADE8CE390E00F94DA
:107BD0000BB484E0888BCE01BCDE8CE390E00F9484
:107BE0000BB4CE0184DE80E496E00F940BB482E007
:107BF000898B66E0CE0173DE8CE390E00F940BB4CA
:107C000040E068E0CE0179DE6AE279E0CE010F94CF
:107C100064B641E068E0CE0170DE6AE279E0CE0150
:107C20000F9464B642E066E0CE0167DE68E279E078
:107C3000CE01DF91CF910D9464B6FC0160896D7F18
:107C4000608B68604CCECF93DF93EC01262F8D893B
:107C50008230B0F0FE01E80FF11D658B3E8980EDAA
:107C6000860F8A3058F4316081E090E00D8802C0C0
:107C7000880F991F0A94E2F7382B01C03E7F3E8B94
:107C80004D8981E0840F8D8B50E04830510508F01C
:107C9000B6C0FA01EE58FF4F0D9491C12B3109F097
:107CA000AEC0AEC01E8A2B3509F0A9C0A9C02233D0
:107CB00009F4A6C02F3309F4A3C08E897AC08F8936
:107CC000823331F08F3349F4223309F098C098C0E1
:107CD0002A3419F4CE0105DE92C08E8982FF8FC04E
:107CE0002B3309F066C08CC08F898F3341F4888DA7
:107CF000823309F084C0253309F081C081C08E89A8
:107D000082FF7DC0988D9B3311F480FD79C083FF85
:107D100076C02B3309F073C073C04F894F3371F4B1
:107D2000888D823309F06BC0898D853309F067C077
:107D30002C3609F064C0CE0180DF61C08E8982FFDD
:107D40005EC0988D9B3339F484FF05C0283489F5D3
:107D50004053698D2CC083FF52C0998D9B3309F02D
:107D60004EC027C08E8982FF4AC0488D4B3361F4D4
:107D7000982F9073903341F4283431F44F89405355
:107D80006A8D6053898D32C083FF39C0998D9B33D2
:107D9000B1F585FF34C0283461F440538F89880FD2
:107DA0008056982F990F990F980F490F6A8D60533D
:107DB00024C080FF24C024C08E89982F9C709C30E2
:107DC000F1F4998D9B33D9F480768036C1F4283450
:107DD000B1F4488D40538F89880F8056982F990FA2
:107DE000990F980F490F6B8D60538A8D880F8056BD
:107DF000982F990F990F980F690FCE017EDD1D8A7C
:107E000081E090E0DF91CF910895CF92DF92EF92E1
:107E1000FF920F931F93CF93DF931F921F92CDB7C3
:107E2000DEB78C01677088E0689FB0011124606440
:107E3000C80149835A8353DD4981C42E5A81D52E06
:107E4000E12CF12CD6016D916D01D801ED91FC91E1
:107E50000190F081E02DC8011995BFEFEB1AFB0AE4
:107E6000E8E0EE16F10471F70F900F90DF91CF91DB
:107E70001F910F91FF90EF90DF90CF900895FC013C
:107E80002589211102C06B3109F4DDCE41E001DD0D
:107E900081E090E008951F920F920FB60F92112487
:107EA0000BB60F922F933F934F935F936F938F93E4
:107EB0009F93EF93FF938091C00084FF03C0809154
:107EC000C60019C06091C60020915D0A30915E0A1B
:107ED000C90101968F77992740915F0A5091600AF6
:107EE0008417950741F0F901E352F64F60839093B0
:107EF0005E0A80935D0AFF91EF919F918F916F9140
:107F00005F914F913F912F910F900BBE0F900FBE3D
:107F10000F901F9018951F920F920FB60F92112479
:107F20000BB60F922F933F934F935F936F938F9363
:107F30009F93EF93FF938091610A813001F58091C7
:107F4000D00084FF03C08091D60019C06091D60094
:107F500020915D0A30915E0AC90101968F779927B9
:107F600040915F0A5091600A8417950741F0F9012A
:107F7000E352F64F608390935E0A80935D0AFF910F
:107F8000EF919F918F916F915F914F913F912F91C1
:107F90000F900BBE0F900FBE0F901F901895CF92B1
:107FA000DF92EF92FF926A017B01411581EE580743
:107FB0006105710509F463C082E08093C00060E050
:107FC00079E08DE390E0A70196010F9475C12150EF
:107FD000310941095109CA01B90122E030E040E00C
:107FE00050E00F9475C191E03093C5002093C40018
:107FF0008091C10080618093C1008091C100886040
:108000008093C1008091C10080688093C1008091FD
:10801000610A8130D1F5992341F082E08093D0004C
:1080200060E079E08DE390E006C01092D00060E857
:1080300074E88EE190E0A70196010F9475C121507C
:10804000310941095109CA01B90122E030E040E09B
:1080500050E00F9475C13093D5002093D4008091E7
:10806000D10080618093D1008091D100886080939D
:10807000D1008091D10080688093D10006C0109219
:10808000C00090E020E130E0AFCFFF90EF90DF90B4
:10809000CF90089520915F0A3091600A80915D0A27
:1080A00090915E0A8217930771F0F901E352F64F3F
:1080B00080812F5F3F4F2F7733273093600A2093C3
:1080C0005F0A90E008958FEF9FEF089580915F0A17
:1080D0009091600A90935E0A80935D0A08954F9292
:1080E0005F926F927F928F929F92AF92BF92CF9248
:1080F000DF92EF92FF920F931F93CF93DF93CDB751
:10810000DEB7A0970FB6F894DEBF0FBECDBF5C01FF
:108110004115510561057105E9F420E030E040E3C7
:1081200050E060E070E0A0960FB6F894DEBF0FBE9E
:10813000CDBFDF91CF911F910F91FF90EF90DF9016
:10814000CF90BF90AF909F908F907F906F905F90F7
:108150004F905BC08E010F5F1F4FC12CD12C760159
:108160004801422E512C612C712C8FEFC81AD80A6D
:10817000E80AF80ACB01BA01A30192010F9453C196
:10818000CA01F80161938F01A901BC014115510594
:108190006105710551F7F1E0CF1AD108E108F10846
:1081A000F401EC0DFD1D80818A3010F440E301C024
:1081B00047E3480F552747FD5095652F752F20E061
:1081C00030E0C50122D081E0C81AD108E108F108E9
:1081D000EFEFCE16DE06EE06FE0611F7A0960FB6FE
:1081E000F894DEBF0FBECDBFDF91CF911F910F91ED
:1081F000FF90EF90DF90CF90BF90AF909F908F90C7
:108200007F906F905F904F9008952115310539F45C
:108210008091C00085FFFCCF4093C60008952A30AE
:10822000310509F43FC05BCF9A01462F552747FD22
:108230005095652F752FE9CFCF93DF93EC0120E0A8
:1082400030E04DE050E060E070E0DFDF20E030E063
:108250004AE050E060E070E0CE01DF91CF91D5CFF1
:10826000FB012191BF01222339F03091C00035FF7D
:10827000FCCF2093C600F4CFDFCF9A01AB01662775
:1082800057FD6095762FC1CFCF93DF93EC019A0114
:10829000AB01662757FD6095762FB7DFCE01DF91E2
:1082A000CF91CACFCF92DF92EF92FF92CF93DF931D
:1082B000EC016A017B0177FF0FC020E030E04DE266
:1082C00050E060E070E0A1DFF094E094D094C094BE
:1082D000C11CD11CE11CF11C2AE0B701A601CE0192
:1082E000DF91CF91FF90EF90DF90CF90F8CE2115E6
:1082F000310539F48091C00085FFFCCF4093C60062
:108300000895EDCECF93DF93EC019A01462F50E014
:1083100060E070E0ECDFCE01DF91CF918DCFCF93A5
:10832000DF93EC019A01AB0160E070E0E0DFCE0189
:10833000DF91CF9181CFCF93DF93EC01D8DFCE01D6
:10834000DF91CF9179CF8F929F92AF92BF92CF92D0
:10835000DF92EF92FF921F93CF93DF93EC016A01BC
:108360007B01122F20E030E0A901C701B6010F9474
:108370007CBC87FF0CC020E030E04DE250E060E0C4
:1083800070E0CE0142DFF7FAF094F7F8F094B12CE8
:1083900060E070E080E09FE3B11641F020E030E063
:1083A00040E251E40F9483BCB394F6CF9B01AC013F
:1083B000C701B6010F94A3BB6B017C010F94F0BC05
:1083C0004B015C010F941CBD9B01AC01C701B601C0
:1083D0000F94A2BB6B017C012AE0B501A401CE0180
:1083E0007EDE112361F0EDE0F6E08191882339F023
:1083F0009091C00095FFFCCF8093C600F6CF11236B
:1084000019F120E030E040E251E4C701B6010F94D9
:1084100051BF6B017C010F94EBBC4B01AA2497FC6C
:10842000A094BA2CB501A401CE013CDFC501B40172
:108430000F941EBD9B01AC01C701B6010F94A2BBF6
:108440006B017C011150DBCFDF91CF911F91FF9029
:10845000EF90DF90CF90BF90AF909F908F90089556
:1084600072CFCF93DF93EC016EDFCE01DF91CF911E
:10847000E3CE9091C00095FFFCCF8093C60080E0D2
:1084800090E00895FC01659175918591949108950E
:10849000EF92FF920F931F93CF93DF93EC01CC0FDA
:1084A000DD1FCC0FDD1FCE018653904FEBDF9E0109
:1084B000225C344F79018E010E5C144FF80120814B
:1084C0003181428153810F94A3BBF7016083718393
:1084D00082839383CE018E51904FD4DF9E012C5C1A
:1084E0003D4F7901F80120813181428153810F9400
:1084F000A3BBF7016083718382839383CE018A5289
:10850000904FC0DFC85DDD4FF8012081318142818D
:1085100053810F94A3BB688379838A839B83DF9104
:10852000CF911F910F91FF90EF900895CF93C82F97
:1085300040910C0250910D0260910E0270910F0259
:108540004093F50A5093F60A6093F70A7093F80A7D
:1085500020915602309157023093C30B2093C20BE7
:1085600024E630E030935702209356020F94A5B3CF
:108570006093F00A7093F10A8093F20A9093F30AE1
:108580008C2FCF910D94A11380E00F94A1138091B3
:10859000F50A9091F60AA091F70AB091F80A809333
:1085A0000C0290930D02A0930E02B0930F028091E3
:1085B000C20B9091C30B90935702809356020F9475
:1085C000A5B36093F00A7093F10A8093F20A909336
:1085D000F30A0895682F772767FD70958091A5109D
:1085E0009091A61086559F4E0F9443C590939C1072
:1085F00080939B1021E0892B09F420E0822F0895BD
:1086000080919B1090919C104AE050E060E070E0F7
:1086100001960F9454C3CB01089580919B109091C3
:108620009C104AE050E060E070E001960D9454C365
:108630002091A5103091A610BC01C90186559F4E0E
:108640000F947BC590939C1080939B1021E0892B05
:1086500009F420E0822F08950F931F93CF93DF93A7
:1086600000919B1010919C1065E470E0C8010F947C
:1086700043C5EC01009751F460E070E0C801019639
:10868000DF91CF911F910F910D94ECC118828091D1
:108690009B1090919C1060E070E001960F94ECC1EB
:1086A00025E42883DF91CF911F910F910895809148
:1086B0009B1090919C1060E070E001960D94ECC1CD
:1086C0002F923F924F925F926F927F928F929F92E2
:1086D000AF92BF92CF92DF92EF92FF920F931F93D0
:1086E000CF93DF93CDB7DEB760970FB6F894DEBFB8
:1086F0000FBECDBF1C012A013B014801590120E0FA
:1087000030E04CE052E4C301B2010F94A2BB25E576
:1087100035E547E052E40F9483BC6B017C010F9474
:1087200059BD0F94EBBC8B0177FF12C020E030E005
:1087300040E85FE3C701B6010F947FBE18160CF046
:108740005DC0C12CD12CE0E8EE2EEFE3FE2E56C02A
:1087500066307105DCF02AEA3AE24CE453E4C301E6
:10876000B2010F94A2BB25E535E547E052E40F9432
:1087700083BC6B017C0120E030E0A9010F947CBC3C
:1087800087FF3FC0C12CD12C76013BC0882777FDE5
:108790008095982F0F941EBD25E535E547E052E4FE
:1087A0000F9451BF20E030E04CE052E40F94A3BBA3
:1087B0009B01AC01C301B2010F94A2BB25E535E5D5
:1087C00047E052E40F9483BC6B017C0120E030E071
:1087D000A9010F947CBC87FD17C020E030E040E881
:1087E0005FE3C701B6010F947FBE181684F4C12C55
:1087F000D12C70E8E72E7FE3F72E09C000E010E0EF
:1088000006C005E010E003C0C12CD12C760120E0A9
:1088100030E040EC50E4C501B4010F94A2BB2BEA58
:108820003AEA42E052E40F9483BC2B013C010F94DE
:1088300059BD0F94EBBC788B6F8777FF12C020E097
:1088400030E040E85FE3C301B2010F947FBE181629
:108850000CF05FC0412C512C60E8662E6FE3762E41
:1088600058C0AF85B8891697E4F026E535E549E2AA
:1088700053E4C501B4010F94A2BB2BEA3AEA42E0EB
:1088800052E40F9483BC2B013C0120E030E0A901AD
:108890000F947CBC87FD40C0E5E0F0E0F88BEF87EB
:1088A00046C0882777FD8095982F0F941EBD2BEA30
:1088B0003AEA42E052E40F9451BF20E030E040EC4D
:1088C00050E40F94A3BB9B01AC01C501B4010F940C
:1088D000A2BB2BEA3AEA42E052E40F9483BC2B019C
:1088E0003C0120E030E0A9010F947CBC87FD1CC056
:1088F00020E030E040E85FE3C301B2010F947FBEA7
:108900001816ACF4412C512C50E8652E5FE3752EFF
:108910000EC0188A1F860BC0412C512C320125E055
:1089200030E0388B2F8703C0412C512C3201A70136
:10893000960160E070E080E89FE30F94A2BB69833A
:108940007A838B839C83C80101969E838D83AF8538
:10895000B8891196BA87A987A301920160E070E0F7
:1089600080E89FE30F94A2BB6B877C878D879E87EF
:1089700047E02F853889429FF001439FF00D112475
:10898000F887EF83E00FF11FEE0FFF1FEE0FFF1FC1
:10899000E20DF31D218132814381548169817A8105
:1089A0008B819C810F9451BF4B015C01EF81F88555
:1089B0008D819E81E80FF91FEE0FFF1FEE0FFF1F45
:1089C000E20DF31D2181328143815481C701B6013B
:1089D0000F9451BF9B01AC01C501B4010F94A3BB1F
:1089E0009B01AC016B857C858D859E850F9451BF65
:1089F0004B015C0127E0E985FA852E9FD0012F9F6E
:108A0000B00D1124B887AF83FD01E00FF11FEE0F09
:108A1000FF1FEE0FFF1FE20DF31D21813281438105
:108A2000548169817A818B819C810F9451BF6983C4
:108A30007A838B839C83AF81B8858D819E81A80FBB
:108A4000B91FAA0FBB1FAA0FBB1FA20DB31D119602
:108A50002D913D914D915C911497C701B6010F94F2
:108A600051BF9B01AC0169817A818B819C810F94FC
:108A7000A3BB9B01AC01C301B2010F9451BF9B0189
:108A8000AC01C501B4010F94A3BB60960FB6F89476
:108A9000DEBF0FBECDBFDF91CF911F910F91FF9031
:108AA000EF90DF90CF90BF90AF909F908F907F908E
:108AB0006F905F904F903F902F9008954F925F92EC
:108AC0006F927F929F92AF92BF92CF92DF92EF927E
:108AD000FF920F931F93CF93DF937C015B018A0179
:108AE000E9019090D812911014C0FC01808191810D
:108AF000A281B381FA0180839183A283B383FB01B6
:108B000080819181A281B38188839983AA83BB8369
:108B10007FC091FE55C0FC0120813181428153818B
:108B20006091C8127091C9128091CA129091CB12B3
:108B30000F9451BF2B013C01F5012081318142810D
:108B400053816091CC127091CD128091CE12909190
:108B5000CF120F9451BF9B01AC01C301B2010F941E
:108B6000A3BBF8016083718382839383F701208123
:108B70003181428153816091D0127091D1128091E4
:108B8000D2129091D3120F9451BF6B017C01F50169
:108B900020813181428153816091D4127091D5122C
:108BA0008091D6129091D7120F9451BF9B01AC01C6
:108BB000C701B6010F94A3BB688379838A839B8323
:108BC00090FE26C02091B0123091B1124091B212A5
:108BD0005091B312F80160817181828193810F9469
:108BE000A3BBF80160837183828393832091B412C5
:108BF0003091B5124091B6125091B71268817981C7
:108C00008A819B810F94A3BB688379838A839B832A
:108C1000DF91CF911F910F91FF90EF90DF90CF9058
:108C2000BF90AF909F907F906F905F904F9008950E
:108C30002F923F924F925F926F927F928F929F926C
:108C4000AF92BF92CF92DF92EF92FF920F931F935A
:108C5000CF93DF93CDB7DEB728970FB6F894DEBF7A
:108C60000FBECDBF8C011B019E012F5F3F4FAE0198
:108C70004B5F5F4F23DF20E030E0A9016D817E81F3
:108C80008F8198850F947CBC87FF07C01D821E8250
:108C90001F821886FF24F39401C0F12C20E030E0FD
:108CA00040E850EC69817A818B819C810F947CBC77
:108CB00087FF0AC080E090E0A0E8B0EC89839A8347
:108CC000AB83BC83FF24F39420E030E04FE753E410
:108CD0006D817E818F8198850F947FBE181654F424
:108CE00080E090E0AFE7B3E48D839E83AF83B887E5
:108CF000FF24F39420E030E042E553E469817A8177
:108D00008B819C810F947FBE18164CF480E090E01C
:108D1000A2E5B3E489839A83AB83BC8303C0FF20BD
:108D200009F483C0C980DA80EB80FC808D809E804E
:108D3000AF80B8847090D81271100BC0F801808297
:108D40009182A282B382F101C082D182E282F38257
:108D50006AC070FE1CC02091B0123091B1124091D7
:108D6000B2125091B312C501B4010F94A2BB4B01D2
:108D70005C012091B4123091B5124091B61250911D
:108D8000B712C701B6010F94A2BB6B017C0171FE43
:108D90004AC02091B8123091B9124091BA12509144
:108DA000BB12C501B4010F9451BF2B013C012091AE
:108DB000BC123091BD124091BE125091BF12C7013A
:108DC000B6010F9451BF9B01AC01C301B2010F94D6
:108DD000A3BBF80160837183828393832091C012C7
:108DE0003091C1124091C2125091C312C501B40119
:108DF0000F9451BF4B015C012091C4123091C512F8
:108E00004091C6125091C712C701B6010F9451BFCD
:108E10009B01AC01C501B4010F94A3BBF1016083B8
:108E2000718382839383FF24F3948F2D28960FB64A
:108E3000F894DEBF0FBECDBFDF91CF911F910F9190
:108E4000FF90EF90DF90CF90BF90AF909F908F906A
:108E50007F906F905F904F903F902F900895CF93A9
:108E6000DF931F92CDB7DEB7BE016F5F7F4F0F94C8
:108E7000A7980F90DF91CF910895682F87EF9FE01B
:108E80000D940CC90895FC012491222341F03091E6
:108E9000C00035FFFCCF2093C6000196F4CF22E03E
:108EA00030E08CED99E0DCCAFC012491222341F0F2
:108EB0003091C00035FFFCCF2093C6000196F4CF5F
:108EC0002AE030E08CED99E012CACF9366EB73E0B4
:108ED0008CED99E0C5D9C1E0C093B1026FEF89E68E
:108EE0009FE00F940CC9C093DF02CF91089566EC08
:108EF00073E08CED99E0B4D91092B10260E089E69C
:108F00009FE00F940CC91092DF02089587ED93E063
:108F10009F938F930F9410C60F941C1D81E00F94A4
:108F200068980F94CE4E82E00F94A19586E69FE05C
:108F30000F94FAC861E0680F86E69FE00F940CC9B1
:108F400081E00F94689882E00F94A195E0918E0BD8
:108F5000F0E0EE0FFF1FEF5FF14C859194910F94BD
:108F6000E64F61E089EA9FE00E943EC161E083EA4A
:108F70009FE00E943EC10F900F9061E085E99FE065
:108F80000C943EC11092CE0B60E08CEC9BE00E94F2
:108F900090BA81E08093B1020895EF92FF920F930F
:108FA0001F93CF93DF931F92CDB7DEB789830F94C2
:108FB000CE4E8981823009F468C0B4F5882309F463
:108FC00042C0813009F0F4C09FB7F894809102014B
:108FD0008460809302019FBFEFEFF1EE24E0E15047
:108FE000F0402040E1F700C000009FB7F894809166
:108FF00002018B7F809302019FBF40E050E0BA01E5
:109000008DEE9FE00F941EC940E050E0BA0181EF61
:109010009FE00F941EC90F90DF91CF911F910F9188
:10902000FF90EF900D94A377833009F45CC08430F7
:1090300009F0BEC00F90DF91CF911F910F91FF906B
:10904000EF900D9477A09FB7F8948091020184600F
:10905000809302019FBF2FEF81EE94E0215080406A
:109060009040E1F700C000009FB7F89480910201A2
:109070008B7F809302019FBF0F90DF91CF911F9153
:109080000F91FF90EF900D94774F0F94774F80EFF3
:10909000F4DE1092F31B1092F21B6091F41B84EC2F
:1090A0009FE00F940CC962EF7BE181EC9FE00F948D
:1090B000FC4E9FB7F8948091020184608093020176
:1090C0009FBF8FEF91EEE4E081509040E040E1F7E8
:1090D00000C000009FB7F894809102018B7F8093BD
:1090E00002019FBF65C087E89FE00F94186646E7BE
:1090F0005FE062E081E00F94E77B9FB7F894809196
:1091000002018460809302019FBFFFEF21EE84E0A3
:10911000F15020408040E1F700C000009FB7F89474
:10912000809102018B7F809302019FBF1092DC0A25
:109130001092DB0A4FE65FE063E083E00F94E77B89
:109140004091DB0A5091DC0A63E083E00F94D94E32
:10915000E12CF12C09E210E06FEFC7010F942AC94E
:10916000C701B8010F9440C1892BD9F48091DB0A63
:109170009091DC0A01969093DC0A8093DB0A48E622
:109180005FE063E083E00F94E77B4091DB0A50915E
:10919000DC0A63E083E00F94D94E86E69FE00F94EB
:1091A00018669FEFE91AF90AE114E0E1FE06A1F65C
:1091B0000F90DF91CF911F910F91FF90EF90089545
:1091C0006DEC7AE086E39FE00D94E3C58F929F9269
:1091D000AF92BF92CF92DF92EF92FF928091F41BF9
:1091E00081119DC00F94A5B36B017C0120911002E9
:1091F000222309F48CC0409115025091160241308F
:10920000510509F484C08091110290911202A0913D
:109210001302B091140246015701881A990AAA0A4A
:10922000BB0A30E0A8EEB3E00F9497C1861697060C
:10923000A806B9060CF473C04430510559F13CF44A
:10924000423051050CF463C0EEEEFFE00EC0453035
:10925000510509F05CC0EEEEFFE042C09091C00005
:1092600095FFFCCF8093C600319684918111F6CF93
:10927000E0E8FEE08491882341F09091C00095FFE2
:10928000FCCF8093C6003196F5CF8091C00085FF5A
:10929000FCCF3AC0EEEEFFE08491882341F090913C
:1092A000C00095FFFCCF8093C6003196F5CFEAE66B
:1092B000FEE08491882341F09091C00095FFFCCF9F
:1092C0008093C6003196F5CF8091C00085FFFCCF1A
:1092D0001BC09091C00095FFFCCF8093C6003196D3
:1092E00084918111F6CFE3E5FEE08491882341F07B
:1092F0009091C00095FFFCCF8093C6003196F5CFCA
:109300008091C00085FFFCCF8AE08093C600C092A8
:109310001102D0921202E0921302F0921402FF9016
:10932000EF90DF90CF90BF90AF909F908F90089577
:1093300080E1EEE3FBE0A9E0BBE001900D928A95AD
:10934000E1F708954F925F926F927F928F929F9272
:10935000AF92BF92CF92DF92EF92FF92CF93DF93C3
:1093600000D01F92CDB7DEB70F941C1D8BE432D90D
:10937000882391F071D96B017C0120E030E0A901D4
:109380000F947FBE87FD08C0C092C113D092C21354
:10939000E092C313F092C41382E51CD9882359F0DC
:1093A0005BD96B017C0120E030E0A9010F947CBC0B
:1093B00087FF83C006C0C12CD12CE0E8EE2EEFEB76
:1093C000FE2E84E407D9882321F046D94B015C01A5
:1093D00006C0812C912C70E8A72E7FEBB72E87E575
:1093E000F9D8882321F038D92B013C0106C0412C43
:1093F000512C60E8662E6FEB762E88E4EBD888233C
:1094000031F02AD969837A838B839C8308C080E0FA
:1094100090E0A0E8BFEB89839A83AB83BC8320E014
:1094200030E0A901C501B4010F947FBE87FD45C09E
:1094300020E030E0A901C301B2010F947FBE87FD97
:109440003CC020E030E0A90169817A818B819C8158
:109450000F947FBE87FD31C020E030E0A901C50137
:10946000B4010F947CBC882391F120E030E040E00F
:109470005FE3C501B4010F9451BF6B017C012981E9
:109480003A814B815C81C301B2010F9451BF4B0102
:109490005C01A7019601C701B6010F9451BF2BEDE6
:1094A0003FE049E450E40F9451BF9B01AC01C5017A
:1094B000B4010F9483BC6B017C0120E030E0A90172
:1094C000C701B6010F947FBE87FF04C00BC0C12C3B
:1094D000D12C7601C092BD13D092BE13E092BF137F
:1094E000F092C013EEEEFFE08491882341F090915A
:1094F000C00095FFFCCF8093C6003196F5CFECE01D
:10950000FBE08491882341F09091C00095FFFCCF4F
:109510008093C6003196F5CF4091C1135091C2138C
:109520006091C3137091C41322E030E08CED99E098
:109530000E9430428091C00085FFFCCF8AE080937A
:10954000C600E6E0FBE08491882341F09091C000E2
:1095500095FFFCCF8093C6003196F5CFC090BD1328
:10956000D090BE13E090BF13F090C01320E030E025
:10957000A901C701B6010F947CBC882369F022E0E1
:1095800030E0B701A6018CED99E00E943042809155
:10959000C00085FFFCCF11C0E1E0FBE0849188238F
:1095A00041F09091C00095FFFCCF8093C6003196AA
:1095B000F5CF8091C00085FFFCCF8AE08093C60084
:1095C0000F900F900F900F90DF91CF91FF90EF9041
:1095D000DF90CF90BF90AF909F908F907F906F90D3
:1095E0005F904F9008952F923F924F925F926F92AB
:1095F0007F928F929F92AF92BF92CF92DF92EF9223
:10960000FF920F931F93CF93DF931F92CDB7DEB7D7
:109610000F94CE4EE3EEF0E44591549161E080E08A
:109620000F94E77B81E00F94A1138983E1EBFFE0C6
:10963000E4918E2F992781950CF490951C0184E07C
:109640000F94F938A6E4BBE01D921D921D921C9266
:109650001397E2E4FBE02081318142815381AEE344
:10966000BBE06D917D918D919C91FAE4CF2EFBE052
:10967000DF2EE12CF12C87010F941B1059DE86ECB4
:109680009FE00E9442422DEC3CEC4CE85FE30F94DB
:1096900051BF4B015C01B101882777FD8095982F60
:1096A0000F941EBD9B01AC01C501B4010F9451BFC5
:1096B000E1E1FBE020813181428153810F94A3BB22
:1096C0002B013C01A1E1BBE06D937D938D939C93B5
:1096D0001397E0E6F2E0608171818281938160936B
:1096E0000C0270930D0280930E0290930F0220E003
:1096F00030E040E752E40F9483BC4B015C01ADE0E5
:10970000BBE02D913D914D915C91E9E0FBE06081E2
:10971000718182819381AAE2BBE0BF93AF93A5E1FF
:10972000CA2EABE0DA2E830172010F946D0382E042
:109730000F944A360F941C1D0F94793980E00F94D2
:10974000A113A6E4BBE01D921D921D921C921397DB
:10975000E2E4FBE02081318142815381AEE3BBE052
:109760006D917D918D919C91BAE4CB2EBBE0DB2E67
:10977000E12CF12C87010F941B10DADD8AE0829D29
:10978000B001839D700D1124882777FD8095982F57
:109790000F941EBDE1E1FBE02081318142815381C4
:1097A0000F94A3BB2B013C01A1E1BBE06D937D9322
:1097B0008D939C93139720E030E040E05FE3E0E678
:1097C000F2E060817181828193810F9451BF609337
:1097D0000C0270930D0280930E0290930F0220E012
:1097E00030E040E752E40F9483BC4B015C01ADE0F4
:1097F000BBE02D913D914D915C91E9E0FBE06081F2
:10980000718182819381AAE2BBE0BF93AF9315E19E
:10981000C12E1BE0D12E830172010F946D030F94B2
:109820001C1D89810F94A11380E090E0A4E5B3E4AE
:10983000E6E4FBE080839183A283B383A2E4BBE0F0
:109840002D913D914D915C91EEE3FBE06081718142
:10985000828193810AE4C02E0BE0D02EE12CF12C02
:1098600004E513E40F941B1081E00F900F900F900C
:109870000F900F90DF91CF911F910F91FF90EF907C
:10988000DF90CF90BF90AF909F908F907F906F9020
:109890005F904F903F902F9008952F923F924F925C
:1098A0005F926F927F928F929F92AF92BF92CF9270
:1098B000DF92EF92FF920F931F93CF93DF93CDB779
:1098C000DEB729970FB6F894DEBF0FBECDBF3C01BF
:1098D00081E00F94A1138F8382E06816710408F071
:1098E00081C2F301E155F04FE491D301AA0FBB1FF0
:1098F000AA0FBB1FBA83A983A85ABD4FBE83AD83ED
:109900008D919D910D90BC91A02D80930C02909310
:109910000D02A0930E02B0930F0281E0062C01C04D
:10992000880F0A94EAF70F94F938E981FA81E25C2A
:10993000F44FF987E8871082118212821382E09037
:10994000460BF090470B0091480B1091490B20916A
:10995000420B3091430B4091440B5091450B609169
:109960003E0B70913F0B8091400B9091410BEAE4CC
:10997000CE2EEBE0DE2E0F941B10E981FA81E75F1B
:10998000F44F2F0180E090E0A0E4B0E48083918365
:10999000A283B38320E030E040E752E460910C0200
:1099A00070910D0280910E0290910F020F9483BC72
:1099B0004B015C01E090110BF090120B0091130B26
:1099C0001091140B20910D0B30910E0B40910F0B49
:1099D0005091100B6091090B70910A0B80910B0B49
:1099E00090910C0BFAE22F2EFBE03F2E3F922F922C
:1099F000A5E1CA2EABE0DA2E0F946D030F941C1D67
:109A00000F94891380E00F94A113A885B9851D9246
:109A10001D921D921C921397E090460BF090470BFD
:109A20000091480B1091490B2091420B3091430B50
:109A30004091440B5091450B60913E0B70913F0B50
:109A40008091400B9091410BBAE4CB2EBBE0DB2E12
:109A50000F941B1080E090E0A0E8BFEBF201808340
:109A60009183A283B38320E030E040E752E4609129
:109A70000C0270910D0280910E0290910F020F94D2
:109A800083BC4B015C01E090110BF090120B009134
:109A9000130B1091140B20910D0B30910E0B409174
:109AA0000F0B5091100B6091090B70910A0B809174
:109AB0000B0B90910C0B3F922F92E5E1CE2EEBE039
:109AC000DE2E0F946D030F941C1D81E00F94A113E3
:109AD00089819A818254904F0E9442422DEC3CEC45
:109AE0004CE85FEB0F9451BFD2016D937D938D9342
:109AF0009C93139720E030E040E752E460910C0221
:109B000070910D0280910E0290910F020F9483BC10
:109B10004B015C01E090110BF090120B0091130BC4
:109B20001091140B20910D0B30910E0B40910F0BE7
:109B30005091100B6091090B70910A0B80910B0BE7
:109B400090910C0B3F922F920F946D030F941C1D5C
:109B50000F94891380E00F94A113E885F985108292
:109B6000118212821382E090460BF090470B009115
:109B7000480B1091490B2091420B3091430B4091BF
:109B8000440B5091450B60913E0B70913F0B8091BF
:109B9000400B9091410BFAE4CF2EFBE0DF2E0F94A7
:109BA0001B1080E090E0A0E2B1E4F2018083918399
:109BB000A283B38320E030E040E752E460910C02DE
:109BC00070910D0280910E0290910F020F9483BC50
:109BD0004B015C01E090110BF090120B0091130B04
:109BE0001091140B20910D0B30910E0B40910F0B27
:109BF0005091100B6091090B70910A0B80910B0B27
:109C000090910C0B3F922F92A5E1CA2EABE0DA2E79
:109C10000F946D030F941C1D0F94891381E00F9412
:109C2000A11380E090E0A0E7B1ECF2018083918382
:109C3000A283B38320E030E040E05FE3AD81BE81EA
:109C40006D917D918D919C910F9451BF60930C0209
:109C500070930D0280930E0290930F0220E030E08B
:109C600040E752E40F9483BC4B015C01E090110B80
:109C7000F090120B0091130B1091140B20910D0B0F
:109C800030910E0B40910F0B5091100B6091090B0E
:109C900070910A0B80910B0B90910C0B3F922F92BD
:109CA0000F946D030F941C1DC3010E944842F301E1
:109CB000E15DF44F81E080830F9479390F9489132B
:109CC00080E00F94A1132AE037ED43E25FE3E885DB
:109CD000F98560817181828193810F94A2BBA885EF
:109CE000B9856D937D938D939C931397E090460B6C
:109CF000F090470B0091480B1091490B2091420BBB
:109D00003091430B4091440B5091450B60913E0BB9
:109D100070913F0B8091400B9091410BBAE4CB2E98
:109D2000BBE0DB2E0F941B102AE037ED43E25FE32C
:109D3000E885F98560817181828193810F94A3BB4D
:109D4000A885B9856D937D938D939C931397F201AC
:109D500060837183828393832AE939E949E95EE369
:109D600060910C0270910D0280910E0290910F0291
:109D70000F9451BF20E030E040E752E40F9483BCE1
:109D80004B015C01E090110BF090120B0091130B52
:109D90001091140B20910D0B30910E0B40910F0B75
:109DA0005091100B6091090B70910A0B80910B0B75
:109DB00090910C0B3F922F92E5E1CE2EEBE0DE2E40
:109DC0000F946D030F941C1D10920C0210920D0243
:109DD00010920E0210920F020FB6F894DEBF0FBE63
:109DE000CDBF62C192E06916710409F05DC1E1EB7B
:109DF000FFE074901092460B1092470B1092480BA4
:109E00001092490B2091420B3091430B4091440B2F
:109E10005091450B60913E0B70913F0B8091400B30
:109E20009091410BFAE4CF2EFBE0DF2EE12CF12CD8
:109E300087010F941B1086EC9FE00E9442424B0169
:109E40005C01672D772767FD7095872F972F0F94FB
:109E50001EBD2B013C0120E030E040EC5FE3C5017A
:109E6000B4010F9451BFA30192010F9451BF6983B4
:109E70007A838B839C836093110B7093120B809376
:109E8000130B9093140B60916002709161028091AA
:109E900062029091630260930C0270930D028093B2
:109EA0000E0290930F0220E030E040E752E40F945E
:109EB00083BC4B015C0120910D0B30910E0B409146
:109EC0000F0B5091100B6091090B70910A0B809150
:109ED0000B0B90910C0BAAE22A2EABE03A2E3F928C
:109EE0002F92B5E1CB2EBBE0DB2EE980FA800B810F
:109EF0001C810F946D030F941C1D1092460B109241
:109F0000470B1092480B1092490B2091420B309155
:109F1000430B4091440B5091450B60913E0B709167
:109F20003F0B8091400B9091410B1AE4C12E1BE036
:109F3000D12EE12CF12C87010F941B108AEB9FE0AE
:109F40000E9442429058A30192010F9451BF69832D
:109F50007A838B839C836093110B7093120B809395
:109F6000130B9093140B20E030E040E752E4609133
:109F70000C0270910D0280910E0290910F020F94CD
:109F800083BC4B015C0120910D0B30910E0B409175
:109F90000F0B5091100B6091090B70910A0B80917F
:109FA0000B0B90910C0B3F922F9205E1C02E0BE012
:109FB000D02EE980FA800B811C810F946D030F94E1
:109FC0001C1D8AEB9FE00E9442429B01AC010F9452
:109FD000A3BBA30192010F9451BF2B013C016093DD
:109FE000110B7093120B8093130B9093140B20E0C2
:109FF00030E040E05FE36091600270916102809127
:10A000006202909163020F9451BF60930C027093AF
:10A010000D0280930E0290930F0220E030E040E7A3
:10A0200052E40F9483BC4B015C0120910D0B3091E5
:10A030000E0B40910F0B5091100B6091090B70911A
:10A040000A0B80910B0B90910C0B3F922F92830186
:10A0500072010F946D030F941C1D82E090E00E942A
:10A0600048428091460B9091470BA091480BB091CC
:10A07000490B8093110B9093120BA093130BB09389
:10A08000140B10920C0210920D0210920E021092FC
:10A090000F020F94891381E08093310B0F900F9082
:10A0A0000F900F900F900F908F8129960FB6F89414
:10A0B000DEBF0FBECDBFDF91CF911F910F91FF90FB
:10A0C000EF90DF90CF90BF90AF909F908F907F9058
:10A0D0006F905F904F903F902F900D94A113CF926F
:10A0E000DF92EF92FF920F931F9322D980E090E0CE
:10A0F000D4DB81E090E0D1DBE090460BF090470BA1
:10A100000091480B1091490B2091420B3091430B69
:10A110004091440B5091450B60913E0B70913F0B69
:10A120008091400B9091410BFAE4CF2EFBE0DF2EA3
:10A130000F941B101F910F91FF90EF90DF90CF9025
:10A140000D9489130F94A5B36093F00A7093F10AEC
:10A150008093F20A9093F30A089520E030E0A90179
:10A1600068EB71E084E50F94FDB769E170E080E091
:10A1700090E00F94D4B384E50F9421BB64E170E0C8
:10A1800080E090E00D94D4B37F928F929F92AF9233
:10A19000BF92CF92DF92EF92FF920F931F93CF93D4
:10A1A000DF9300D01F92CDB7DEB71092DA1A10926B
:10A1B000D91A1092D81A1092D71A0F94CE4E81E95C
:10A1C0009EE00F9418668E010F5F1F4F7E0125E001
:10A1D000E20EF11C8CED99E00E944A408F3FEFEFB8
:10A1E0009E07C1F3F80181938F01EE15FF0591F7EA
:10A1F00089809A80AB80BC808091C00085FFFCCFB5
:10A200008BE28093C600C12CD12C7601ABE27A2E72
:10A2100080918D0B882309F450C00EE71AE0C81412
:10A22000D904EA04FB04A1F08CED99E00E944A40B5
:10A230008F3FFFEF9F07C1F32FEFC21AD20AE20A46
:10A24000F20AF80181938F01FAE00E3B1F0739F7FC
:10A250006EE77AE08CEC9BE00E945DB98091C000D3
:10A2600085FFFCCF7092C6000F94082AC814D90449
:10A27000EA04FB0469F671DF60E08CEC9BE00E946D
:10A2800090BA10928D0BEFE7F0E485919491FC0168
:10A290002491222341F03091C00035FFFCCF209360
:10A2A000C6000196F4CF8091C00085FFFCCF8AE004
:10A2B0008093C60080E090E000C00F900F900F9058
:10A2C0000F90DF91CF911F910F91FF90EF90DF9052
:10A2D000CF90BF90AF909F908F907F9008952F92D6
:10A2E0003F924F925F926F927F928F929F92AF9226
:10A2F000BF92CF92DF92EF92FF920F931F93CF9373
:10A30000DF931F921F92CDB7DEB7382E811112C096
:10A310001092D81A1092D71A1092DA1A1092D91AEB
:10A320001092DC1A1092DB1A1092DE1A1092DD1ACB
:10A330000F94234F80E00F94689889ED92E10E947A
:10A3400008F80E946FD90E9459F710922F0B1092B3
:10A35000300B1092310B81E00E949642EFE4F1E461
:10A36000859194910E942F47BADE3DD9882309F444
:10A3700079C1E8DE31104EC084E090E0909316027F
:10A3800080931502EBEAFEE38591949140E060E052
:10A390000F94559A882331F0E7E6FFE38591949175
:10A3A0000F946DA2E0918E0BF0E0EE0FFF1FE353D0
:10A3B000FF4B859194910F946DA2E0918E0BF0E08C
:10A3C000EE0FFF1FE754F04C859194910F946DA20E
:10A3D00082E090E09093160280931502E0918E0B3C
:10A3E000F0E0EE0FFF1FE958FF4B859194910E941A
:10A3F0002F4741E050E062E080E00F94D94EE091B9
:10A400008E0BF0E0EE0FFF1FED58FF4B85919491FE
:10A410000F94186680E090E0A0EAB0E48093460BC9
:10A420009093470BA093480BB093490B20E030E08A
:10A4300040E252E460916002709161028091620298
:10A44000909163020F9483BC4B015C012091420BFD
:10A450003091430B4091440B5091450B60913E0B62
:10A4600070913F0B8091400B9091410BEAE2FBE031
:10A47000FF93EF93EAE4CE2EEBE0DE2EE12CF12CFD
:10A4800000EA10E40F946D030F941C1D86E50E94F2
:10A49000EA420F900F90882361F0E0919B10F091B9
:10A4A0009C108181893039F08F7D41F00E940043FA
:10A4B00003C01A8205C081E08A8302C0A1E0AA839A
:10A4C0003320B1F00E94C4420E94C4D90E94E0DB54
:10A4D0000E94B4F0882309F4C1C087EF9FE00F9475
:10A4E000FAC8803F09F0BAC081E00E943D47B6C07B
:10A4F0008FEF0E943D4760E070E088EF9FE00F948F
:10A5000026C91982BE016F5F7F4F8A810E9485ED47
:10A510003C010E94C442212C312C10EA412E10E44F
:10A52000512E2092460B3092470B4092480B50928E
:10A53000490B20E030E040E252E46091600270910B
:10A54000610280916202909163020F9483BC4B017F
:10A550005C012091420B3091430B4091440B509190
:10A56000450B60913E0B70913F0B8091400B909199
:10A57000410BAAE2BBE0BF93AF930AE4C02E0BE00D
:10A58000D02E820171010F946D030F941C1D0F904A
:10A590000F9077FC47C0198289ED92E10E9408F87C
:10A5A0000E9436D981E00E94964299DDAE014F5F4C
:10A5B0005F4F6A8181E00E94DAF23C010E94C4424E
:10A5C0002092460B3092470B4092480B5092490B19
:10A5D00020E030E040E252E460916002709161025C
:10A5E00080916202909163020F9483BC4B015C01E5
:10A5F0002091420B3091430B4091440B5091450BFD
:10A6000060913E0B70913F0B8091400B9091410BFC
:10A61000AAE2BBE0BF93AF930F946D030F941C1D90
:10A620000F900F906981C3010F94D7A277FC16C0D9
:10A6300086EE0E943D478FE59FE00F94FAC8813077
:10A6400059F0E0918E0BF0E0EE0FFF1FEB5BFE4B3D
:10A65000859194910F946DA211E001C010E00F94C8
:10A66000793901C010E081E00F946898812F0F9034
:10A670000F90DF91CF911F910F91FF90EF90DF909E
:10A68000CF90BF90AF909F908F907F906F905F9092
:10A690004F903F902F9008958F929F92AF92BF92CC
:10A6A000CF92DF92EF92FF920F931F93CF93DF939E
:10A6B000159881E08093820B82E090E09093800B6C
:10A6C00080937F0BE0918E0BF0E0EE0FFF1FED5DAE
:10A6D000FF4B859194910F94E64F20E030E04CE8D9
:10A6E00052E460914A0B70914B0B80914C0B90910E
:10A6F0004D0B0F94A3BB60934A0B70934B0B80934D
:10A700004C0B90934D0BE090460BF090470B009153
:10A71000480B1091490B2091420B3091430B409113
:10A72000440B5091450B60913E0B70913F0B809113
:10A73000400B9091410BCAE2DBE0DF93CF93812C79
:10A74000912CE0ECAE2EE0E4BE2EFAE4CF2EFBE03E
:10A75000DF2E0F946D0320E030E048EC51E460916F
:10A760004A0B70914B0B80914C0B90914D0B0F94B9
:10A77000A3BB60934A0B70934B0B80934C0B90934D
:10A780004D0BE090460BF090470B0091480B109159
:10A79000490B2091420B3091430B4091440B509157
:10A7A000450B60913E0B70913F0B8091400B909157
:10A7B000410BDF93CF93812C912CA0E8AA2EAFE31D
:10A7C000BA2E0F946D030F941C1D0F900F900F90D5
:10A7D0000F908091F41B882331F181E00F946898E9
:10A7E00082E00F94A195E0918E0BF0E0EE0FFF1F39
:10A7F000EF5FF14C859194910F94E64F1092810B8D
:10A800001092820B1092800B10927F0BDF91CF91F0
:10A810001F910F91FF90EF90DF90CF90BF90AF907E
:10A820009F908F9008958091810B8823B1F2E091E1
:10A830008E0BF0E0EE0FFF1FED57FF4B85919491CB
:10A8400041E060E00F94559A91E0811101C090E0E1
:10A85000CAE2DBE09111C1CF81E00F94689882E0F9
:10A860000F94A19520E030E048EC51E460914A0B50
:10A8700070914B0B80914C0B90914D0B0F94A3BB9F
:10A8800060934A0B70934B0B80934C0B90934D0B42
:10A89000E090460BF090470B0091480B1091490B4C
:10A8A0002091420B3091430B4091440B5091450B4A
:10A8B00060913E0B70913F0B8091400B9091410B4A
:10A8C000DF93CF93812C912CE0E8AE2EEFE3BE2EE8
:10A8D000FAE4CF2EFBE0DF2E0F946D030F941C1DC6
:10A8E000E0918E0BF0E0EE0FFF1FED57FF4B8591CF
:10A8F000949141E060E00F94559A0F900F90811170
:10A900006CCFAACF0F94A5B36093F00A7093F10AAD
:10A910008093F20A9093F30AE091A510F091A610AB
:10A92000E955FF4E80818130B9F4EDEBFFE385916D
:10A930009491FC012491222341F03091C00035FF15
:10A94000FCCF2093C6000196F4CF8091C00085FF14
:10A95000FCCF8AE08093C60008958CED99E00E94B8
:10A960006640E5E6FFE385919491FC012491222362
:10A9700041F03091C00035FFFCCF2093C600019616
:10A98000F4CF40918B1050918C1060918D1070918C
:10A990008E104F5F5F4F6F4F7F4F2AE030E08CED9E
:10A9A00099E00E9405418091C00085FFFCCF8AE0BC
:10A9B0008093C600A7CF8F929F92AF92BF92CF9203
:10A9C000DF92EF92FF920F931F93CF93DF93B9EB38
:10A9D000EB2EB5E0FB2E0EE31BE0C9E0DBE084ECE0
:10A9E000C82E8BE0D82EF70181917F010E94EA42A8
:10A9F000882319F10E9457434B015C01F6018081C5
:10AA0000811103C06091F40A01C061E070E080E050
:10AA100090E00F941EBDF801208131814281538165
:10AA20000F9451BF9B01AC01C501B4010F94A3BBAE
:10AA3000688379838A839B8309C0F801808191812F
:10AA4000A281B38188839983AA83BB830C5F1F4F44
:10AA50002496FFEFCF1ADF0A8DEBE81685E0F806A3
:10AA600011F686E40E94EA428823D9F00E945743F7
:10AA70006B017C016093F90A7093FA0A8093FB0AD8
:10AA80009093FC0A20E030E0A9010F947FBE1816D5
:10AA900044F4C0920C02D0920D02E0920E02F092A9
:10AAA0000F02DF91CF911F910F91FF90EF90DF90F8
:10AAB000CF90BF90AF909F908F9008957CDF89E4F6
:10AAC0000E94EA42882359F00E9457436093FD0A8E
:10AAD0007093FE0A8093FF0A9093000B08C01092B7
:10AAE000FD0A1092FE0A1092FF0A1092000B8AE4EF
:10AAF0000E94EA42882359F00E9457436093010B59
:10AB00007093020B8093030B9093040B08951092A3
:10AB1000010B1092020B1092030B1092040B08957C
:10AB2000CF92DF92EF92FF92CF93DF93EC01BC01C3
:10AB30006C5F7F4F0E94184620E030E0A9016091D1
:10AB40003C0270913D0280913E0290913F020F9431
:10AB5000A3BB6B017C019B01AC01688579858A856B
:10AB60009B850F947CBC87FF04C0C886D986EA8683
:10AB7000FB86C0903002D0903102E0903202F0901B
:10AB80003302A7019601688579858A859B850F9494
:10AB90007FBE181624F4C886D986EA86FB86DF9124
:10ABA000CF91FF90EF90DF90CF9008952F923F923A
:10ABB0004F925F926F927F928F929F92AF92BF92CD
:10ABC000CF92DF92EF92FF920F931F93CF93DF9379
:10ABD000CDB7DEB7AB970FB6F894DEBF0FBECDBFD3
:10ABE0009F878E87798B688B5B8B4A8B3D8B2C8BF9
:10ABF0001F8B0E8BED82DC018D909D90AD90BC90F3
:10AC000040903E0B50903F0B6090400B7090410B7A
:10AC1000DB018D919D910D90BC91A02D8887998726
:10AC2000AA87BB87C090420BD090430BE090440BA7
:10AC3000F090450B2091460B3091470B4091480B0B
:10AC40005091490BEA89FB896081718182819381EE
:10AC50000F94A2BB688F798F8A8F9B8F8091D912B6
:10AC6000811173C0AE89BF898D909D90AD90BC90CD
:10AC7000EA89FB89E080F18002811381A889B98982
:10AC80002D913D914D915C91EE85FF8560817181A3
:10AC900082819381FE013596FF93EF93CC88DD8806
:10ACA0000F946D03EE85FF8580819181A281B38130
:10ACB00080933E0B90933F0BA093400BB093410BBE
:10ACC000E889F98980819181A281B3818093420BC7
:10ACD0009093430BA093440BB093450BEA89FB89F7
:10ACE00080819181A281B3818093460B9093470B21
:10ACF000A093480BB093490BEC89FD898081918129
:10AD0000A281B38180934A0B90934B0BA0934C0B81
:10AD1000B0934D0B0F900F90AB960FB6F894DEBF2B
:10AD20000FBECDBFDF91CF911F910F91FF90EF909C
:10AD3000DF90CF90BF90AF909F908F907F906F905B
:10AD40005F904F903F902F900895A3019201C5010D
:10AD5000B4010F94A2BB2B013C0120E030E0A9011B
:10AD60000F947FBE53014201181624F0B7FAB09435
:10AD7000B7F8B094A7019601688579858A859B8587
:10AD80000F94A2BB688779878A879B8720E030E091
:10AD9000A9010F947FBE288539854A855B851816E1
:10ADA0000CF05058C501B4010F94A3BB6B017C019A
:10ADB00020E030E0A9010F947FBE18160CF052CFAE
:10ADC00020E030E040EF51E4C701B6010F9483BCAE
:10ADD0000F9469BC0F94EBBC7D876C876230710562
:10ADE0000CF440CF20914A0B30914B0B40914C0B0F
:10ADF00050914D0BAC89BD896D917D918D919C9148
:10AE00000F94A2BB6C8F7D8F8E8F9F8F22242394F3
:10AE1000312C8C859D85AA2797FDA095BA2F88A7F0
:10AE200099A7AAA7BBA7DE011596BF83AE83B10180
:10AE3000882777FD8095982F0F941EBD6B017C01AC
:10AE400068A579A58AA59BA50F941EBD9B01AC01A1
:10AE5000C701B6010F9483BC6B017C01EE89FF89A9
:10AE600080809180A280B3802C8D3D8D4E8D5F8D32
:10AE70000F9451BF9B01AC0160914A0B70914B0B39
:10AE800080914C0B90914D0B0F94A3BB69837A83F7
:10AE90008B839C83288D398D4A8D5B8DC701B601CC
:10AEA0000F9451BF2091460B3091470B4091480BB6
:10AEB0005091490B0F94A3BB68A379A38AA39BA3CA
:10AEC000288539854A855B85C701B6010F9451BF36
:10AED0002091420B3091430B4091440B5091450B14
:10AEE0000F94A3BB6CA37DA38EA39FA3A301920188
:10AEF000C701B6010F9451BF20913E0B30913F0B1B
:10AF00004091400B5091410B0F94A3BBFF81FF93E5
:10AF10002E812F93DE0111966D01E8A0F9A00AA100
:10AF20001BA12CA13DA14EA15FA10F946D03BFEF0A
:10AF30002B1A3B0A0F900F90EC85FD852E163F06CD
:10AF400009F075CF8FCE4F925F926F927F928F9262
:10AF50009F92AF92BF92CF92DF92EF92FF920F93A8
:10AF60001F93CF93DF93CDB7DEB728970FB6F89432
:10AF7000DEBF0FBECDBF89E09BE0D2DD0F94A5B34D
:10AF80006093F00A7093F10A8093F20A9093F30AA7
:10AF90008091090B90910A0BA0910B0BB0910C0BB7
:10AFA0008D839E83AF83B8879C01AD0160913E0B7A
:10AFB00070913F0B8091400B9091410B0F947CBCA2
:10AFC000811197C040900D0B50900E0B60900F0BAD
:10AFD0007090100BA30192016091420B7091430B92
:10AFE0008091440B9091450B0F947CBC811181C0E2
:10AFF00020E030E040E752E460910C0270910D02D5
:10B0000080910E0290910F020F9483BC4B015C0162
:10B01000E090110BF090120B0091130B1091140B98
:10B020008AE29BE09F938F9325E1C22E2BE0D22EE4
:10B03000A30192016D817E818F8198850F946D03AC
:10B040000F900F908091090B90910A0BA0910B0B20
:10B05000B0910C0B80933E0B90933F0BA093400B51
:10B06000B093410B80910D0B90910E0BA0910F0BA3
:10B07000B091100B8093420B9093430BA093440B21
:10B08000B093450B8091110B9091120BA091130B73
:10B09000B091140B8093460B9093470BA093480BF1
:10B0A000B093490B8091150B9091160BA091170B43
:10B0B000B091180B80934A0B90934B0BA0934C0BC1
:10B0C000B0934D0B28960FB6F894DEBF0FBECDBFE0
:10B0D000DF91CF911F910F91FF90EF90DF90CF9074
:10B0E000BF90AF909F908F907F906F905F904F90A8
:10B0F0000895E0902A0B60915602709157028827BC
:10B1000077FD8095982F0F941EBD20910C023091F1
:10B110000D0240910E0250910F020F9451BF2EE389
:10B1200033EC4EE259E30F9451BF69837A838B83EA
:10B130009C838E010F5F1F4F25E13BE041E15BE007
:10B140006DE07BE089E09BE031DD7CCF4F925F9248
:10B150006F927F928F929F92AF92BF92CF92DF9227
:10B16000EF92FF920F931F93CF93C62FE0912A0B7C
:10B17000F0E0882309F4D9C0DF01AA5DB44F8C91B7
:10B180008111AFC180913E0B90913F0BA091400B7C
:10B19000B091410B8093090B90930A0BA0930B0B7A
:10B1A000B0930C0B8091420B9091430BA091440BF8
:10B1B000B091450B80930D0B90930E0BA0930F0B4A
:10B1C000B093100B8091460B9091470BA091480BC8
:10B1D000B091490B8093110B9093120BA093130B1A
:10B1E000B093140BC0904A0BD0904B0BE0904C0BDB
:10B1F000F0904D0BC092150BD092160BE092170BEE
:10B20000F092180BEE0FFF1FEE0FFF1FE05CFD4FDB
:10B210002081318142815381662349F0609120026F
:10B2200070912102809122029091230208C06091C6
:10B2300024027091250280912602909127020F949A
:10B2400083BC9B01AC01C701B6010F94A3BB609303
:10B250004A0B70934B0B80934C0B90934D0B8AE4ED
:10B260009BE00F94C61180900C0290900D02A0906C
:10B270000E02B0900F0220E030E040E752E460910F
:10B280001C0270911D0280911E0290911F020F946A
:10B2900051BF60930C0270930D0280930E02909345
:10B2A0000F02E0912A0BF0E0EA5DF44F81E0808329
:10B2B0004ADE2091220B3091230B4091240B5091B8
:10B2C000250B6091460B7091470B8091480B909134
:10B2D000490B0F94A2BB7B018C016093460B7093CA
:10B2E000470B8093480B9093490B2091420B309170
:10B2F000430B4091440B5091450B60913E0B709174
:10B300003F0B8091400B9091410BEAE4CE2EEBE095
:10B31000DE2E0F941B1017DE80920C0290920D020D
:10B32000A0920E02B0920F02DCC0EA5DF44F808161
:10B33000882309F4D6C080903E0B90903F0BA090DC
:10B34000400BB090410B8092090B90920A0BA09297
:10B350000B0BB0920C0B4090420B5090430B609043
:10B36000440B7090450B40920D0B50920E0B609267
:10B370000F0B7092100B6091460B7091470B8091F0
:10B38000480B9091490B6093110B7093120B8093B3
:10B39000130B9093140B00914A0B10914B0B2091BF
:10B3A0004C0B30914D0B0093150B1093160B209303
:10B3B000170B3093180B2091220B3091230B4091E7
:10B3C000240B5091250B0F94A3BB7B018C01609340
:10B3D000460B7093470B8093480B9093490B3AE4CC
:10B3E000C32E3BE0D32EA3019201C501B4010F94FB
:10B3F0001B1010912A0BCC2389F020911A0B30914D
:10B400001B0B40911C0B50911D0B60912002709101
:10B410002102809122029091230210C020911E0BE4
:10B4200030911F0B4091200B5091210B6091240211
:10B430007091250280912602909127020F94A3BB60
:10B4400024E0129FF0011124E05CFD4F2081318146
:10B45000428153810F9483BC9B01AC0160914A0BE4
:10B4600070914B0B80914C0B90914D0B0F94A2BBA4
:10B4700060934A0B70934B0B80934C0B90934D0B46
:10B480008AE49BE00F94C611C0900C02D0900D028C
:10B49000E0900E02F0900F0220E030E040E752E42E
:10B4A000609118027091190280911A0290911B020A
:10B4B0000F9451BF60930C0270930D0280930E02A3
:10B4C00090930F02E0912A0BF0E0EA5DF44F1082B6
:10B4D0003ADDC0920C02D0920D02E0920E02F09280
:10B4E0000F02CF911F910F91FF90EF90DF90CF90BF
:10B4F000BF90AF909F908F907F906F905F904F9094
:10B500000895AF92BF92CF92DF92EF92FF920F9386
:10B510001F93CF93DF93D82F2091010B3091020B13
:10B520004091030B5091040B6091FD0A7091FE0A4B
:10B530008091FF0A9091000B0F948CBEC62F172F9D
:10B54000082FF92E6091560270915702882777FDD7
:10B550008095982F0F941EBD20910C0230910D0202
:10B5600040910E0250910F020F9451BF20E030E045
:10B5700040E752E40F9483BC20E030E048EC52E412
:10B580000F9483BC20912A0B2F93DF93FF920F938C
:10B590001F93CF935B016C01B2E0EB2E01E020E042
:10B5A0004DEF5AE069E07BE08EE39BE00E94EDF90D
:10B5B0008091090B90910A0BA0910B0BB0910C0B91
:10B5C00080933E0B90933F0BA093400BB093410BA5
:10B5D00080910D0B90910E0BA0910F0BB091100B61
:10B5E0008093420B9093430BA093440BB093450B75
:10B5F0008091110B9091120BA091130BB091140B31
:10B600008093460B9093470BA093480BB093490B44
:10B610008091150B9091160BA091170BB091180B00
:10B6200080934A0B90934B0BA0934C0BB0934D0B14
:10B630000F94A5B36093F00A7093F10A8093F20A15
:10B640009093F30A0F900F900F900F900F900F9020
:10B65000DF91CF911F910F91FF90EF90DF90CF90EE
:10B66000BF90AF900895EC01EAEFFAE0849188234F
:10B6700041F09091C00095FFFCCF8093C6003196B9
:10B68000F5CF70E04AE050E08CED99E00E94444133
:10B69000F8940F941427179A10922F0B169A109261
:10B6A000300B149AE4EFFFE08491882341F09091ED
:10B6B000C00095FFFCCF8093C6003196F5CFEFE92F
:10B6C000F0E485919491FC012491222341F0309182
:10B6D000C00035FFFCCF2093C6000196F4CF8091C7
:10B6E000C00085FFFCCF8AE08093C6002097C9F098
:10B6F000FE018491FE01882349F09091C00095FFDE
:10B70000FCCF8093C60031968491F5CF8091C00024
:10B7100085FFFCCF8AE08093C600CE010E942F47B0
:10B7200006C0E7E3F0E4859194910F94115078946A
:10B73000C6E0D0E0219751F068EC70E080E090E046
:10B740000F94D4B380E00F94A195F4CFF894A8950A
:10B75000FECFCF92DF92EF92FF920F931F93CF9382
:10B76000C82F8091A1109091A210039714F40E9409
:10B77000EAC20F94A5B30091EC0A1091ED0A209152
:10B78000EE0A3091EF0AC090F00AD090F10AE090F2
:10B79000F20AF090F30A6C197D098E099F090617C9
:10B7A00017072807390740F4012B022B032B21F040
:10B7B00064E08DE599E057DF40910802509109025D
:10B7C00060910A0270910B02452B462B472B19F111
:10B7D0000F94A5B30091F00A1091F10A2091F20A9A
:10B7E0003091F30A601B710B820B930B00910802DE
:10B7F0001091090220910A0230910B0206171707D7
:10B800002807390740F49091C6138091C513981307
:10B8100002C0CC2349F0CF911F910F91FF90EF9080
:10B82000DF90CF900D949B01179A10922F0B169AD0
:10B830001092300B149AEFCF0F9414278091DE0AE8
:10B8400081113DC081E08093DE0A80918B10909140
:10B850008C10A0918D10B0918E10809387109093D2
:10B860008810A0938910B0938A10E4EFFFE08491D0
:10B87000882341F09091C00095FFFCCF8093C600D3
:10B880003196F5CFE5E9F0E485919491FC0124919E
:10B89000222341F03091C00035FFFCCF2093C60039
:10B8A0000196F4CF8091C00085FFFCCF8AE08093A1
:10B8B000C600E7EAFEE3859194910D94E64F089562
:10B8C0008091DE0A0895CF93DF93EC0180912A0BDB
:10B8D0008093DF0A84E50E94EA42811102C080E081
:10B8E00084C00E9457430F94F0BC6093DF0A662324
:10B8F000B1F3EEEEFFE08491882341F09091C00017
:10B9000095FFFCCF8093C6003196F5CFCD36D1059B
:10B9100009F435C064F4C836D105B1F0C936D10593
:10B9200009F052C0E7E1F0E4A591B49124C0CA3D0A
:10B93000D10509F432C0CD3DD10509F045C0E7E09D
:10B94000F0E4A591B4913DC0E9E1F0E485919491D2
:10B95000FC012491222309F437C03091C00035FF47
:10B96000FCCF2093C6000196F3CF9091C00095FFC5
:10B97000FCCF8093C6008D918111F7CF25C0E5E102
:10B98000F0E4A591B4918D918823F1F09091C000DD
:10B9900095FFFCCF8093C600F6CFE9E0F0E4A591D7
:10B9A000B4918D91882381F09091C00095FFFCCFD8
:10B9B0008093C600F6CF9091C00095FFFCCF809396
:10B9C000C6008D918111F7CF6091DF0A70E04AE0E7
:10B9D00050E08CED99E00E943D418091C00085FFD0
:10B9E000FCCF8AE08093C60081E0DF91CF9108957B
:10B9F0004F925F926F927F928F929F92AF92BF927F
:10BA0000CF92DF92EF92FF92CF93DF9300D01F92FD
:10BA1000CDB7DEB72B013C0129833A834B835C838E
:10BA20008DEE9FE00F94FAC88F3F01F58EEE9FE0F8
:10BA30000F94FAC88F3FD1F48FEE9FE00F94FAC8AD
:10BA40008F3FA1F480EF9FE00F94FAC88F3F71F40D
:10BA500040E050E0BA018DEE9FE00F941EC940E037
:10BA600050E0BA0181EF9FE00F941EC981EF9FE083
:10BA70000F9402C94B015C018DEE9FE00F9402C947
:10BA80006B017C0169817A818B819C812CE330E0A0
:10BA900040E050E00F9453C1C20ED31EE41EF51EC9
:10BAA000B701A6018DEE9FE00F941EC9C301B2013C
:10BAB00028EE33E040E050E00F9453C1BA01A901F1
:10BAC000480D591D6A1D7B1D81EF9FE00F941EC913
:10BAD0001092870B1092880B1092890B10928A0B90
:10BAE0000F900F900F900F90DF91CF91FF90EF90FC
:10BAF000DF90CF90BF90AF909F908F907F906F908E
:10BB00005F904F900895CF92DF92EF92FF92209135
:10BB10004E0B2223F1F020E030E040E05FE30F9491
:10BB200051BF6B017C0120E030E0A9010F947CBC87
:10BB3000882379F0A7019601C701B6010F9451BF80
:10BB40002BED3FE049E450E40F9451BF9B01AC0161
:10BB500004C020E030E040E85FE360E070E080E8AF
:10BB60009FE30F9483BCFF90EF90DF90CF900895F8
:10BB70006091440270914502809146029091470283
:10BB8000C2DF60934002709341028093420290931F
:10BB900043020895CF93DF93EC010F94082A81E0CC
:10BBA000D8DD80E00F94A195209799F0C233D1059C
:10BBB00040F062E370E080E090E00F94D4B3E2974D
:10BBC000ECCFBE0180E090E00F94D4B3C0E0D0E0B1
:10BBD000E4CFDF91CF9108952F923F924F925F92E1
:10BBE0006F927F928F929F92AF92BF92CF92DF928D
:10BBF000EF92FF921F93CF93DF934B015C01CC2414
:10BC0000CA94DC2C76015FEE252E5AE0352E68EEC4
:10BC1000462E63E0562E612C712C1AE08091190B90
:10BC2000811126C12FEFC216D206E206F20651F0AC
:10BC3000F7FC1EC10F94A5B36C197D09683B7B40CE
:10BC400008F016C10F94A5B3681979098A099B09F0
:10BC5000693E73408105910508F47FC08091F41B13
:10BC6000811177C0E7EFFAE08491882341F0909149
:10BC7000C00095FFFCCF8093C6003196F5CFE091D0
:10BC8000DF0A24E0E29FF0011124EF52F54E4081DB
:10BC900051816281738121E030E08CED99E00E9456
:10BCA0003042E3EFFAE08491882341F09091C000A4
:10BCB00095FFFCCF8093C6003196F5CF6091DF0AE7
:10BCC00070E04AE050E08CED99E00E943D41F101C6
:10BCD0008491EFEEFAE0882349F09091C00095FF3F
:10BCE000FCCF8093C60031968491F5CFF7FE03C058
:10BCF000E8E3F9E025C00F94A5B34B015C01C7014F
:10BD0000B6016854744F8F4F9F4F681979098A099B
:10BD10009B09A30192010F9453C1BA01A9012AE022
:10BD200030E08CED99E00E9405418091C00085FFD4
:10BD3000FCCF0DC09091C00095FFFCCF8093C60052
:10BD400081918111F7CF8091C00085FFFCCF1093C6
:10BD5000C6000F94A5B34B015C010F94082A80E044
:10BD6000F8DC80E00F94A195FFEFCF16DF06EF0619
:10BD7000FF0609F046C08091DD0AE091DF0AF0E09D
:10BD8000EF01CC0FDD1FCC0FDD1FCF52D54EEE0FD4
:10BD9000FF1FE752F54E8823D1F080819181BC01CD
:10BDA000882777FD8095982F0F941EBD20E030E006
:10BDB00040E85FE30F94A2BB9B01AC0168817981ED
:10BDC0008A819B810F947FBE87FF4DC027CF8081E2
:10BDD0009181BC01882777FD8095982F0F941EBD17
:10BDE00020E030E040E85FE30F94A3BB9B01AC018F
:10BDF000688179818A819B810F947CBC18169CF59F
:10BE00000DCFF7FC0BCFE091DF0AF0E0EF01CC0F94
:10BE1000DD1FCC0FDD1FCF52D54EEE0FFF1FE752B7
:10BE2000F54E80819181BC01882777FD8095982F00
:10BE30000F941EBD9B01AC01688179818A819B8131
:10BE40000F94A2BB0F94EBBC97FF07C09095809511
:10BE5000709561957F4F8F4F9F4F663071058105BB
:10BE600091050CF4DBCE0F94A5B36B017C01D6CE0B
:10BE7000DF91CF911F91FF90EF90DF90CF90BF9017
:10BE8000AF909F908F907F906F905F904F903F907A
:10BE90002F900895CF93DF931F921F92CDB7DEB7F7
:10BEA000BE016F5F7F4F88EF9FE00F940D4F898138
:10BEB0009A818156904F803A9F4020F11A821982D0
:10BEC000E6ECFAE08491882341F09091C00095FF60
:10BED000FCCF8093C6003196F5CF8091C00085FFDE
:10BEE000FCCF8AE08093C600BE016F5F7F4F88EF72
:10BEF0009FE00F94FC4E89E89AE00F946DA281E0D8
:10BF00000F9468980F900F90DF91CF9108952F9222
:10BF10003F924F925F926F927F928F929F92AF92D9
:10BF2000BF92CF92DF92EF92FF920F931F93CF9326
:10BF3000DF93CDB7DEB7CA58D2400FB6F894DEBF54
:10BF40000FBECDBFC958DD4F688379838A839B8339
:10BF5000C757D240FE01E75FFD4F88E2DF011D9227
:10BF60008A95E9F7E850F24080E991E0DF019C0111
:10BF70001D9221503040E1F7C75ADD4F19821882D7
:10BF8000C955D240CE01875A9D4F5C014E019FE6B4
:10BF9000891A9EEF990ADE01AF51BE4F3D0190EB29
:10BFA000C92E9FE0D92E23E2E22EF12C00E010E012
:10BFB000C359DD4F8882CD56D240CD58DD4F98828F
:10BFC000C357D240B701882777FD8095982F0F94EB
:10BFD0001EBDD3016D937D938D939D933D01F5011E
:10BFE000619171915F01882777FD8095982F0F945B
:10BFF0001EBDD4016D937D938D939D934D010F5F75
:10C000001F4F0630110559F0B501C6010F940D4FB1
:10C01000B5E0EB0EF11CE2E0CE0ED11CD3CFCF5138
:10C02000DE4F288139814A815B81C15ED140C95888
:10C03000DD4F688179818A819B81C757D2400F94F7
:10C040007CBC87FD2BC3FE01EF51FE4F7F016E01CB
:10C05000FFE2CF1AFEEFDF0A3E012BEB621A2DEF53
:10C06000720AC359DD4F0881CD56D240CD58DD4FFD
:10C070001881C357D24085E090E0CF58DD4F9983B7
:10C080008883C157D240CF58DD4FA881B981C157AD
:10C09000D2401197CF58DD4FB983A883C157D24002
:10C0A000F701208931894289538964897589868994
:10C0B00097890F94A2BB4B015C01D80150962D913A
:10C0C0003D914D915C91539754966D917D918D91D9
:10C0D0009C9157970F94A2BBA50194010F9483BC28
:10C0E000F60192938293729362936F01D301BE9291
:10C0F000AE929E928E923D0104501109B4E0EB1A6B
:10C10000F108CF58DD4FE881F981C157D240EF2BBC
:10C1100009F0B9CF6E01FFECCF1AFDEFDF0A3E0147
:10C1200027E4621A2EEF720A2E013DE3430E511CE2
:10C13000CE0101967C0101E010E0D6018D909D902A
:10C14000AD90BC90139714962D913D914D915C91BB
:10C150001797C501B4010F94A3BB9B01AC010F94C9
:10C16000A3BBF70164A775A786A797A701301105A0
:10C1700041F080A691A6A2A6B3A684829582A6824B
:10C18000B7820F5F1F4FD30114962D913D914D91B2
:10C190005C91179718966D917D918D919C911B974D
:10C1A0000F94A2BB20E030E040EC50E40F9451BF6C
:10C1B000F2016083718382839383F4E0CF0ED11CFC
:10C1C0002CE2E20EF11C34E0630E711C88E2480E92
:10C1D000511C0530110509F0B0CF8E010B5A1F4FCD
:10C1E0006E0191E5C90ED11C22242394312C2C0E12
:10C1F0003D1EA8ED2A0E311CF801B897208131812F
:10C2000042815381F80160817181828193810F9411
:10C2100083BC4B015C01E12CF12C3601F8E26F1A72
:10C22000710826014E0C5F1CF301EE0DFF1D2481E9
:10C23000358146815781C501B4010F9451BF9B01DF
:10C24000AC01D20114966D917D918D919C911797BF
:10C250000F94A2BBF2016483758386839783F4E015
:10C26000EF0EF11C24E1E216F104D9F6045D1F4F34
:10C2700038E2C30ED11C0215130509F0BDCF1E0113
:10C2800085EB280E311C6E0191EBC90ED11C3E01CD
:10C29000A7EE6A1AADEF7A0A14E0E12EF12C27011D
:10C2A00000E010E0812C912CA12CB12CF601E00FC4
:10C2B000F11FD301A00FB11F2D913D914D915C91C4
:10C2C00060817181828193810F9451BF9B01AC0188
:10C2D000B401C5010F94A3BB4B015C01BFEF4B1A26
:10C2E0005B0A0C5F1F4FE5E04E165104F9F69B0107
:10C2F000AC01D1016D917D918D919C910F94A2BB68
:10C30000F60120813181428153810F9483BCD30196
:10C310006D937D938D939C931397B1E0EB1AF10885
:10C32000E8E22E1A3108FCE2CF1AD10824E0621AA2
:10C330007108E114F10409F0B2CFCB50DE4F8881CF
:10C340009981AA81BB81C55FD140C957DD4F8883E0
:10C350009983AA83BB83C758D2408E01075F1D4FC4
:10C36000DE01AF5CBD4FC558DD4FB983A883CB5705
:10C37000D240C359DD4F2880CD56D240CD58DD4F35
:10C380003880C357D240FE01EF51FE4FC358DD4FF6
:10C39000F983E883CD57D240C358DD4FA881B981D6
:10C3A000CD57D240CD90DD90ED90FD90C358DD4F3C
:10C3B000B983A883CD57D240C958DD4F2881398130
:10C3C0004A815B81C757D240C701B6010F947CBC3C
:10C3D0001816B4F0C358DD4FE881F981CD57D2402B
:10C3E0002081318142815381C958DD4F6881798133
:10C3F0008A819B81C757D2400F947CBC1816FCF4ED
:10C40000CF58DD4F28813981C157D24024303105C2
:10C4100009F01FC1C957DD4F288139814A815B81ED
:10C42000C758D240C958DD4F688179818A819B8184
:10C43000C757D2400F947FBE18160CF00AC1D8011E
:10C4400014968D919D910D90BC91A02DC158DD4FFA
:10C4500088839983AA83BB83CF57D240F801408059
:10C46000518062807380C558DD4FA881B981CB5758
:10C47000D2408D919D910D90BC91A02DC359DD4F5F
:10C4800088839983AA83BB83CD56D240D1018D91F5
:10C490009D910D90BC91A02DCD57DD4F8883998340
:10C4A000AA83BB83C358D240A7019601C958DD4F68
:10C4B000688179818A819B81C757D2400F94A2BB42
:10C4C000CD58DD4F688379838A839B83C357D240DD
:10C4D00020E030E040E450E40F94B4BF6B017C01F5
:10C4E000A3019201C158DD4F688179818A819B81C6
:10C4F000CF57D2400F94A2BB4B015C0120E030E04B
:10C5000040EC50E4C359DD4F688179818A819B8179
:10C51000CD56D2400F9451BF9B01AC01C501B4016F
:10C520000F9483BCA70196010F9451BF6B017C014E
:10C5300020E030E040E05FE3C301B2010F9451BF5F
:10C540004B015C01CD58DD4F288139814A815B81E7
:10C55000C357D240CA01B9010F9451BF9B01AC012E
:10C56000C501B4010F9451BF9B01AC01C701B601D5
:10C570000F94A3BB6B017C01CD57DD4F288139811E
:10C580004A815B81C358D240F10164817581868103
:10C5900097810F94A2BBC359DD4F288139814A810D
:10C5A0005B81CD56D2400F9483BC4B015C01C359D3
:10C5B000DD4F288139814A815B81CD56D240CA0145
:10C5C000B9010F94A3BBA30192010F9451BF2B019A
:10C5D0003C01C359DD4F288139814A815B81CD56A9
:10C5E000D240C158DD4F688179818A819B81CF57C4
:10C5F000D2400F9451BF9B01AC01C301B2010F9413
:10C60000A3BB20E030E040EC50E40F9483BC9B01DE
:10C61000AC01C501B4010F94A2BBCD58DD4F2881F8
:10C6200039814A815B81C357D2400F9451BF9B012E
:10C63000AC01C701B6010F94A3BBCD57DD4F2881D4
:10C6400039814A815B81C358D2400F94A3BB4B010F
:10C650005C01CF58DD4F28813981C157D2402F5F0F
:10C660003F4FCF58DD4F39832883C157D2400C5FED
:10C670001F4FC558DD4F88819981CB57D240049612
:10C68000C558DD4F99838883CB57D24094E0290E5B
:10C69000311C2530310509F07FCE04C0812C912C4E
:10C6A000A12CB12CB401C501C657DD4F0FB6F894CB
:10C6B000DEBF0FBECDBFDF91CF911F910F91FF90D5
:10C6C000EF90DF90CF90BF90AF909F908F907F9032
:10C6D0006F905F904F903F902F900895CF92DF9290
:10C6E000EF92FF926B017C018091BF0B8823A1F038
:10C6F00086EA9FE00F94FAC8882371F0C701B6015B
:10C7000006DC2091AA193091AB194091AC195091D7
:10C71000AD190F9483BC03C060E070E0CB01FF90C3
:10C72000EF90DF90CF9008954F925F926F927F923B
:10C730008F929F92AF92BF92CF92DF92EF92FF9231
:10C740000F931F93CF93DF93CDB7DEB728970FB624
:10C75000F894DEBF0FBECDBF0F941C1D8091560212
:10C76000909157029093C30B8093C20BE0912A0BD8
:10C77000F0E0EE0FFF1FE752F54E608171818827D0
:10C7800077FD8095982F0F941EBD6093B30B709327
:10C79000B40B8093B50B9093B60B8091280B9091BE
:10C7A000290B9093B20B8093B10B0F94A5B36093B8
:10C7B000990B70939A0B80939B0B90939C0B809199
:10C7C0003E0B90913F0BA091400BB091410B8983A0
:10C7D0009A83AB83BC838093A10B9093A20BA0930D
:10C7E000A30BB093A40B4090420B5090430B60906E
:10C7F000440B7090450B4092A50B5092A60B609293
:10C80000A70B7092A80B8091460B9091470BA091BB
:10C81000480BB091490B8D839E83AF83B88780937B
:10C82000A90B9093AA0BA093AB0BB093AC0B6091A8
:10C830004A0B70914B0B80914C0B90914D0B609378
:10C84000AD0B7093AE0B8093AF0B9093B00B20E0C9
:10C8500030E040E85FE30F94A2BB60934A0B709313
:10C860004B0B80934C0B90934D0B8AE29BE09F9374
:10C870008F93812C912CB8ECAB2EB3E4BB2E1AE431
:10C88000C12E1BE0D12EED80FE800F811885A30103
:10C89000920169817A818B819C810F946D0320E0E4
:10C8A00030E040EA51E46091460B7091470B809173
:10C8B000480B9091490B0F94A3BB2B013C010F90A7
:10C8C0000F9020E030E042E553E40F947FBE18164D
:10C8D0004CF04092460B5092470B6092480B70927E
:10C8E000490B0CC080E090E0A2E5B3E48093460BD6
:10C8F0009093470BA093480BB093490BE090460BE5
:10C90000F090470B0091480B1091490B2091420B7E
:10C910003091430B4091440B5091450B60913E0B7D
:10C9200070913F0B8091400B9091410BAAE26A2ECF
:10C93000ABE07A2E7F926F92812C912CB0E7AB2ED8
:10C94000B1E4BB2EEAE4CE2EEBE0DE2E0F946D03B5
:10C950001092DA1A1092D91A1092DC1A1092DB1A7D
:10C960001092DE1A1092DD1A80E090E0A8E4B2E4A2
:10C9700080933E0B90933F0BA093400BB093410BE1
:10C9800080E090E0AEE3B3E48093420B9093430BDE
:10C99000A093440BB093450BE090460BF090470BEF
:10C9A0000091480B1091490B7F926F92812C912C32
:10C9B000F8E4AF2EF2E4BF2E9C01AD01C501B40135
:10C9C0000F946D031092290B1092280B0F900F906B
:10C9D0000F900F9028960FB6F894DEBF0FBECDBF14
:10C9E000DF91CF911F910F91FF90EF90DF90CF904B
:10C9F000BF90AF909F908F907F906F905F904F907F
:10CA00000D941C1DE0912A0B84E0E89FF001112495
:10CA1000EF52F54E4081518162817381E6E8FAE080
:10CA20008491882341F09091C00095FFFCCF8093C2
:10CA3000C6003196F5CF22E030E08CED99E00E94FF
:10CA40003042E2E8FAE08491882341F09091C000FE
:10CA500095FFFCCF8093C6003196F5CF60912A0BED
:10CA600070E04AE050E08CED99E00E943D41EEE735
:10CA7000FAE08491882341F09091C00095FFFCCFAB
:10CA80008093C6003196F5CF4091BF1A5091C01ADD
:10CA90006091C11A7091C21A21E030E08CED99E0EA
:10CAA0000E9430428091C00085FFFCCF8AE08093D5
:10CAB000C6000895CF93DF93CDB7DEB72A970FB6A0
:10CAC000F894DEBF0FBECDBF0F94A5B36F837887F8
:10CAD00089879A87179A10922F0B169A1092300B0B
:10CAE0006CE082E00F94F8396CE082E00F94393A00
:10CAF00064E183E00F94F83964E183E00F94393AFC
:10CB0000E9E7FAE08491882341F09091C00095FF15
:10CB1000FCCF8093C6003196F5CF8091C00085FF91
:10CB2000FCCF8AE08093C60083E40F94153D1C017E
:10CB30004090831050908410609085107090861003
:10CB40000F946012481A590A610871080E9422C89D
:10CB5000481A590A6108710877FE03C0412C512C0C
:10CB600032019091C6138091C513981799F0E09106
:10CB7000C51327E5E29FF0011124E953FC4E20E0A4
:10CB800030E040E752E462A173A184A195A10F9423
:10CB900051BF08C060910C0270910D0280910E028D
:10CBA00090910F020F94EBBC7E836D830F94F20182
:10CBB0000E94C8C01092CE0B789420E030E040E88C
:10CBC0005FE360914A0B70914B0B80914C0B9091FD
:10CBD0004D0B0F94A2BB69837A838B839C83E09077
:10CBE000460BF090470B0091480B1091490B209198
:10CBF000420B3091430B4091440B5091450B609197
:10CC00003E0B70913F0B8091400B9091410BAAE23B
:10CC1000BBE0BF93AF93812C912CE8ECAE2EE3E404
:10CC2000BE2EDE0111966D010F946D0320E030E001
:10CC300040E85FE360914A0B70914B0B80914C0B85
:10CC400090914D0B0F94A2BB69837A838B839C8355
:10CC50002AE037ED43E25FE36091460B7091470BAA
:10CC60008091480B9091490B0F94A3BB6B017C0101
:10CC700067E074E062197309F4E076956795FA95B8
:10CC8000E1F780E090E00F941CBD2091AA1930914B
:10CC9000AB194091AC195091AD190F9483BC9B0115
:10CCA000AC01C701B6010F94A3BB7B018C0120919D
:10CCB000420B3091430B4091440B5091450B6091D6
:10CCC0003E0B70913F0B8091400B9091410BAAE27B
:10CCD000BBE0BF93AF93812C912CA0E2AA2EA2E4DB
:10CCE000BA2EDE0111966D010F946D03B301A201FE
:10CCF00081E99FE00F941EC90F900F900F900F9045
:10CD000005E71FE0F12CB3E0EB2E8091D9128823C8
:10CD100041F18F2D6E2D0F941FC1B5E18B02F001F3
:10CD2000112423E09202E00DF11D1124EE0FFF1FEC
:10CD3000EE0FFF1FE752FD4E20E030E04AE754E4DB
:10CD400061817281838194810F9451BF20E030E032
:10CD500040E05FE30F94A3BB0F9459BD0F94EBBC6D
:10CD600002C060E070E0C8010F9426C9F3940E5F22
:10CD70001F4F89E0F812C9CFB10183E79FE00F94FC
:10CD800026C940913E0B50913F0B6091400B709132
:10CD9000410B8DE99FE00F941EC94091420B5091C9
:10CDA000430B6091440B7091450B81EA9FE00F9417
:10CDB0001EC94091460B5091470B6091480B7091F2
:10CDC000490B8DE89FE00F941EC9BE016B5F7F4F3A
:10CDD00089E89FE00F94FC4EE0912A0BF0E0EE0F03
:10CDE000FF1FE752F54E60818CE89FE00F940CC95D
:10CDF0006091D71A8BE89FE00F940CC96091280BC3
:10CE000088E89FE00F940CC961E085EA9FE00F94E9
:10CE10000CC90F941C1DE4E7FAE08491882341F0CB
:10CE20009091C00095FFFCCF8093C6003196F5CF5E
:10CE300083E40F94153D4AE050E0BC018CED99E08D
:10CE40000E948F4184E69FE00F94FAC861E0680F6A
:10CE500084E69FE00F940CC9E9E6FAE08491882308
:10CE600041F09091C00095FFFCCF8093C6003196B1
:10CE7000F5CF8091C00085FFFCCF8AE08093C6008B
:10CE80000F94A5B3AB01BC018F819885A985BA85A4
:10CE9000481B590B6A0B7B0B2AE030E08CED99E0C4
:10CEA0000E949B41F894FFCF6F987798EAE6F0E0F4
:10CEB00080818F7B8083808180688083EF9A089552
:10CEC0001F920F920FB60F9211240BB60F920F9371
:10CED0001F932F933F934F935F936F937F938F9302
:10CEE0009F93AF93BF93EF93FF938091280B909103
:10CEF000290B8B3491050CF441C080916A0086FFA8
:10CF00000BC00F94A5B36093950B7093960B809311
:10CF1000970B9093980B2CC00F94A5B30091950B91
:10CF20001091960B2091970B3091980B601B710B11
:10CF3000820B930B2091280B3091290B253631055C
:10CF40002CF003E010E020E030E004C004E010E04A
:10CF500020E030E0601771078207930748F0809166
:10CF6000700B9091710B02969093710B8093700BE4
:10CF700080916A0090E4892780936A00FF91EF9185
:10CF8000BF91AF919F918F917F916F915F914F91E1
:10CF90003F912F911F910F910F900BBE0F900FBEDD
:10CFA0000F901F9018956C987498EAE6F0E08081D5
:10CFB0008160808380818D7F8083EC9A08951F92A9
:10CFC0000F920FB60F9211240BB60F922F933F932F
:10CFD0004F935F936F937F938F939F93AF93BF9381
:10CFE000EF93FF93EC98E4E6FAE08491882341F014
:10CFF0009091C00095FFFCCF8093C6003196F5CF8D
:10D000008091C00085FFFCCF8AE08093C6008091AC
:10D01000CE0B81114FDDFF91EF91BF91AF919F91A9
:10D020008F917F916F915F914F913F912F910F90D1
:10D030000BBE0F900FBE0F901F9018954F925F92EE
:10D040006F927F928F929F92BF92CF92DF92EF92D8
:10D05000FF920F931F93CF93DF93CDB7DEB7EA977D
:10D060000FB6F894DEBF0FBECDBF88E89FE00F94E7
:10D07000FAC8B82EBE01675C7F4F89E89FE00F9425
:10D080000D4FEDE0F9E08491882341F09091C000CC
:10D0900095FFFCCF8093C6003196F5CF69AD7AAD90
:10D0A0004AE050E08CED99E00E94444183E69FE025
:10D0B0000F94FAC8882E912C4AE050E0B4018CED10
:10D0C00099E00E94444103E11FE0E12CF12C3E0174
:10D0D00084E3680E711CE814F9042CF5FE01BC967B
:10D0E0002F016801C6010F94FAC8F20181932F0144
:10D0F000FFEFCF1ADF0A46145704A1F71CAABE019E
:10D10000645D7F4F8CED99E00E943041BE01645D0B
:10D110007F4F8CEC9BE00E94A6BE8FEFE81AF80AC6
:10D12000085F1F4FD8CF8E01015E1F4F85E9E82EA3
:10D130008FE0F82ED02EC12EC7010F94FAC8F80147
:10D1400081938F01FFEFEF1AFF0A8DE9E8168FE058
:10D15000F80691F71FA2ED2DFC2D8191882339F05F
:10D160009091C00095FFFCCF8093C600F6CF68E099
:10D1700079E08D2D9C2D0F949EC4CF92DF9281E09B
:10D1800099E09F938F938E010F5F1F4F1F930F9313
:10D190000F94CEC60F900F900F900F900F900F909E
:10D1A0007E0195E0E90EF11CF7018081882349F0AA
:10D1B000992787FD90950F948DC4F70181937F0186
:10D1C000F3CF60E0C8010E943EC181E99FE00F9467
:10D1D00002C9F62EE72ED82EC92EE6EEF8E084918D
:10D1E000882341F09091C00095FFFCCF8093C6004A
:10D1F0003196F5CF2AE030E04F2D5E2D6D2D7C2D40
:10D200008CED99E00E949B4161E082EE98E00E94E3
:10D210003EC16DED78E0C8010F94A9C48DE99FE08F
:10D220000F9402C96DAB7EAB8FAB98AFCE01C596A4
:10D230000F945E53BC01C8010F9438C56AED78E0C5
:10D24000C8010F949EC481EA9FE00F9402C96DABA0
:10D250007EAB8FAB98AFCE01C5960F945E53BC01E9
:10D26000C8010F9438C563ED78E0C8010F949EC4DF
:10D2700060E0C8010E943EC16EEC78E0C8010F94E6
:10D28000A9C48DE89FE00F9402C96DAB7EAB8FAB54
:10D2900098AFCE01C5960F945E53BC01C8010F94A0
:10D2A00038C560E0C8010E943EC161E083EC98E0AF
:10D2B0000E943EC18AAD8F9389AD8F938CEB98E02D
:10D2C0009F938F931F930F930F94CEC660E0C80176
:10D2D0000E943EC165EB78E0C8010F94A9C48B2D74
:10D2E00090E09EAB8DABCE01C5960F943356BC013A
:10D2F000C8010F9438C560E0C8010E943EC1CF92BA
:10D30000DF92EF92FF928CEA98E09F938F931F93A6
:10D310000F930F94CEC660E0C8010E943EC161E049
:10D3200088EA98E00E943EC10FB6F894DEBF0FBEB7
:10D33000CDBFEA960FB6F894DEBF0FBECDBFDF912A
:10D34000CF911F910F91FF90EF90DF90CF90BF9002
:10D350009F908F907F906F905F904F9008954F9225
:10D360005F926F927F92AF92BF92CF92DF92EF92D5
:10D37000FF920F931F93CF93DF93CDB7DEB7E09764
:10D380000FB6F894DEBF0FBECDBF2B013C01690183
:10D390007A0180917D0A8111E5C0F8940F944012C2
:10D3A0008091831090918410A0918510B091861087
:10D3B0008093790A90937A0AA0937B0AB0937C0AAF
:10D3C0000F9460124091790A50917A0A60917B0A19
:10D3D00070917C0A481B590B610971094093790AC5
:10D3E00050937A0A60937B0A70937C0A0E9422C849
:10D3F0004091790A50917A0A60917B0A70917C0A77
:10D40000481B590B610971094093790A50937A0AB4
:10D4100060937B0A70937C0A9091C6138091C51328
:10D42000981799F0E091C51387E5E89FF001112462
:10D43000E953FC4E20E030E040E752E462A173A1E2
:10D4400084A195A10F9451BF08C060910C02709106
:10D450000D0280910E0290910F026093650A709305
:10D46000660A8093670A9093680A0F94F20180E13C
:10D47000EEE3FBE0A9E6BAE001900D928A95E1F7B0
:10D4800080912A0B8093640A809107028093630A3B
:10D490000E94C8C01092CE0B81E080937D0A7894E0
:10D4A00020E030E0A901C301B2010F947CBC8111DE
:10D4B0000AC020E030E0A901C701B6010F947CBC8E
:10D4C000882309F44FC063EA78E0FE0131965F01DA
:10D4D000CF010F94A9C4F50101900020E9F78F0155
:10D4E000015011092091710A3091720A4091730A1A
:10D4F0005091740AC301B2010F94A3BB23E048E02A
:10D500000F94CCC160EA78E0C5010F949EC4F50188
:10D5100001900020E9F78F010150110923E046E056
:10D52000C701B6010F94CCC16DE978E0C5010F9435
:10D530009EC4F50101900020E9F78F010150110907
:10D540006091600270916102809162029091630229
:10D5500023E048E00F94CCC160E0C5010E943EC1C9
:10D560000E94DDC2E0960FB6F894DEBF0FBECDBFBD
:10D57000DF91CF911F910F91FF90EF90DF90CF90AF
:10D58000BF90AF907F906F905F904F90089520E094
:10D5900030E0A90160E070E080E291E4E0CE8F929B
:10D5A0009F92AF92BF92CF92DF92EF92FF920F9332
:10D5B0001F93CF93DF9300D01F92CDB7DEB79B01AF
:10D5C000AC0180917D0A882309F497C08091640A98
:10D5D00080932A0B8091650A9091660AA091670A50
:10D5E000B091680A80930C0290930D02A0930E02F2
:10D5F000B0930F026091750A7091760A8091770A54
:10D600009091780A0F94A2BB69837A838B839C8361
:10D61000CE0101960F94C61120E030E040E551E4C0
:10D620006091600270916102809162029091630248
:10D630000F9483BC4B015C01E090710AF090720A78
:10D640000091730A1091740A20916D0A30916E0A4C
:10D6500040916F0A5091700A6091690A70916A0A4C
:10D6600080916B0A90916C0AEAE2FBE0FF93EF93E2
:10D67000E5E7CE2EEAE0DE2E0F946D030F941C1D1D
:10D6800080E1E9E6FAE0AEE3BBE001900D928A9515
:10D69000E1F780E1EEE3FBE0A9E0BBE001900D9251
:10D6A0008A95E1F74091790A50917A0A60917B0A54
:10D6B00070917C0A40936A0E50936B0E60936C0ECF
:10D6C00070936D0E85EB9DE00E94ACA88091790A65
:10D6D00090917A0AA0917B0AB0917C0A8093831082
:10D6E00090938410A0938510B093861081E080936E
:10D6F000CE0B10927D0A0F900F900F900F900F900D
:10D700000F90DF91CF911F910F91FF90EF90DF90DD
:10D71000CF90BF90AF909F908F90089560E070E0A1
:10D72000CB013DCFFBDF81E08093B1020895E8E8B3
:10D73000F8E08491882341F09091C00095FFFCCFE0
:10D740008093C6003196F5CF40913E0B50913F0B30
:10D750006091400B7091410B23E030E08CED99E03B
:10D760000E943042E5E8F8E08491882341F09091EE
:10D77000C00095FFFCCF8093C6003196F5CF409155
:10D78000420B5091430B6091440B7091450B23E089
:10D7900030E08CED99E00E943042E2E8F8E08491BC
:10D7A000882341F09091C00095FFFCCF8093C60084
:10D7B0003196F5CF4091460B5091470B6091480B45
:10D7C0007091490B23E030E08CED99E00E943042EB
:10D7D000E0E8F8E08491882341F09091C00095FF43
:10D7E000FCCF8093C6003196F5CF8091C00085FFB5
:10D7F000FCCF8AE08093C6000895E8E6F8E08491C3
:10D80000882341F09091C00095FFFCCF8093C60023
:10D810003196F5CF0F948B1DAB01BC0123E030E0B6
:10D820008CED99E00E943042E5E6F8E0849188238F
:10D8300041F09091C00095FFFCCF8093C6003196D7
:10D84000F5CF81E00F948B1DAB01BC0123E030E0EC
:10D850008CED99E00E943042E2E6F8E08491882362
:10D8600041F09091C00095FFFCCF8093C6003196A7
:10D87000F5CF82E00F948B1DAB01BC0123E030E0BB
:10D880008CED99E00E943042E0E6F8E08491882334
:10D8900041F09091C00095FFFCCF8093C600319677
:10D8A000F5CF8091C00085FFFCCF8AE08093C60051
:10D8B0000895EF92FF920F931F93CF93DF93ECE4C1
:10D8C000F8E08491882341F09091C00095FFFCCF4F
:10D8D0008093C6003196F5CF09ED12E1FAE4EF2E00
:10D8E000F8E0FF2EC0E0D0E0F801EC0FFD1F418111
:10D8F00052816381748123E030E08CED99E00E94D5
:10D900003042F7018491EAE4F8E0882349F09091ED
:10D91000C00095FFFCCF8093C60031968491F5CF6F
:10D920002496CC31D10501F7045E1F4FF3E10D3988
:10D930001F07C1F6E9E4F8E08491882341F0909153
:10D94000C00095FFFCCF8093C6003196F5CF809143
:10D95000C00085FFFCCF8AE08093C600DF91CF91A5
:10D960001F910F91FF90EF9008952F923F924F9249
:10D970005F926F927F928F929F92AF92BF92CF925F
:10D98000DF92EF92FF920F931F93CF93DF93CDB768
:10D99000DEB7C355D1090FB6F894DEBF0FBECDBFB9
:10D9A00082E090E0909316028093150286EE93E059
:10D9B0000E9418438823B1F080919B1090919C1095
:10D9C0006AE270E005960F9443C5009711F0DC0100
:10D9D0001C9280919B1090919C1005960F94D94FAA
:10D9E0000C94979887ED93E00E941843882321F0C8
:10D9F0000E9486470C9497988BEE93E00E94184300
:10DA0000882319F08FDE0C94979889EF93E00E9499
:10DA10001843882321F00E94C2470C94979886E00F
:10DA200094E00E941843882309F4C4C18CE094E078
:10DA30000E941843882391F08091F41B882311F4ED
:10DA40000C9497980F94A5B36093C80B7093C90B6F
:10DA50008093CA0B9093CB0B0C94979881E194E040
:10DA60000E941843882361F060918B0B70918C0B9E
:10DA70004AE050E08CED99E00E948F410C94979819
:10DA800085E194E00E941843882309F446C0E9E147
:10DA9000F4E08191882339F09091C00095FFFCCF8C
:10DAA0008093C600F6CF80916A0B90916B0B2CE3AC
:10DAB000289FB001299F700D11244AE050E08CEDA1
:10DAC00099E00E943D416DE174E08CED99E00E9487
:10DAD0003041E2E2F4E08191882339F09091C00076
:10DAE00095FFFCCF8093C600F6CF80916C0B909190
:10DAF0006D0B2CE3289FB001299F700D11244AE083
:10DB000050E08CED99E00E943D416DE174E08CEDB8
:10DB100099E00E9430410C94979888E294E00E942A
:10DB200018438823C1F08091F41B882361F0609131
:10DB3000F21B7091F31B4AE050E08CED99E00E94DB
:10DB400044410C9497986BE274E08CED99E00E944C
:10DB500030410C9497988DE394E00E9418438823F9
:10DB600079F160919B1070919C106D5F7F4F21E067
:10DB700041E08CEC9BE00E9400BB8091BD0D909138
:10DB8000BE0DA091BF0DB091C00D80936A0E909311
:10DB90006B0EA0936C0EB0936D0E85EB9DE00E9412
:10DBA000E3A72091C00025FFFCCF8093C6000A9711
:10DBB00021F760E08CEC9BE00E9490BA0C9497985F
:10DBC00080E494E00E941843882399F00E94AD50AD
:10DBD00081E080938D0B60919B1070919C106C5F25
:10DBE0007F4F21E040E08CEC9BE00E9400BB0C9456
:10DBF000979884E494E00E941843882309F445C070
:10DC00008091F41B882309F49ECF1092610AE7E407
:10DC1000F4E08191882339F09091C00095FFFCCF0A
:10DC20008093C600F6CF00E010E0FF24F3948091CB
:10DC30005D0A90915E0A20915F0A3091600A821B12
:10DC4000930B8F779927892B89F08CED99E00E94AF
:10DC50004A40F092610A9091C00095FFFCCF8093FA
:10DC6000C6000F5F1F4F1092610AE1CF033111050B
:10DC7000F4F281E08093610A8091C00085FFFCCFBF
:10DC80008AE08093C6000C9497988AE494E00E94FE
:10DC900018438823A9F0EEE4F4E08191882339F059
:10DCA0009091C00095FFFCCF8093C600F6CF809185
:10DCB000C00085FFFCCF8AE08093C6000C94979843
:10DCC00088E594E00E9418438823A9F0ECE5F4E08D
:10DCD0008191882339F09091C00095FFFCCF80930B
:10DCE000C600F6CF8091C00085FFFCCF8AE080930C
:10DCF000C6000C9497988AE794E00E941843882302
:10DD000021F00F94774F0C9497988FE794E00E943E
:10DD10001843882341F060E070E088EF9FE00F94A3
:10DD2000FC4E0C94979882E894E00E941843882354
:10DD300059F062E874E08CED99E00E94304140E0D7
:10DD400052EC61E070E010C08DE894E00E9418434E
:10DD5000882381F06DE874E08CED99E00E943041F9
:10DD600040E054E961E170E08CED99E00E94CF3F22
:10DD70000C94019A89E994E00E941843882361F089
:10DD80000F94A5B36093BB0B7093BC0B8093BD0B3A
:10DD90009093BE0B0C9497988EE994E00E941843E0
:10DDA000882311F40C94979861E080E00E94CD479D
:10DDB0000C9497988EE50E94EA4281110C949798F2
:10DDC00087E40E94EA42882311F40C94967E0E9414
:10DDD00057430F94EBBC6C34710509F430C47CF5E7
:10DDE0006430710509F409C154F46230710509F415
:10DDF000ECC00CF0F6C077FF78C00C9497986C31AB
:10DE0000710509F451C17CF46A30710509F446C109
:10DE10006B30710511F00C94979860E080E00E94DF
:10DE2000A6580C9497986E31710509F44DC36B3464
:10DE3000710511F00C94979808E210E0F6C367356D
:10DE4000710511F40C94167E14F56035710511F40A
:10DE50000C94EF776CF46F34710511F00C94979873
:10DE60000FEF10E0A4E0CA2EADE0DA2E0C94DA77C2
:10DE70006135710511F40C945D7D6635710511F005
:10DE80000C94979886EE0E943D470C9497986C35B9
:10DE9000710511F40C941F7E7CF46A35710511F440
:10DEA0000C941B7E6B35710511F00C94979881E0F2
:10DEB0008093F40A0C9497986236710511F40C94CF
:10DEC000817E6336710511F00C9497981092F41BC3
:10DED0000F947C4F6091F41B84EC9FE00F940CC96D
:10DEE00082E00F94A1950C9497988091DE0A81119D
:10DEF0000C9497980E94DB546091870B7091880B6B
:10DF00008091890B90918A0B0F941CBD6B017C0151
:10DF100040904A0B50904B0B60904C0B70904D0B07
:10DF20008090150B9090160BA090170BB090180BCB
:10DF3000A5019401C301B2010F94A2BB20E030E01F
:10DF400048EC52E40F9451BF9B01AC01C701B601EC
:10DF50000F947FBE1816E4F4A3019201C501B40129
:10DF60000F94A2BB20E030E048EC52E40F9451BF84
:10DF70009B01AC01C701B6010F94A3BB0F94F0BC89
:10DF80006093870B7093880B8093890B90938A0B17
:10DF90008091270B8823A9F088E50E94EA4281112D
:10DFA00010C089E50E94EA4281110BC08AE50E94F7
:10DFB000EA42811106C085E40E94EA4281110C9474
:10DFC000A0980E94A3570C9497988091DE0A811123
:10DFD0000C9497980E945E5581E00E94815A0C949F
:10DFE00097988091DE0A81110C9497980E945E5553
:10DFF00080E00E94815A0C94979880E50E94EA4242
:10E00000882339F00E9457430F94F0BC6B017C01C8
:10E0100003C0C12CD12C760183E50E94EA428823FB
:10E0200061F00E94574320E030E04AE754E40F9447
:10E0300051BF0F94F0BC6B017C01C114D104E10409
:10E04000F10431F0E1EBF0E4859194910F94E64F07
:10E050000F941C1D0F94A5B34B015C018C0C9D1CEF
:10E06000AE1CBF1C0F94A5B36093F00A7093F10A25
:10E070008093F20A9093F30A0F94A5B3681579057B
:10E080008A059B0510F00C9497980F94082A80E05D
:10E090000E94A95B80E00F94A195EECF60E081E043
:10E0A0000E94A6580C9497980F941C1DE2E3FEE082
:10E0B0008491882341F09091C00095FFFCCF80931C
:10E0C000C6003196F5CF33DBE4E2FEE0849188238D
:10E0D00041F09091C00095FFFCCF8093C60031962F
:10E0E000F5CF8BDB81E08093C00B88E50E94EA428C
:10E0F000182F89E50E94EA42082F8AE50E94EA4229
:10E10000782E101308C0181711F0012F04C07724BF
:10E11000739401E011E00E946FD96090D9121092BF
:10E12000D91282E00F948B1D6093460B7093470BBE
:10E130008093480B9093490B71100E943EF74091D9
:10E140000C0250910D0260910E0270910F024093EB
:10E15000F50A5093F60A6093F70A7093F80A8091D3
:10E160005602909157029093C30B8093C20B84E6A2
:10E1700090E090935702809356020F94A5B360935A
:10E18000F00A7093F10A8093F20A9093F30A81E007
:10E190000F94A11380E1EEE3FBE0A9E0BBE0019066
:10E1A0000D928A95E1F710920C0210920D021092D6
:10E1B0000E0210920F02112321F080E090E00E94E5
:10E1C0004D4C002321F081E090E00E944D4C88E509
:10E1D0000E94EA42882341F00E940D43672B682B7E
:10E1E000692B11F00C94CF9889E50E94EA428823AC
:10E1F00041F00E940D43672B682B692B11F00C94A2
:10E20000E598772009F4F1C080912F0B882321F045
:10E210008091300B811108C080E090E00E944D4C4D
:10E2200081E090E00E944D4C0E94C4D9E5EAF3E4FD
:10E2300085919591A591B49189839A83AB83BC8391
:10E24000E1EAF3E485919591A591B4918F8F98A31C
:10E25000A9A3BAA32DE03BE049E05BE0BE016F5FFC
:10E260007F4FCE014F960E945E450E9436D920E036
:10E2700030E040E850EC60910D0B70910E0B8091F6
:10E280000F0B9091100B0F947CBC87FF0CC080E0AB
:10E2900090E0A0E8B0EC80930D0B90930E0BA09350
:10E2A0000F0BB093100B80E090E0A0EAB0E48093F5
:10E2B000110B9093120BA093130BB093140B20E04F
:10E2C00030E040E251E4609160027091610280911F
:10E2D0006202909163020F9483BC60930C0270936E
:10E2E0000D0280930E0290930F021092460B109233
:10E2F000470B1092480B1092490B80E00F94A1132A
:10E30000E090460BF090470B0091480B1091490BA1
:10E310002091420B3091430B4091440B5091450B9F
:10E3200060913E0B70913F0B8091400B9091410B9F
:10E33000FAE4CF2EFBE0DF2E0F941B1080900C022E
:10E3400090900D02A0900E02B0900F02E090110B81
:10E35000F090120B0091130B1091140B20910D0BE8
:10E3600030910E0B40910F0B5091100B6091090BE7
:10E3700070910A0B80910B0B90910C0BEAE2FBE081
:10E38000FF93EF93A5E1CA2EABE0DA2E0F946D0355
:10E390000F941C1D8091090B90910A0BA0910B0BFF
:10E3A000B0910C0B80933E0B90933F0BA093400BCE
:10E3B000B093410B80910D0B90910E0BA0910F0B20
:10E3C000B091100B8093420B9093430BA093440B9E
:10E3D000B093450B81E00F94A1130F94891382E051
:10E3E00090E00E944D4C0F900F908AE50E94EA4207
:10E3F000882341F00E940D43672B682B692B11F095
:10E400000C94FB98E090460BF090470B0091480B62
:10E410001091490B2091420B3091430B4091440BDA
:10E420005091450B60913E0B70913F0B8091400BDA
:10E430009091410BEAE4CE2EEBE0DE2E0F941B1000
:10E4400080E00F94A1138091F50A9091F60AA091B3
:10E45000F70AB091F80A80930C0290930D02A093F2
:10E460000E02B0930F028091C20B9091C30B909358
:10E470005702809356020F94A5B36093F00A7093ED
:10E48000F10A8093F20A9093F30A0F9489130E9481
:10E49000C4D90E94E0DB88E50E94EA4281110C9415
:10E4A000119989E50E94EA4281110C94119987E53E
:10E4B0000E94EA4281110C9411998AE50E94EA4275
:10E4C00081110C94119987C50F941C1D81E00E9445
:10E4D00096428091600290916102A0916202B09197
:10E4E000630280930C0290930D02A0930E02B093EE
:10E4F0000F0220E030E043E060E070E080E291EC69
:10E500000E946FDCE3E4F1E485919491FC01249195
:10E51000222341F03091C00035FFFCCF2093C6008C
:10E520000196F4CFEBEFFDE08491882341F09091C8
:10E53000C00095FFFCCF8093C6003196F5CF409187
:10E540003E0B50913F0B6091400B7091410B25E0C9
:10E5500030E08CED99E00E943042E6EFFDE08491DE
:10E56000882341F09091C00095FFFCCF8093C600B6
:10E570003196F5CF4091420B5091430B6091440B83
:10E580007091450B25E030E08CED99E00E9430421F
:10E59000E1EFFDE08491882341F09091C00095FF68
:10E5A000FCCF8093C6003196F5CF4091460B509139
:10E5B000470B6091480B7091490B25E030E08CEDE2
:10E5C00099E00E943042EFEEFDE08491882341F013
:10E5D0009091C00095FFFCCF8093C6003196F5CF97
:10E5E0000E94C4420C9497989091C00095FFFCCF74
:10E5F0008093C60081918111F7CFB801882777FDFC
:10E600008095982F0F941EBD0E94875FAB01BC01BF
:10E6100022E030E08CED99E00E9431420F5F1F4F05
:10E620000F36110511F40C9497984AE050E0B801A8
:10E630008CED99E00E943D41ECE2F9E0DBCF809166
:10E640002F0B882341F08091300B882321F080919B
:10E65000310B811109C00E94DDC261E088EE9DE0AE
:10E660000E9425C20C94979881E090E09093160246
:10E6700080931502EAECFDE08491882341F09091AB
:10E68000C00095FFFCCF8093C6003196F5CF8091F6
:10E69000C00085FFFCCF8AE08093C6001A821982F1
:10E6A000C090CB1AD090CC1AE090CD1AF090CE1A30
:10E6B00020E030E040EA50E4C701B6010F9483BC8B
:10E6C0000F94EBBC45E0469F9001479F300D11240D
:10E6D000B901882777FD8095982F0F941EBD2B01D7
:10E6E0003C0120E030E04CE052E40F947CBC87FF1A
:10E6F00006C0412C512C2CE0622E22E4722EA70180
:10E700009601C301B2010F947CBC87FF0AC020E0D0
:10E7100030E040EA50E4C301B2010F94A3BB2B01E7
:10E720003C01E6EBFDE08491882341F09091C0002C
:10E7300095FFFCCF8093C6003196F5CF22E030E004
:10E74000B301A2018CED99E00E94314220E030E05B
:10E7500040EF51E4C301B2010F94A2BB20E030E0CE
:10E760004CE852E40F94A3BB0F94EBBC7093D81AFF
:10E770006093D71A84E090E09093800B80937F0B96
:10E7800081E090E090937E0B80937D0BE0918E0B67
:10E79000F0E0EE0FFF1FE956F14C8591949121E0D6
:10E7A000892B09F420E02093820B80E090E0A0EA1E
:10E7B000B1E480933E0B90933F0BA093400BB0933A
:10E7C000410B80E090E0A0E7B2E48093420B90938D
:10E7D000430BA093440BB093450B8AE999E9A9E157
:10E7E000BEE38093460B9093470BA093480BB093E6
:10E7F000490B8AE29BE09F938F93812C912C18E424
:10E80000A12E12E4B12E0AE4C02E0BE0D02E1AE99C
:10E81000E12E19E9F12E09E11EE320E030E040E7A6
:10E8200052E460E070E080EA91E40F946D030F948D
:10E830001C1D0F900F90A30192016091CB1A709153
:10E84000CC1A8091CD1A9091CE1A0F947CBC87FF80
:10E8500007C088EE93E00E94CA5D0E940265EBCF7C
:10E8600060E086EA9FE00F940CC980E090E0A0EAA7
:10E87000B0E48093460B9093470BA093480BB09362
:10E88000490B2091420B3091430B4091440B509126
:10E89000450B60913E0B70913F0B8091400B909126
:10E8A000410BEAE2FBE0FF93EF93812C912CE8E42B
:10E8B000AE2EE2E4BE2EFAE4CF2EFBE0DF2EE12CFA
:10E8C000F12C00EA10E40F946D03E1EAF3E4859182
:10E8D0009591A591B49180933E0B90933F0BA0939B
:10E8E000400BB093410BE5EAF3E425913591459156
:10E8F00054912093420B3093430B4093440B50931D
:10E90000450BE090460BF090470B0091480B10919F
:10E91000490B60913E0B70913F0B8091400B9091A1
:10E92000410BEAE2FBE0FF93EF93812C912CB8E4DA
:10E93000AB2EB2E4BB2E0F946D030F941C1D20E090
:10E9400030E043E060E070E080E89FEB0E946FDC25
:10E950008091460B9091470BA091480BB091490BC9
:10E960008AAF9BAFACAFBDAFE5EBFDE084910F90FC
:10E970000F900F900F904091460B5091470B609174
:10E98000480B7091490B882349F09091C00095FF86
:10E99000FCCF8093C60031968491F5CF8091C00062
:10E9A00085FFFCCF8AE08093C600EEEAFDE084910B
:10E9B000882341F09091C00095FFFCCF8093C60062
:10E9C0003196F5CF22E030E08CED99E00E943042A4
:10E9D000EDEAFDE08491882341F09091C00095FF1D
:10E9E000FCCF8093C6003196F5CF8091C00085FFA3
:10E9F000FCCF8AE08093C6002EEAC22E2FE0D22EF2
:10EA000033E2E32EF12C0FEF1FEF4AE0342EB70173
:10EA1000882777FD8095982F0F941EBD4B015C01D0
:10EA2000E6EAFDE08491882341F09091C00095FFD3
:10EA3000FCCF8093C6003196F5CF4AE050E0B80194
:10EA40006E5F7F4F8CED99E00E943D41E9E9FDE06A
:10EA50008491882341F09091C00095FFFCCF809372
:10EA6000C6003196F5CF8091C00085FFFCCF309273
:10EA7000C600E5E8FDE08491882341F09091C00054
:10EA800095FFFCCF8093C6003196F5CF4AE050E069
:10EA9000B7018CED99E00E943D41E6E7FDE08491ED
:10EAA000882341F09091C00095FFFCCF8093C60071
:10EAB0003196F5CF4AE050E060E070E08CED99E0EF
:10EAC0000E943D41E5E7FDE08491882341F090916B
:10EAD000C00095FFFCCF8093C6003196F5CF8091A2
:10EAE000C00085FFFCCF3092C6000F3FFFEF1F072D
:10EAF00031F0BE016F5F7F4FC6010F94FC4EA50140
:10EB00009401C301B2010F947CBC181664F40F5F2A
:10EB10001F4F25E0E20EF11C32E0C30ED11C053080
:10EB2000110509F074CF280187E2481A88EF580AC6
:10EB3000440C551C380193E0690E711C85E0809FE0
:10EB40001001819F300C112419AE18AEADE22A0ECF
:10EB5000311CC301029705970CF0CBC168AD79ADAC
:10EB6000620D731D882777FD8095982F0F941EBD29
:10EB700022966CAF7DAF8EAF9FAF2297EEE6FDE0A1
:10EB80008491882341F09091C00095FFFCCF809341
:10EB9000C6003196F5CF4AE050E0B3018CED99E024
:10EBA0000E943D41EBE6FDE08491882341F0909185
:10EBB000C00095FFFCCF8093C6003196F5CF8091C1
:10EBC000C00085FFFCCFFAE0F093C60070927E0B88
:10EBD00060927D0B20E030E040EF51E422966CAD76
:10EBE0007DAD8EAD9FAD22970F94A2BB20E030E0AB
:10EBF00040E251E40F9451BF20E030E040EA50E49D
:10EC00000F9483BC20E030E048E452E40F94A3BBAF
:10EC10000F94EBBC7093D81A6093D71A80E090E001
:10EC2000A0EAB1E480933E0B90933F0BA093400B7E
:10EC3000B093410B80E090E0A0E7B2E48093420BF8
:10EC40009093430BA093440BB093450B8AE999E949
:10EC5000A9E1BEE38093460B9093470BA093480B2A
:10EC6000B093490BAAE2BBE0BF93AF93812C912CE8
:10EC7000A8E4AA2EA2E4BA2EBAE4CB2EBBE0DB2E87
:10EC80001AE9E12E19E9F12E09E11EE320E030E056
:10EC900040E752E460E070E080EA91E40F946D0395
:10ECA0000F941C1D0F900F9022962CAD3DAD4EADD4
:10ECB0005FAD22976091CB1A7091CC1A8091CD1ADA
:10ECC0009091CE1A0F947CBC87FF07C088EE93E02A
:10ECD0000E94CA5D0E940265E7CF80E090E0A0EA52
:10ECE000B0E48093460B9093470BA093480BB093EE
:10ECF000490B2091420B3091430B4091440B5091B2
:10ED0000450B60913E0B70913F0B8091400B9091B1
:10ED1000410BAAE2BBE0BF93AF93812C912C18E486
:10ED2000A12E12E4B12E0AE4C02E0BE0D02EE12C6D
:10ED3000F12C00EA10E40F946D03E1EAF3E485910D
:10ED40009591A591B49180933E0B90933F0BA09326
:10ED5000400BB093410BE5EAF3E4259135914591E1
:10ED600054912093420B3093430B4093440B5093A8
:10ED7000450BE090460BF090470B0091480B10912B
:10ED8000490B60913E0B70913F0B8091400B90912D
:10ED9000410BAAE2BBE0BF93AF93812C912CF8E426
:10EDA000AF2EF2E4BF2E0F946D030F941C1D20E0D4
:10EDB00030E043E060E070E080E89FEB0E946FDCB1
:10EDC0002AAD3BAD4CAD5DAD6091460B7091470BEC
:10EDD0008091480B9091490B0F94A2BB2091AA19E6
:10EDE0003091AB194091AC195091AD190F9451BFAE
:10EDF0000F94EBBC7A836983EAE6FDE084910F907F
:10EE00000F900F900F90882349F09091C00095FFCC
:10EE1000FCCF8093C60031968491F5CF8091C000DD
:10EE200085FFFCCFFAE0F093C600E6E5FDE08491B3
:10EE3000882341F09091C00095FFFCCF8093C600DD
:10EE40003196F5CF4091CB1A5091CC1A6091CD1AE2
:10EE50007091CE1A22E030E08CED99E00E943042B1
:10EE6000E7E4FDE08491882341F09091C00095FF94
:10EE7000FCCF8093C6003196F5CF2AAD3BAD4CADAB
:10EE80005DAD6091460B7091470B8091480B90915E
:10EE9000490B0F94A2BBAB01BC0122E030E08CED2A
:10EEA00099E00E943042E6E4FDE08491882341F03D
:10EEB0009091C00095FFFCCF8093C6003196F5CFAE
:10EEC0008091C00085FFFCCFFAE0F093C600BE0140
:10EED0006F5F7F4FC2010F94FC4E22E0420E511C27
:10EEE0003FEF631A730A88AD99AD059699AF88AF65
:10EEF00030CE1092800B10927F0B1092820B61E04B
:10EF000086EA9FE00F940CC9E7E0FDE08491882336
:10EF100041F09091C00095FFFCCF8093C6003196E0
:10EF2000F5CF8091C00085FFFCCF8AE08093C600BA
:10EF3000179A10922F0B169A1092300B149AE09198
:10EF40008E0BF0E0EE0FFF1FED56F14C8591949182
:10EF50000F946DA281E00F94689882E00F94A195C0
:10EF60001092D81A1092D71A0C94979884E690E0D1
:10EF70000E94CA5D91E0E91AF108C1F74AE050E049
:10EF8000B8018CED99E00E943D41F6012491E4E046
:10EF9000FDE0211117C060916C0B70916D0B4AE080
:10EFA00050E08CED99E00E9444410550110911F4A4
:10EFB0000C9497981093290B0093280BF4E6EF2EEE
:10EFC000F12CD4CF3091C00035FFFCCF2093C60088
:10EFD00031962491DECF0F941C1D1092C00B81E05E
:10EFE0008093900B86E50E94EA42882359F0E091D5
:10EFF0009B10F0919C108181893021F08F7D11F060
:10F000000E94004320912F0B8091F81B9091F91BD7
:10F01000222341F02091300B222321F02091310B4B
:10F0200021110FC0029749F00E94DDC261E08DEF0F
:10F030009CE00E9425C20C9497981092900B0C941F
:10F0400097981092620A029721F41092900B0C94F8
:10F050009798F091820B2896FFAF289720917F0B0D
:10F060003091800B2A963FAF2EAF2A9780917D0B6F
:10F0700090917E0B2C969FAF8EAF2C9781E0809362
:10F08000820B81E090E09093800B80937F0B83E173
:10F0900090E090937E0B80937D0B81E00F94A1957F
:10F0A00089ED92E10E9408F80E943EF780E090E02E
:10F0B000A0EAB0E48093460B9093470BA093480BD3
:10F0C000B093490B20E030E040E752E460916002E9
:10F0D0007091610280916202909163020F9483BCEF
:10F0E0004B015C012091420B3091430B4091440B4A
:10F0F0005091450B60913E0B70913F0B8091400BFE
:10F100009091410BEAE2FBE0FF93EF931AE4C12EEA
:10F110001BE0D12EE12CF12C00EA10E40F946D03DA
:10F12000E1EAF3E485919591A591B49180933E0B2A
:10F1300090933F0BA093400BB093410BE5EAF3E4AF
:10F1400085919591A591B4918093420B9093430B37
:10F15000A093440BB093450B62E47BE08EE39BE00D
:10F160000E94184620E030E040EF51E460915802E0
:10F170007091590280915A0290915B020F9483BC66
:10F180004B015C01E090460BF090470B0091480B5F
:10F190001091490B2091420B3091430B4091440B4D
:10F1A0005091450B60913E0B70913F0B8091400B4D
:10F1B0009091410BEAE2FBE0FF93EF930F946D0314
:10F1C0000F941C1D20E030E040EA51E460915802A9
:10F1D0007091590280915A0290915B020F9483BC06
:10F1E0000F94EBBC8B0120E030E040E252E46091F0
:10F1F00060027091610280916202909163020F94AB
:10F2000083BC0F94EBBC7B010E9422D923968FAF65
:10F21000239780E00E9496420F900F900F900F90DE
:10F22000A1EAB3E4BBAFAAAF212C312CC701AA27B6
:10F2300097FDA095BA2F60968CAF9DAFAEAFBFAFD4
:10F240006097C801AA2797FDA095BA2F64968CAF46
:10F250009DAFAEAFBFAF6497C10163E070E00F94A4
:10F2600040C17FAF6EAF99AF88AF9EAD90FF08C031
:10F27000A2E0B0E0E8ADF9ADAE1BBF0BB9AFA8AFEF
:10F280002396FFAD2397FF2379F12114310461F117
:10F290008EAD9FAD880F991F2EAD3FAD820F931F8E
:10F2A000A8ADB9AD8A0F9B1F880F991F8D53904F42
:10F2B0000F9407C9BC01882777FD8095982F0F947C
:10F2C0001EBD2AE037ED43E25CE30F9451BF20916D
:10F2D000DA123091DB124091DC125091DD120F9462
:10F2E000A3BB2B013C0103C0412C512C320180E017
:10F2F00090E0A0EAB0E48093460B9093470BA09374
:10F30000480BB093490B60966CAD7DAD8EAD9FAD53
:10F3100060970F941EBD27966CAF7DAF8EAF9FAFE9
:10F3200027972091420B3091430B4091440B509111
:10F33000450B60913E0B70913F0B8091400B90917B
:10F34000410BAAE2BBE0BF93AF9327968CAC9DAC78
:10F35000AEACBFAC2797EAE4CE2EEBE0DE2EE12C7C
:10F36000F12C00EA10E40F946D030F941C1DEAAD1C
:10F37000FBAD85919591A591B49180933E0B9093AF
:10F380003F0BA093400BB093410BEAADFBAD34961D
:10F3900085919591A591B4918093420B9093430BE5
:10F3A000A093440BB093450B62E47BE08EE39BE0BB
:10F3B0000E94184664966CAD7DAD8EAD9FAD64978E
:10F3C0000F941EBD4B015C01E090460BF090470B83
:10F3D0000091480B1091490B2091420B3091430B47
:10F3E0004091440B5091450B60913E0B70913F0B47
:10F3F0008091400B9091410BAAE2BBE0BF93AF9389
:10F400000F946D030F941C1D0F900F900F900F9091
:10F410002396FFAD2397FF2361F02114310449F0B7
:10F4200020E030E040E85FE3C301B2010F94A2BBEB
:10F4300004C060E070E080E291EC20E030E043E066
:10F440000E946FDC811108C0E0918E0BF0E0EE0F9E
:10F45000FF1FE35EFE4B1FC0C090460BD090470BD2
:10F46000E090480BF090490BA701960160E070E036
:10F4700080EA90E40F94A2BB2DEC3CEC4CEC5DE3F5
:10F480000F947CBC87FF0AC0E0918E0BF0E0EE0F7A
:10F49000FF1FE75EFE4B65907490ABC023962FADC7
:10F4A00023972223B9F0A7019601C301B2010F945B
:10F4B000A2BB9F7720E030E040E85FE30F947FBE7F
:10F4C000181644F4E0918E0BF0E0EE0FFF1FEF5D95
:10F4D000FE4BE1CF6091CB1A7091CC1A8091CD1A7E
:10F4E0009091CE1A0E946E636B017C01E9EEFCE004
:10F4F0008491882341F09091C00095FFFCCF8093C8
:10F50000C6003196F5CF4091460B5091470B609164
:10F51000480B7091490B25E030E08CED99E00E949A
:10F520003042EFEDFCE08491882341F09091C000DF
:10F5300095FFFCCF8093C6003196F5CF25E030E0F3
:10F54000B701A6018CED99E00E943042EEEDFCE09F
:10F550008491882341F09091C00095FFFCCF809367
:10F56000C6003196F5CF8091C00085FFFCCFFAE050
:10F57000F093C60087E02EAD3FAD829F8001839F50
:10F58000100D1124A8ADB9AD0A0F1B1F000F111FDC
:10F59000000F111F07521D4EA70196016091460BE7
:10F5A0007091470B8091480B9091490B0F94A2BB2F
:10F5B000F801618372838383948380917D0B9091A2
:10F5C0007E0B019790937E0B80937D0BFFEF2F1A9C
:10F5D0003F0A81E00F94A1952AAD3BAD285F3F4FD4
:10F5E0003BAF2AAF39E02316310409F035CE612C48
:10F5F000712C80E090E0A0EAB0E48093460B9093F9
:10F60000470BA093480BB093490B2091420B3091CC
:10F61000430B4091440B5091450B60913E0B709110
:10F620003F0B8091400B9091410BEAE2FBE0FF938E
:10F63000EF9327968CAC9DACAEACBFAC2797EAE4B9
:10F64000CE2EEBE0DE2EE12CF12C00EA10E40F943C
:10F650006D030F941C1D0F900F9089E02816310444
:10F6600021F060E0C3010C940C840E94C442EBECD6
:10F67000FCE08491882341F09091C00095FFFCCF7D
:10F680008093C6003196F5CF8091C00085FFFCCFF6
:10F690008AE08093C6000E9426F7EAEBFCE08491A2
:10F6A000882341F09091C00095FFFCCF8093C60065
:10F6B0003196F5CF8091C00085FFFCCF8AE0809322
:10F6C000C60080EC9FE00F94FAC8A82EDE011196C8
:10F6D0003D01B12C32E5932E46E4842EBCE4B9837F
:10F6E0009A828B8282E48C83F30181913F010E9494
:10F6F000EA42882319F00E940D431DC0F1E0AF12C9
:10F7000035C1FB1528F0B11009C08FEB9FE00BC08D
:10F7100022E0B21206C08DEB9FE005C08EEB9FE0A9
:10F7200002C08CEB9FE00F94FAC8682F772767FD23
:10F730007095872F972F611571058105910509F443
:10F7400015C10F941EBD2FE632E143E85AE30F9432
:10F7500051BF6B017C019F7727E139ED4EEC5DE3F2
:10F760000F947FBE18160CF037C0E4EFFFE08491D1
:10F77000882341F09091C00095FFFCCF8093C60094
:10F780003196F5CFE6E9FCE08491882341F0909131
:10F79000C00095FFFCCF8093C6003196F5CF22E0E4
:10F7A00030E0B701A6018CED99E00E943042EDE80F
:10F7B000FCE08491882341F09091C00095FFFCCF3C
:10F7C0008093C6003196F5CF8091C00085FFFCCFB5
:10F7D0008AE08093C600CAC0F2E0BF1609F469C08F
:10F7E00023E0B21609F494C031E0B31689F120E0A9
:10F7F00030E040E05FE3C701B6010F9451BF1B0149
:10F800002C010AED12E1A2019101D80114966D912B
:10F810007D918D919C9117970F94A3BBF801648300
:10F82000758386839783A7019601608171818281A8
:10F8300093810F94A3BBD8016D937D938D939C937B
:10F840001397045E1F4FB3E10E321B07E1F68EC023
:10F8500020E030E040E05FE3C701B6010F9451BF04
:10F860001B012C010EED12E1A2019101F801608152
:10F870007181828193810F94A3BBD8016D937D9395
:10F880008D939C931397A701960114966D917D918A
:10F890008D919C9117970F94A3BBF8016483758396
:10F8A00086839783045E1F4FF3E102331F07E1F65F
:10F8B0005DC020E030E040E05FE3C701B6010F9497
:10F8C00051BF1B012C010AED12E1A2019101D801E7
:10F8D0005C966D917D918D919C915F970F94A3BBE8
:10F8E000F801648F758F868F978FA70196016081CD
:10F8F0007181828193810F94A3BBD8016D937D9315
:10F900008D939D938D01B2E1063E1B07F1F62EC04B
:10F9100020E030E040E05FE3C701B6010F9451BF43
:10F920001B012C0106EF12E1A2019101F801608197
:10F930007181828193810F94A3BBD8016D937D93D4
:10F940008D939D938D01A701960158966D917D91A0
:10F950008D919C915B970F94A3BBF801608F718F81
:10F96000828F938FF3E102301F07F1F6B39424E006
:10F97000B212B4CEECE6FCE08491882341F0909181
:10F98000C00095FFFCCF8093C6003196F5CF8091E3
:10F99000C00085FFFCCF8AE08093C60089ED92E12C
:10F9A0000E9423F8EAE5FCE08491882341F09091DD
:10F9B000C00095FFFCCF8093C6003196F5CF8091B3
:10F9C000C00085FFFCCF8AE08093C60081E0809371
:10F9D000D912EEE3FCE08491882341F09091C000BD
:10F9E00095FFFCCF8093C6003196F5CF8091C00083
:10F9F00085FFFCCF8AE08093C6000E944EF0EDE2C6
:10FA0000FCE08491882341F09091C00095FFFCCFE9
:10FA10008093C6003196F5CF8091C00085FFFCCF62
:10FA20008AE08093C600E0912A0B34E0E39FF00166
:10FA30001124EF52F54E20E030E042E053E46081C3
:10FA40007181828193810F947FBE181694F4809106
:10FA5000BF0B882371F086EA9FE00F94FAC88823D1
:10FA600041F08091D71A9091D81AC29714F00C9453
:10FA7000739981E090E09093160280931502289686
:10FA80008FAD28978093820B2A96AEADBFAD2A9793
:10FA9000B093800BA0937F0B2C96EEADFFAD2C970F
:10FAA000F0937E0BE0937D0B1092900B10928F0BD6
:10FAB00082E00F94A1950C9497988091D912882395
:10FAC00009F49EC0E3E2FCE08491882341F0909128
:10FAD000C00095FFFCCF8093C6003196F5CF4AE079
:10FAE00050E067E070E08CED99E00E943D41E1E27A
:10FAF000FCE08491882341F09091C00095FFFCCFF9
:10FB00008093C6003196F5CF4AE050E067E070E0A0
:10FB10008CED99E00E943D41EEE0FCE08491882369
:10FB200041F09091C00095FFFCCF8093C6003196C4
:10FB3000F5CF4AE050E065E070E08CED99E00E947E
:10FB40003D41ECEFFBE08491882341F09091C000AF
:10FB500095FFFCCF8093C6003196F5CF8091C00011
:10FB600085FFFCCF8AE08093C60000E010E099EFAB
:10FB7000A92E9BE0B92E27EF822E2BE0922EE12CAE
:10FB8000F12C98012F573C4E6901F5018491E9EF62
:10FB9000FBE0882349F09091C00095FFFCCF809353
:10FBA000C60031968491F5CFF601EE0DFF1D41811F
:10FBB00052816381748125E030E08CED99E00E94F0
:10FBC0003042F4E0EF0EF11C2CE1E216F104E9F60C
:10FBD000F4018491E7EFFBE0882349F09091C000A5
:10FBE00095FFFCCF8093C60031968491F5CF0C51E0
:10FBF00011090C33FFEF1F0709F0C1CF0C94979840
:10FC0000E9EDFBE08491882341F09091C00095FFDD
:10FC1000FCCF8093C6003196F5CF8091C00085FF60
:10FC2000FCCF8AE08093C6000C94979881E00E94F4
:10FC30003D470C9497981092F40A0C94979885E499
:10FC40000E94EA42811102C00F941C1D19EB612E23
:10FC500015E0712E02E3802E0BE0902E8EE3A82E8D
:10FC60008BE0B82E512CD3018D913D010E94EA42C8
:10FC70008823D9F1B3E05B120CC00E945743F50111
:10FC800060837183828393838AE49BE00F94C6111F
:10FC90002CC00E945743D4012D913D914D915C9110
:10FCA0000F94A3BBF5016083718382839383E090FB
:10FCB000460BF090470B0091480B1091490B209197
:10FCC000420B3091430B4091440B5091450B609196
:10FCD0003E0B70913F0B8091400B9091410BBAE429
:10FCE000CB2EBBE0DB2E0F941B105394F4E08F0E51
:10FCF000911C24E0A20EB11C34E05312B4CF0C943A
:10FD0000979881E08093F41B0F94A5B36093C80B80
:10FD10007093C90B8093CA0B9093CB0B6091F41B2B
:10FD200084EC9FE00F940CC90C9497988DE40E948A
:10FD3000EA42882311F40C941D97E0919B10F091F6
:10FD40009C10319681918032E9F38930D9F3805348
:10FD50008A30B0F0EAECFBE08491882341F0909186
:10FD6000C00095FFFCCF8093C6003196F5CF8091FF
:10FD7000C00085FFFCCF8AE08093C6000C94979862
:10FD80000E9457430F94EBBC6B3C710511F40C942B
:10FD9000088C0CF0F7C06135710511F40C9486875E
:10FDA0000CF077C06A31710509F447C3D4F56431AA
:10FDB000710509F4DDC294F46131710509F4CCC216
:10FDC00034F46230710508F409C20C94089762316A
:10FDD000710511F40C94B5870C940897673171057F
:10FDE00009F400C37CF46531710509F4F5C266318C
:10FDF000710511F00C9408978CEC9BE00E944EB6B4
:10FE00000C9497986831710509F407C3693171053D
:10FE100011F00C9408978CEC9BE00E9459B60C945E
:10FE200097986F31710509F419C48CF46C31710520
:10FE300009F417C30CF40FC36D31710511F40C9460
:10FE400097986E31710509F43BC30C9408976C3296
:10FE5000710509F4AAC454F46032710509F468C349
:10FE60006A32710509F45AC40C9408976D32710511
:10FE700009F4AAC46F32710511F00C94089784E05C
:10FE800090E090931602809315020F947E6A0C9472
:10FE900097986037710509F4BCC4A4F56C357105F9
:10FEA00011F40C940988A4F46335710511F40C94D1
:10FEB000B08714F40C94AC876435710511F40C947C
:10FEC000B5876535710511F40C94EE870C9408978D
:10FED0006A36710509F4E4C754F46836710509F40B
:10FEE0007AC46936710509F4AAC40C9408976B3674
:10FEF000710511F40C9480876D36710509F4E8C51D
:10FF00000C9408976837710511F40C94FE89C4F4B9
:10FF10006237710511F40C94F68814F40C948C88F3
:10FF20006337710511F40C94B6886737710511F0C9
:10FF30000C940897EDE0F0E4859194910C940F8A6D
:10FF40006E3B710509F46EC65CF46937710511F4F6
:10FF50000C94038A6C38710509F460C40C940897FA
:10FF6000683C710511F40C94768B693C710511F0B5
:10FF70000C94089709EB15E022E9E22E29E1F22E14
:10FF80000C94ED8B673F81E0780711F40C9433906B
:10FF90000CF07EC06C32A1E07A0711F40C94388E1C
:10FFA000C4F5603D710511F40C94128DA4F46D3C00
:10FFB000710511F40C94478C14F40C94258C6E3C50
:10FFC000710511F40C94BE8C6F3C710511F40C9406
:10FFD000DB8C0C9408976D3D710511F40C94AC8D7D
:10FFE00064F4613D710511F40C943A8D6C3D71051A
:10FFF00011F40C949B8D0C940897623E710511F4DA
:020000021000EC
:100000000C94D68D603F710511F40C9497980C9464
:1000100008976036E1E07E07E4F46E35F1E07F0793
:1000200014F00C9497986E3221E0720711F40C943E
:10003000DD8F14F40C94708E6F3281E0780711F428
:100040000C94EC8F6033714011F40C943B8F0C9442
:100050000897643FA1E07A0711F40C9425904CF4C2
:100060006039714011F00C9408970F941C1D0C948A
:100070009798653FF1E07F0711F40C942C90663F50
:10008000714011F00C9408970E9413340C949798C7
:100090006E3833E0730711F40C9446950CF047C0AA
:1000A0006D3B92E0790711F40C949796FCF4683557
:1000B000B2E07B0711F40C9444915CF46D3F714005
:1000C00011F00C9408970F94774FEEEEFFE00C942C
:1000D0003F90693522E0720711F40C9401956A355E
:1000E000724011F40C940F950C940897643883E0D7
:1000F000780711F40C941D956CF46E3BA2E07A071E
:1001000011F40C949A966335734011F40C94519049
:100110000C9408976B38E3E07E0711F40C9420955B
:100120006C38734011F40C9497980C9408976339C9
:1001300023E0720711F40C94B095D4F4603983E095
:10014000780711F40C947B9514F40C94499561395B
:10015000A3E07A0711F40C94AD956239734011F065
:100160000C94089710924A1B0F947A3A0C94979823
:100170006639E3E07E0711F40C9465966CF46439FB
:1001800023E0720711F40C94B6956539734011F4AD
:100190000C9433960C940897603A83E0780709F43E
:1001A00030C2673E734011F00C9408971092DE0A3B
:1001B0000F9417508091871090918810A09189100A
:1001C000B0918A1080938B1090938C10A0938D1017
:1001D000B0938E100E94AD540C94979800919B1090
:1001E00010919C100E5F1F4F80E50E94EA42882309
:1001F00079F00E9457430F94F0BC6B017C01BB2443
:10020000B394611571058105910531F4B12C04C0D9
:10021000B12CC12CD12C760183E50E94EA428823BF
:1002200099F00E94574320E030E04AE754E40F94ED
:1002300051BF0F94F0BC6B017C01AA24A3946115FB
:1002400071058105910509F4A12C6AE270E0C801ED
:100250000F9443C5009711F0DC011C92F801CF0107
:1002600021912032E1F3B11007C0A11005C0222373
:1002700019F00F94D94F06C0E3E7FEE385919491FE
:100280000F94E64F81E00F94B94F0F941C1D0F940B
:10029000A5B36093F00A7093F10A8093F20A9093E9
:1002A000F30AC114D104E104F104F1F00F94A5B3F1
:1002B0004B015C018C0C9D1CAE1CBF1C84E090E0CB
:1002C00090931602809315020F94A5B368157905D3
:1002D0008A059B0510F00C94B5990F946C5181110F
:1002E0000C94B5990C94C0990F946A51882311F419
:1002F0000C94979884E090E09093160280931502F6
:100300000F946C51811109C00F94082A81E00E945A
:10031000A95B80E00F94A195F3CF82E090E09093E9
:100320001602809315028091CE0BE0918E0BF0E0C7
:10033000EE0FFF1F882341F0E35AF04C8591949112
:100340000F94E64F0C949798EF5FF14C8591949140
:100350000F94E64F0C949798E1ECFFE3859194910C
:100360000F94E64F17981698159814980C94979830
:10037000E3EFF0E485919491FC012491222341F074
:100380003091C00035FFFCCF2093C6000196F4CF1A
:100390008091C00085FFFCCF8AE08093C6008CEC82
:1003A0009BE00E9423B5E9EAF0E485919491FC0179
:1003B0002491222341F03091C00035FFFCCF2093DF
:1003C000C6000196F4CF8091C00085FFFCCF8AE083
:1003D0008093C6000C9497988CEC9BE00E9479B5B2
:1003E0000C94979880919B1090919C106AE270E019
:1003F00004960F9443C5009711F0DC011C926091A4
:100400009B1070919C106C5F7F4F21E041E08CEC61
:100410009BE00E9400BB0C9497988CEC9BE00E94A0
:1004200052B60F94A5B36093E80A7093E90A8093DB
:10043000EA0A9093EB0A0C9497988091CF0B88234B
:1004400011F40C94979883E50E94EA4281110C9470
:10045000CA990C9497988CEC9BE00E9404B80C9479
:10046000979880919B1090919C106AE270E004969E
:100470000F9443C58C010097A9F08091A51090912D
:10048000A6106EE470E086559F4E0F9443C560E25F
:1004900070E00F9443C5019690939C1080939B103D
:1004A000F801108260919B1070919C106C5F7F4FDF
:1004B00021E040E08CEC9BE00E9400BB0C949798FC
:1004C0008091CF0B882311F40C94979860E08CEC0A
:1004D0009BE00E9490BA80919B1090919C106AE2E0
:1004E00070E004960F9443C58C010097A9F08091A9
:1004F000A5109091A6106EE470E086559F4E0F9463
:1005000043C560E270E00F9443C5019690939C1040
:1005100080939B10D8011C9260919B1070919C104D
:100520006C5F7F4F8CEC9BE00E94C3B60C94979855
:100530008091CE0B81110F941C1D00919B10109186
:100540009C100C5F1F4F6AE270E0C8010F9443C516
:100550007C0161E270E0C8010F9443C5009719F077
:100560008C010F5F1F4FE114F10411F0F7011082AD
:1005700080E50E94EA42F82E20919B1030919C1059
:100580000217130708F4F12C8091CF0B882311F484
:100590000C94979821E02F2541E0B8018CEC9BE06A
:1005A0000E9400BB83E50E94EA428823B9F02091B3
:1005B0009B1030919C102017310780F40E940D434E
:1005C000AB01BC0140936A0E50936B0E60936C0EAE
:1005D00070936D0E85EB9DE00E94ACA88CEC9BE0C7
:1005E0000E9452B6F1100C9497980F94A5B36093A3
:1005F000E80A7093E90A8093EA0A9093EB0A0C9454
:10060000979880919B1090919C106AE270E00596FB
:100610000F9443C58C010097A9F08091A51090918B
:10062000A6106EE470E086559F4E0F9443C560E2BD
:1006300070E00F9443C5019690939C1080939B109B
:10064000D8011C9260919B1070919C106B5F7F4F42
:100650008CEC9BE00E943EBE0C9497980F94A5B33F
:100660006093E40A7093E50A8093E60A9093E70AA0
:100670000091E80A1091E90A2091EA0A3091EB0A08
:10068000601B710B820B930B28EE33E040E050E0CF
:100690000F9453C1CA01B9012CE330E040E050E0AF
:1006A0000F9453C17F936F933F932F938BEB9BE0FA
:1006B0009F938F93CE0101969F938F930F94CEC6F5
:1006C000EEEEFFE084910FB6F894DEBF0FBECDBF13
:1006D000EEEEFFE0882349F09091C00095FFFCCF3B
:1006E0008093C60031968491F5CFFE0131968191B9
:1006F000882339F09091C00095FFFCCF8093C6000D
:10070000F6CF8091C00085FFFCCF8AE08093C600C1
:10071000CE0101960F94D94F0C94979883E50E94CF
:10072000EA42882311F40C9497980E9457430F943F
:10073000EBBCF62EE72E862F9E2D8C0180E50E94C5
:10074000EA42882331F00F3F110509F010F40C94B0
:10075000DB990DE010E0E1E8F5E0819191918017DF
:10076000910711F40C94979825E0E93BF207A9F75B
:100770000630110539F48F2D9E2D9093290B80930F
:10078000280B04C017FF02C00C94979861E0802FDB
:100790000F9490B56F2D802F0F94C9B56F2D7E2DBE
:1007A000802F0F9478B40C9497988FEF0E943D4758
:1007B00060E070E088EF9FE00F9426C90E94DCD8CB
:1007C0000E946FD90C9497988AE50E94EA420E9491
:1007D0006F510C94979888E690E00E94635C8111B9
:1007E0000C94979883E50E94EA42882371F0009167
:1007F000DF0A0E94574310E0000F111F0752154EE9
:100800000F94EBBCD8016D937C930F9413270C9439
:10081000979863E08DE599E00E94335B83E50E9441
:10082000EA42882311F40C9497980E9457430F943E
:10083000EBBC7093D81A6093D71A0C94979889E6FA
:1008400090E00E94635C81110C949798E5EBFBE0CB
:100850008491882341F09091C00095FFFCCF809354
:10086000C6003196F5CFE091DF0AB4E0EB9FF001CE
:100870001124EF52F54E408151816281738121E054
:1008800030E08CED99E00E943042E2EBFBE0849195
:10089000882341F09091C00095FFFCCF8093C60063
:1008A0003196F5CFE091DF0AF0E0EE0FFF1FE7523F
:1008B000F54E60817181882777FD8095982F0F9480
:1008C0001EBDAB01BC0121E030E08CED99E00E943F
:1008D0003042EEEAFBE08491882341F09091C00021
:1008E00095FFFCCF8093C6003196F5CF4091BF1A9B
:1008F0005091C01A6091C11A7091C21A21E030E083
:100900008CED99E00E943042EBEAFBE08491882371
:1009100041F09091C00095FFFCCF8093C6003196C6
:10092000F5CF6091D71A7091D81A882777FD8095F6
:10093000982F0F941EBDAB01BC0121E030E08CED7F
:1009400099E00E943042E8EAFBE08491882341F07C
:100950009091C00095FFFCCF8093C6003196F5CFF3
:100960004AE050E060E070E08CED99E00E943D418B
:10097000E6EAFBE08491882341F09091C00095FF66
:10098000FCCF8093C6003196F5CF4091D11A50919B
:10099000D21A6091D31A7091D41A21E030E08CED14
:1009A00099E00E943042E3EAFBE08491882341F021
:1009B0009091C00095FFFCCF8093C6003196F5CF93
:1009C0006091D91A7091DA1A882777FD8095982F4F
:1009D0000F941EBDAB01BC0121E030E08CED99E02D
:1009E0000E943042EFE9FBE08491882341F090912E
:1009F000C00095FFFCCF8093C6003196F5CF809163
:100A0000DF0A90E00F9494244AE050E0BC018CEDA2
:100A100099E00E943D41EAE9FBE08491882341F09E
:100A20009091C00095FFFCCF8093C6003196F5CF22
:100A30008FEF9FEF0F9494244AE050E0BC018CEDBF
:100A400099E00E943D41E6E9FBE08491882341F072
:100A50009091C00095FFFCCF8093C6003196F5CFF2
:100A60004091CB1A5091CC1A6091CD1A7091CE1A48
:100A700021E030E08CED99E00E943042E2E9FBE0B9
:100A80008491882341F09091C00095FFFCCF809322
:100A9000C6003196F5CF4091C51A5091C61A6091A3
:100AA000C71A7091C81A21E030E08CED99E00E94DD
:100AB00030428091C00085FFFCCF8AE08093C60061
:100AC00081E090E090931602809315020C94019AB5
:100AD0008DE690E00E94635C81110C949798E09100
:100AE0008E0BF0E0EE0FFF1FE35AFF4B85919491C0
:100AF0000F94E64F81E090E09093860B8093850BF6
:100B00008091F41B882321F081E090E00F94A05F96
:100B100083E50E94EA42882391F00091DF0A0E9457
:100B2000574310E0000F111F0752154E0F94EBBCF6
:100B3000F8017183608381E08093060215C082E52D
:100B40000E94EA42882381F00091DF0A0E94574305
:100B500010E0000F111F0752154E0F94EBBCD80187
:100B60006D937C93109206020F9413270F94A5B3F4
:100B70006B017C010091DF0A10E0F801EE0FFF1F0E
:100B8000E752F54E60817181882777FD8095982F17
:100B90000F941EBDF801EE0FFF1FEE0FFF1FEF5267
:100BA000F54E11E020813181428153810F947FBE47
:100BB00018160CF010E01093DD0A81E090E090939D
:100BC0001602809315021092190BC701B6010E94FC
:100BD000EC5DE0918E0BF0E0EE0FFF1FE75AFF4B4C
:100BE000859194910F94E64F82E090E090931602E5
:100BF000809315029093860B8093850B8091F41B54
:100C0000882321F082E090E00F94A05F0F94A5B3B9
:100C10006093F00A7093F10A8093F20A9093F30ABA
:100C20000C949798E0918E0BF0E0EE0FFF1FEB5DB8
:100C3000FE4B859194910F94E64F83E090E0909362
:100C4000860B8093850B8091F41B882321F081E033
:100C500090E00F94A05F83E50E94EA42882361F050
:100C60000E9457430F94EBBC7093D81A6093D71A25
:100C700081E0809306020FC082E50E94EA42882349
:100C800051F00E9457430F94EBBC7093D81A6093B5
:100C9000D71A109206020F94A5B34B015C01109273
:100CA000190B6091D71A7091D81A882777FD809513
:100CB000982F0F941EBD11E02091BF1A3091C01AD9
:100CC0004091C11A5091C21A0F947FBE18160CF0B1
:100CD00010E01093DD0A81E090E09093160280937B
:100CE00015020FE81BE07BE8E72E7BE0F72EE7E834
:100CF000CE2EEBE0DE2EFAE07F2E8091DD0A6091B1
:100D0000D71A7091D81A882309F490C08091190BD2
:100D100081118CC0882777FD8095982F0F941EBD78
:100D20002091BF1A3091C01A4091C11A5091C21A35
:100D30000F947FBE18160CF090C00F94A5B36819DD
:100D400079098A099B09693E73408105910508F478
:100D500064C08091F41B81115CC0E0912A0B24E0F7
:100D6000E29FF0011124EF52F54E408151816281E2
:100D70007381F8018491EFE8FBE0882349F09091BA
:100D8000C00095FFFCCF8093C60031968491F5CFCB
:100D900022E030E08CED99E00E943042F70184912E
:100DA000EBE8FBE0882349F09091C00095FFFCCF71
:100DB0008093C60031968491F5CF60912A0B70E044
:100DC0004AE050E08CED99E00E943D41F6018491AB
:100DD000E7E8FBE0882349F09091C00095FFFCCF45
:100DE0008093C60031968491F5CF4091BF1A5091FF
:100DF000C01A6091C11A7091C21A21E030E08CEDE6
:100E000099E00E9430428091C00085FFFCCF709233
:100E1000C6000F94A5B34B015C010F94082A80E033
:100E20000E94A95B80E00F94A19567CF882777FD8A
:100E30008095982F0F941EBD2091BF1A3091C01A33
:100E40004091C11A5091C21A0F947CBC87FF05C013
:100E500080910602882309F470CFE0918E0BF0E0B8
:100E6000EE0FFF1FE75DFE4B859194910F94E64FC7
:100E700082E090E0909316028093150284E090E067
:100E80009093860B8093850B0F94A5B36093F00A23
:100E90007093F10A8093F20A9093F30A0C94979856
:100EA00083E50E94EA42882319F10E94574320E01B
:100EB00030E0A9010F947CBC87FD0FC00E9457430E
:100EC00020E030E04FE753E40F947FBE181644F063
:100ED0000E9457430F94EBBC05C060E070E002C075
:100EE0006FEF70E07093290B6093280B0C94979828
:100EF0008FEF90E09093290B8093280B0C94979898
:100F00001092290B1092280B0C9497980F94142789
:100F10000F941C1D149A0F949E1D1092290B109271
:100F2000280B68EE73E080E090E00F94D4B3109249
:100F30001702EFEBFFE34591549125E83BE063E8AE
:100F40007BE081EA94E00E9409CA0F94E64F80E0BA
:100F50000F94A1950C9497981092C70B0C949798A6
:100F600081E08093C70B0C94979883E50E94EA4236
:100F7000882399F00E94574320E030E04AE754E488
:100F80000F9451BF0F94F0BC609308027093090254
:100F900080930A0290930B021DC088E50E94EA42EA
:100FA00081110C94E29989E50E94EA4281110C9426
:100FB000E2998AE50E94EA4281110C94E29985E463
:100FC0000E94EA4281110C94E2990F941C1D149A1C
:100FD0000F949E1D10927C0B0C94979883E50E94B1
:100FE000EA42882311F40C9497980E94574320E01A
:100FF00030E04AE754E40F9451BF0F94F0BC609383
:10100000EC0A7093ED0A8093EE0A9093EF0A0C9429
:10101000979829EB35E039AF28AF02EA19E142EBA6
:10102000C42E49E1D42E52E6E52E59E1F52E312C9D
:10103000A8ADB9AD8D91B9AFA8AF0E94EA4288239F
:1010400009F45CC0B3E03B1252C00E9457432B012D
:101050003C0120E030E040EA51E40F947CBC87FF83
:101060003FC0A3019201F801608171818281938167
:101070000F9483BC4B015C019B01AC016091821910
:101080007091831980918419909185190F9451BFA3
:1010900060938219709383198093841990938519B2
:1010A000A5019401D6016D917D918D919C910F9434
:1010B00051BFF6016083718382839383D7016D9161
:1010C0007D918D919C910F941CBDA50194010F946D
:1010D00051BF0F94F0BCF7016083718382839383C7
:1010E000D8014D925D926D927C92139707C00E9439
:1010F0005743F801608371838283938333940C5F39
:101100001F4FF4E0CF0ED11C24E0E20EF11C34E0BE
:1011100033128ECF0C94979883E50E94EA4288237D
:1011200031F00E940043809310020C949798EEEEE9
:10113000FFE08491882341F09091C00095FFFCCF9F
:101140008093C6003196F5CF4091100250E060E0E8
:1011500070E08CE79BE00E9454478091C00085FFBF
:10116000FCCF8AE08093C6000C94979886E50E9495
:10117000EA428823B9F00F94E8AFFC0124912223BE
:1011800041F03091C00035FFFCCF2093C60001969E
:10119000F4CF8091C00085FFFCCF8AE08093C60029
:1011A0000C94979885E50E94EA42882369F0809123
:1011B0009B1090919C10019690939C1080939B1093
:1011C0000F9459B20C949798E3E1F0E485919491CF
:1011D000FC012491222311F40C9497983091C000C3
:1011E00035FFFCCF2093C6000196F2CFE9E7FBE084
:1011F0008491882341F09091C00095FFFCCF8093AB
:10120000C6003196F5CF40913E0B50913F0B609157
:10121000400B7091410B22E030E08CED99E00E9490
:101220003042E5E7FBE08491882341F09091C000D3
:1012300095FFFCCF8093C6003196F5CF4091420BCD
:101240005091430B6091440B7091450B22E030E0CC
:101250008CED99E00E943042E1E7FBE08491882325
:1012600041F09091C00095FFFCCF8093C60031966D
:10127000F5CF4091460B5091470B6091480B709110
:10128000490B22E030E08CED99E00E943042EDE61F
:10129000FBE08491882341F09091C00095FFFCCF42
:1012A0008093C6003196F5CF40914A0B50914B0B7D
:1012B00060914C0B70914D0B22E030E08CED99E089
:1012C0000E943042E3ECF0E485919491FC0124917A
:1012D000222341F03091C00035FFFCCF2093C6009F
:1012E0000196F4CF80E00F947D1D0F941EBD2091D8
:1012F000A2193091A3194091A4195091A5190F94E6
:1013000083BCAB01BC0122E030E08CED99E00E948F
:101310003042E9E6FBE08491882341F09091C000DF
:1013200095FFFCCF8093C6003196F5CF81E00F94F6
:101330007D1D0F941EBD2091A6193091A7194091D3
:10134000A8195091A9190F9483BCAB01BC0122E0EC
:1013500030E08CED99E00E943042E5E6FBE08491BC
:10136000882341F09091C00095FFFCCF8093C60088
:101370003196F5CF82E00F947D1D0F941EBD209114
:10138000AA193091AB194091AC195091AD190F9435
:1013900083BCAB01BC0122E030E08CED99E00E94FF
:1013A0003042E1E6FBE08491882341F09091C00057
:1013B00095FFFCCF8093C6003196F5CF83E00F9464
:1013C0007D1D0F941EBD2091AE193091AF19409133
:1013D000B0195091B1190F9483BCAB01BC0122E04C
:1013E00030E08CED99E00E9430428091C00085FF92
:1013F000FCCF8AE08093C6000C94979880E00F940D
:10140000A1130C94979881E00F94A1130C949798D2
:101410003091C00035FFFCCF2093C6000196FC013F
:1014200024912111F5CF8091C00085FFFCCF8AE087
:101430008093C600E7E1FEE385919491FC0124913D
:10144000222341F03091C00035FFFCCF2093C6002D
:101450000196F4CF1E9B10C0EDEAF0E485919491C3
:10146000FC0124912223C1F03091C00035FFFCCF54
:101470002093C6000196F4CFEBEAF0E485919491B5
:10148000FC012491222341F03091C00035FFFCCFB4
:101490002093C6000196F4CF8091C00085FFFCCF59
:1014A0008AE08093C600E9E1FEE385919491FC0116
:1014B0002491222341F03091C00035FFFCCF2093CE
:1014C000C6000196F4CF8091060182FF10C0EDEABC
:1014D000F0E485919491FC0124912223C1F0309194
:1014E000C00035FFFCCF2093C6000196F4CFEBEA95
:1014F000F0E485919491FC012491222341F03091F4
:10150000C00035FFFCCF2093C6000196F4CF809138
:10151000C00085FFFCCF8AE08093C600EBE0FEE3CD
:1015200085919491FC012491222341F03091C000D7
:1015300035FFFCCF2093C6000196F4CF1D9B10C051
:10154000EDEAF0E485919491FC0124912223C1F00D
:101550003091C00035FFFCCF2093C6000196F4CF38
:10156000EBEAF0E485919491FC012491222341F06F
:101570003091C00035FFFCCF2093C6000196F4CF18
:101580008091C00085FFFCCF8AE08093C600EDE02B
:10159000FEE385919491FC012491222341F0309146
:1015A000C00035FFFCCF2093C6000196F4CF809198
:1015B000060187FF10C0EDEAF0E485919491FC01EB
:1015C00024912223C1F03091C00035FFFCCF20933D
:1015D000C6000196F4CFEBEAF0E485919491FC010A
:1015E0002491222341F03091C00035FFFCCF20939D
:1015F000C6000196F4CF8091C00085FFFCCF8AE041
:101600008093C600E5E0FEE385919491FC0124916E
:10161000222341F03091C00035FFFCCF2093C6005B
:101620000196F4CF1C9B10C0EDEAF0E485919491F3
:10163000FC0124912223C1F03091C00035FFFCCF82
:101640002093C6000196F4CFEBEAF0E485919491E3
:10165000FC012491222341F03091C00035FFFCCFE2
:101660002093C6000196F4CF8091C00085FFFCCF87
:101670008AE08093C600E7E0FEE385919491FC0147
:101680002491222341F03091C00035FFFCCF2093FC
:10169000C6000196F4CF019910C0EDEAF0E48591FF
:1016A0009491FC0124912223C1F03091C00035FFB8
:1016B000FCCF2093C6000196F4CFEBEAF0E48591CD
:1016C0009491FC012491222341F03091C00035FF18
:1016D000FCCF2093C6000196F4CF8091C00085FF17
:1016E000FCCF8AE08093C6000C94979880912A0BD7
:1016F0008093DF0A84E50E94EA42882329F10E9450
:1017000057430F94F0BC6093DF0A6623E9F0EEEED6
:10171000FFE08491882341F09091C00095FFFCCFB9
:101720008093C6003196F5CFEBE0F0E4A591B4913B
:101730008D91882311F40C9497989091C00095FF97
:10174000FCCF8093C600F4CF84E40E94EA42882351
:1017500011F40C9497980E94574320E030E0A901BF
:101760000F947CBC811103C010924E0B32C00091CB
:10177000DF0A10E00E945743F801EE0FFF1FEE0F43
:10178000FF1FEC5BFD4F6083718382839383E09046
:101790004402F0904502009146021091470220E079
:1017A00030E0A901B701C8010F947CBC811104C0CD
:1017B000E12CF12C00E410E4C701D801809344022D
:1017C00090934502A0934602B093470281E0809334
:1017D0004E0B0E94B85D0C949798D8018D918D01A5
:1017E0000E94EA42882349F00E9457430F94F0BCBC
:1017F000F7016083718382839383F4E0EF0EF11C21
:1018000025E00D3B120749F70F94F8110C949798B7
:1018100009EB15E092EBE92E99E1F92ED8018D91B3
:101820008D010E94EA42882339F00E945743F70154
:101830006083718382839383F4E0EF0EF11C25E0D3
:101840000D3B120759F70C94979883E50E94EA42E2
:10185000882351F00E94574360938A1970938B1923
:1018600080938C1990938D1984E50E94EA42882315
:1018700011F40C9497980E945743609386197093C3
:10188000871980938819909389190C94979883E508
:101890000E94EA42882351F00E94574360938E19B8
:1018A00070938F19809390199093911984E50E94F9
:1018B000EA42882351F00E94574360937219709353
:1018C0007319809374199093751982E40E94EA4207
:1018D000882361F00E9457430F94F0BC6093C219B3
:1018E0007093C3198093C4199093C51988E50E9419
:1018F000EA42882391F00E94574360937A197093CB
:101900007B1980937C1990937D196093761970935D
:101910007719809378199093791989E50E94EA42A2
:10192000882351F00E94574360937A1970937B1972
:1019300080937C1990937D198AE50E94EA4288235E
:1019400051F00E94574360937E1970937F198093E2
:1019500080199093811985E40E94EA42882311F44A
:101960000C9497980E94574360938219709383193F
:1019700080938419909385190C94979809EB15E03E
:1019800082E3E82E8BE0F82ED8018D918D010E9424
:10199000EA42882339F00E945743F701608371833C
:1019A00082839383F4E0EF0EF11C25E00C3B1207D9
:1019B00059F70C94979883E50E94EA42882351F0E6
:1019C0000E9457436093240270932502809326025D
:1019D0009093270286E40E94EA42882381F00E94C5
:1019E000574320E030E040E752E40F9483BC60931B
:1019F0001C0270931D0280931E0290931F028AE5C1
:101A00000E94EA42882311F40C9497980E9457434D
:101A10006093220B7093230B8093240B9093250BE0
:101A20000C94979883E50E94EA42882351F00E9423
:101A3000574360931E0B70931F0B8093200B909362
:101A4000210B86E40E94EA42882311F40C949798B3
:101A50000E94574320E030E040E752E40F9483BCFB
:101A6000609318027093190280931A0290931B02DC
:101A70000C94979883E50E94EA42882311F40C9411
:101A800097980E9457430F94EBBC6115710551F074
:101A90006130710569F481E08093270B1092260B69
:101AA0000C9497981092270B1092260B0C949798F1
:101AB000EEEEFFE08491882341F09091C00095FF05
:101AC000FCCF8093C6003196F5CFE1E8FEE3859127
:101AD0009491FC012491222341F03091C00035FF04
:101AE000FCCF2093C6000196F4CFE091A510F091B1
:101AF000A610E655FF4E8191882339F09091C000E1
:101B000095FFFCCF8093C600F6CFECE5FBE0849117
:101B1000882341F09091C00095FFFCCF8093C600D0
:101B20003196F5CF8091C00085FFFCCF8AE080938D
:101B3000C6000C94979883E50E94EA42882311F42A
:101B40000C9497980E9457430F94EBBC70935702E4
:101B5000609356020C94979883E50E94EA4288238A
:101B600011F40C9497980E9457430F94EBBC6B01AF
:101B70007C0184E50E94EA42882391F08DED90E09B
:101B80000E94635C81110C949798E091DF0AF0E069
:101B9000EE0FFF1FEE5AFD4FD182C0820C94979832
:101BA000D0925502C09254020C94979880E50E94FE
:101BB000EA42882311F40C9497980E9457430F949B
:101BC000EBBCD62E062F172F83E50E94EA4288230E
:101BD00031F00E9457430F94EBBC7B0103C0EE240D
:101BE000EA94FE2CC7010196039710F00C94979885
:101BF000E1E8F5E0819191918017910711F40C943F
:101C0000979825E0E93BF207A9F717FF02C00C946B
